:020000040800F2
:1000000000000110211F0808552B00084DB50208FB
:10001000C11F0808C11F0808C11F08080000000010
:100020000000000000000000000000002948000857
:100030002D48000800000000314800088115010823
:10004000C11F0808C11F0808C11F0808C11F0808F0
:10005000C11F0808C11F0808F1D20008F5D2000826
:10006000C11F0808F9D20008FDD20008213200089B
:1000700035320008493200085D320008713200084C
:100080008532000899320008C11F0808C11F0808FE
:10009000C11F0808C11F0808C11F080801D30008B4
:1000A000CD300008F53000081D310008B9300008D7
:1000B00045310008593100086D310008C11F08089A
:1000C000C11F0808C11F0808C11F0808C11F080870
:1000D000C11F0808D92C0008E52C0008C11F08081A
:1000E00005D30008C11F080835480008A9310008D9
:1000F000D1310008F931000895310008AD3200080F
:10010000C11F0808B536000881310008C11F080862
:10011000F12C0008C11F0808C11F0808C11F0808EA
:10012000C1320008D5320008E9320008FD3200086B
:1001300011330008C11F0808C11F0808C11F0808A3
:10014000C11F0808C11F0808C11F0808814800080E
:1001500025330008393300084D330008FD2C000812
:10016000C11F0808C11F0808C11F0808C11F0808CF
:10017000C11F0808C11F0808C11F0808C11F0808BF
:08018000C11F0808C11F080897
:10019000D0E907239A423CBFC1685218D01A704771
:1001A000D0E9092300699A4238BF1218D31A0138DE
:1001B000C01A7047D0E90902101AB0FA80F040095D
:1001C000704700BF0246036A4069D168C05C0133D2
:1001D0008B4228BF00231362704700BF436A8269C5
:1001E000D154436A0169426B01338B4228BF00231B
:1001F0004362D36843F08003D3607047436B188831
:1002000010F0100002D01A889B880120704700BFB0
:10021000436B99891A88890610B504460AD592B2AB
:10022000900607D5E26A002A2AD09888216B80B20E
:100230009047636B99891A88090692B210D5100607
:100240000ED5D4E909128A4215D0A1692069895CCA
:100250000132C9B29980B2FBF0F100FB1122A26217
:10026000998A1A88C90592B204D5D20744BF4FF6BD
:10027000F7721A8010BDDA6822F08002DA60EFE7C8
:100280009B88E2696169DBB28B54E269E168636B68
:100290000132B2FBF1F001FB1022E261CAE700BFBC
:1002A000036942681F2B10B423D95168203B4FF0DB
:1002B000200C0CFA03F3194218D08169087C03283A
:1002C00013D000240C744868C968046890F805C00D
:1002D0008868194931F81CC0A18989B221EA0C014A
:1002E000A181016821F001010160D3605DF8044B38
:1002F000704711684FF0200C0CFA03F31942F5D047
:100300008169087C032813D000240C744868C968EC
:10031000046890F805C08868074931F81CC0A189B5
:1003200089B221EA0C01A181016821F0010101607B
:100330005DF8044B93607047105208084A1C10B4D3
:1003400018BF4FF0450C494C08BF4FF0800C4FF4DC
:10035000003300E00BB3626B12EA0C0F03F1FF33C2
:10036000F8D0002924DD626B54071DD403291FD067
:100370003E4B5A6BD2071FD402291BD01A69D2B246
:1003800082421DD101295B691CD0062912D113F4C8
:10039000604F43D1364A13600CE0002904DD636BE3
:1003A0005B0701D40329E3D103205DF8044B7047B8
:1003B000002BF9D00020F8E701205DF8044B7047CE
:1003C0001020F2E72B4A1A40002AF3D0002B31DB31
:1003D0005C002DD4980031D4D9002DD41A0131D429
:1003E0005C012DD4D80137D419021DD45A02E7D4A8
:1003F0009C022DD4D80229D4190317D45A0323D42C
:100400009C0331D4D8032DD4190429D45A0425D4FB
:100410009C041FD41807CDD51A20C6E7990405D42B
:100420005A04CDD41B04C5D50F20BEE71320BCE76A
:100430000920BAE71C20B8E70B20B6E70A20B4E78A
:100440000D20B2E70C20B0E71420AEE71220ACE795
:100450001120AAE71920A8E70E20A6E71820A4E794
:100460001720A2E71620A0E715209EE7002C0140E8
:10047000C81E002008E0FFFDF8B5154DEB6A93B1EA
:10048000696B0129044614D0124BDA6A22F0080283
:10049000DA6240F2FF5100229963EA62236823F096
:1004A00001032360F8BD0B4AD36B43F48073D3631D
:1004B000F8BD084E40F2FF570023B763B36040F227
:1004C0004C43F3600C20FFF739FFB763DCE700BF54
:1004D000C81E0020002C0140B54BD3E9011270B5B5
:1004E0008C0F83F83840C1F3836483F83940C1F33B
:1004F000016483F83A40100EC1F3074483F83B408F
:100500000001C1F30724C9B283F83C4083F83D10D1
:10051000D887D98F93F89050C2F3035089B2014322
:10052000C2F30344D987C2F3C03083F84040C2F31A
:100530004031C2F3803483F84100012D83F84240FA
:100540004FF0000083F84310C2F3003183F84410E9
:10055000C2F3072CD96883F8450040F2D680022DFB
:1005600000F0B0802A204FEA4C0C0CF07E0C83F88F
:10057000514083F852C093F85240C1F3C012144363
:100580001A6983F8524001F07F01D40F83F85310A9
:1005900083F85440910DC2F3417483F8554001F043
:1005A0000C01C2F3826483F8564083F8571093F825
:1005B0005710C2F381542143C2F3405583F85710BA
:1005C00083F85850002583F85950C2F3004583F84A
:1005D0005A50C2F3C03583F85B50C2F3803583F8BC
:1005E0005C50C2F3403583F85D505C69C2F300355E
:1005F00083F85E50C2F3812583F85F50C4F307414E
:10060000C2F30125C2F3460283F860504FF0010C9B
:1006100083F861200902220E83F862C083F8642007
:10062000A3F86610B3F86610C4F3072289B2114329
:100630002406A3F8661099699C669A6E0C0E42EA2D
:1006400004429A669C6E0A0A02F47F4222439A662A
:100650009D6EDA69C1F307242C43C9B29C6683F806
:100660006C10110E83F86D10110C090619671C6FC0
:10067000110201F47F0121431967196F120292B22E
:100680000A431A67196F1A6A41EA1261196793F8E7
:100690007410C2F30354214383F87410110A01F457
:1006A0007061A3F87610B3F87610C2F3072489B20C
:1006B0002143C2F34602A3F8761083F8782083F82A
:1006C00079C070BD120402F47C129A649A6C0C0E0C
:1006D00042EA04229A649C6CC1F3074222439A6462
:1006E0009A6C013240F10004A40244EA925492024E
:1006F000C3F880204FF40072C3F88440C1F3072C84
:10070000C3F88820C1F380342DE74FEA8C2C0CF419
:1007100040649C649C6C920002F47F7222439A6451
:100720009D6CC1F3C26445EA91759D6483F84C40A9
:10073000C1F3026483F84D40CA0BC1F3425483F8FD
:100740004E4002F00602C1F3824483F84F4083F822
:10075000502093F85020C1F3C034224383F8502036
:100760009C6C93F850E093F840500EF1020E012279
:1007700002FA05F502FA0EF2D617A2FB052E05FBCA
:1007800006EE04FB0EEE0134A2FB0424A644520A3A
:1007900042EACE52C3F880204FEA5E22C1F3072C12
:1007A000C3F88850C3F88420C1F38034DBE600BF6F
:1007B000C81E002038B50D4B0D4C1A6840F2FF558D
:1007C00040F24D43A5630121A2600D20E360FFF7D5
:1007D000B5FDA56340B96069C0F34320A0F10400F2
:1007E000B0FA80F0400938BD002038BDC81E002096
:1007F000002C01402F4B1A68910102D59A6D5207C7
:100800004BD42C4B1A68500202D5DA6E11063CD438
:10081000284B1A68D20102D59A6D90072DD4254B2A
:100820001A68510102D59A6D120717D4214B1A6824
:10083000120112D59A6DD0060FD59A6D510334D49A
:100840009A6DD20503D49A6D22F010029A65194B65
:1008500019484FF000629A600EE670479A6D500397
:1008600007D49A6DD10503D49A6D22F008029A65D7
:10087000104B4FF080629A60D8E79A6D4FF080710C
:1008800022F002029A659960C9E7DA6E4FF480019E
:1008900022F08002DA669960BAE79A6D4FF0007133
:1008A00022F004029A659960ABE74FF000629A600B
:1008B000704700BF0064024058640240384B5A68D9
:1008C000110303D5D3F8A02052075BD4344B5A68E8
:1008D000D00303D5D3F8B420110649D4304B5A685D
:1008E000520303D5D3F8A020900737D42C4B5A6875
:1008F000D10203D5D3F8A02012071CD4284B5A6884
:10090000920217D5D3F8A020D00613D5D3F8A02093
:10091000510341D4D3F8A020D20505D4D3F8A020A8
:1009200022F01002C3F8A0201D4B1E484FF4001205
:10093000DA60A1E57047D3F8A02050030AD4D3F8B9
:10094000A020D10505D4D3F8A02022F00802C3F8D6
:10095000A020134B4FF48012DA60CFE7D3F8A02029
:100960004FF4802122F00202C3F8A020D960BDE735
:10097000D3F8B4204FF4803122F08002C3F8B420C1
:10098000D960ABE7D3F8A0204FF4002122F0040295
:10099000C3F8A020D96099E74FF40012DA607047DD
:1009A00000640240A064024082B00922274B8DF807
:1009B0000720DA68D00319D4DA68D10640D4DA689F
:1009C000D20541D4DA6812F0E00F3BD1DB6813F0B6
:1009D000020F0CBF092308238DF807309DF807305C
:1009E000012B0AD09DF8070002B0704701238DF853
:1009F00007309DF80730012BF4D1144A12E0D36878
:100A0000DB0519D4D36813F0E00F17D1D36813F0C6
:100A1000020F0CBF092308238DF807309DF807301B
:100A2000012BDFD1D168C8034FF00103F4D4D368A0
:100A3000D906E4D50623EFE70223EDE70723EBE72A
:100A40000623D4E70723D2E70223D0E7003C024085
:100A5000024B01F001011970704700BF0000002037
:100A6000704700BF704700BF704700BF012070474C
:100A7000044BD3F89400D3F89830C01AC0F30A009E
:100A8000704700BFC81E0020074BD3F89C0000B978
:100A90007047D3F89C30052B03D1044B1878C0B2B3
:100AA00070470020704700BFC81E002000000020D3
:100AB000012380F849307047064BD3F8A000D3F8E3
:100AC000A430984234BF03F1FF3303F2FF73181AC6
:100AD000704700BFC81E002010B5D0F8E8350446A6
:100AE0001B699847032384F81231002010BD00BF12
:100AF00008B5042290F81211D0F8E83580F81311E7
:100B000080F81221DB689847002008BD08B5D0F8AE
:100B1000E435DB6903B19847002008BD08B5D0F87B
:100B2000E4351B6A9847002008BD00BF08B5D0F81F
:100B3000E4355B6A9847002008BD00BF70B50378B4
:100B400005460E461446DBB1013080F0C3FB431C62
:100B5000DBB201335B00DAB223800323327073709F
:100B60002C7864B12846022300215A1CD2B2F454D6
:100B7000B15410F8014F0233DBB2002CF5D170BD37
:100B800002221346E8E700BF10B5074C6068FF2853
:100B900007D00649D1F8A820AC3100F08FF8FF2328
:100BA0006360002010BD00BF00000020C81E0020B0
:100BB000432301480B80704708000020122301489E
:100BC0000B8070474C000020042301480B807047C5
:100BD0006000002010B5044C04480A462146FFF787
:100BE000ADFF204610BD00BF7C1F00201CFC080884
:100BF00010B5044C04480A462146FFF79FFF2046E3
:100C000010BD00BF7C1F002030FC080810B5044C4C
:100C100004480A462146FFF791FF204610BD00BF59
:100C20007C1F002038FC080810B5044C04480A4614
:100C30002146FFF783FF204610BD00BF7C1F002028
:100C400044FC080810B5044C04480A462146FFF746
:100C500075FF204610BD00BF7C1F002050FC080817
:100C6000704700BF704700BF704700BF704700BFAC
:100C7000704700BF024B0022C3F89C20704700BFA2
:100C8000C81E0020704700BF074B00200522C3F894
:100C90009C20C3F8B401C3F89400C3F8B801C3F8AA
:100CA000980083F8BC017047C81E0020024B00204A
:100CB000C3F89C00704700BFC81E0020212838B52B
:100CC0000C4626D0222816D0202812D189B1072A16
:100CD0000FD1174DD5F8B83113B1096800209847E6
:100CE0002168A288A379C5F8C011A5F8C42185F8A8
:100CF000C631002038BD0029FBD0022AF9D10C4AA8
:100D0000D2F8B431002BF4D00988D2F8C801984742
:100D1000EFE70029EDD0072AEBD1054BD3F8C0212E
:100D20000A60B3F8C4218A8093F8C6318B71E0E77A
:100D3000C81E00202DE9F8431B4DD5F89440C4F59A
:100D4000006888450E4607461BD305F5E67020442B
:100D50003946324684F00EF83444C4F30A04C5F828
:100D60009440D5F8983003F2FF731B1BC3F30A03BA
:100D7000802B9DBF012385F8BC3102200020BDE8F7
:100D8000F88305F5E679014609EB0400A4F5006453
:100D90004246344483F0EEFF07EB08012246484602
:100DA00083F0E8FFDBE700BFC81E0020034B93F889
:100DB000F009003818BF0120704700BFC81E00208E
:100DC00070B5124D124C296840F2FF5640F24D4367
:100DD0000022A6630D20A160C5F8EC290121E36083
:100DE000FFF7ACFAA66320B96369C3F34323042B6E
:100DF00008D0D5F8243AC5F8E039092385F8F03948
:100E0000002070BD85F8F039022070BDC81E00209A
:100E1000002C014070B50E4D95F8F039042B0446B6
:100E20000E460BD0082B07D1D5F8E83983420CD0F9
:100E3000FFF7C6FF022801D0012070BD082385F806
:100E4000F039C5F8EC69C5F8E849022070BD00BF6B
:100E5000C81E0020034B93F8F009032894BF00201C
:100E600001207047C81E002000487047BC280020A1
:100E700030B4184B00209C7B14B11D688D4206D005
:100E80000130082803F11003F5D130BC7047D2B10E
:100E9000114B03EB40218A4211D0104B93F8B4213F
:100EA00012B9012283F8B4210D4B01225A7000F5CA
:100EB000817003EB001301229A7130BC7047022C41
:100EC000EBD1183BF3E7064B00F5817003EB001301
:100ED0009A71DAE7B45B0020B44B00209C5B0020E1
:100EE0009C4B002030B41D4C002384F8A03004F14A
:100EF000180004E00133082B00F110001ED0056833
:100F00008D42F7D190F80EC0BCF1030FF2D1BAB107
:100F1000134901EB4320824209D094F8B42112B95D
:100F2000012284F8B4210F4901224A7000E01839E7
:100F300003F5817301EB031101238B7130BC704702
:100F40000849D4F89C2003F5817301EB03130132A7
:100F500004219971C4F89C20F0E700BF9C5B00203D
:100F6000B44B00209C4B0020A8B183681BB10E4BF2
:100F700007229A7070470C4A1178D36003294FF00A
:100F8000040014BF4FF480718021C2E90111136184
:100F9000137590707047044A02F580510123537015
:100FA00081F8B431704700BF9C4B002010B58121FF
:100FB00004467FF00FFE204601217FF00BFE204605
:100FC00082217FF007FEFFF771FE002010BD00BFF9
:100FD000034610B4D9691A69002040F20114A3F83D
:100FE00044410860D1699C6D21F002014FF0010C71
:100FF000D161A3F89CC32060D369044923F4003372
:1010000081F8280A5DF8044BD3617047C81E0020A0
:10101000202301480B807047640000201223014800
:101020000B80704784000020042301480B80704728
:10103000980000200A4608B5054920B90548FFF781
:101040007DFD034808BD0448FFF778FD004808BD52
:10105000F428002060FC080878FC080810B5044C4F
:1010600004480A462146FFF769FD204610BD00BF2F
:10107000F428002090FC08081C48D0F8E837D0F885
:10108000EC2710B59B184FF01A040C8001D11848BA
:1010900010BD174AD0F8EA0702F1100411464FF0CC
:1010A000000E4FEA137CB3F1204F34BF0CF1300C2B
:1010B0000CF1370C81F802C081F803E002318C4258
:1010C0004FEA0313EDD102F108040021030FB0F140
:1010D000204F34BF303337339374D174023294428B
:1010E0004FEA0010F2D1024810BD00BF00F0FF1F10
:1010F0009C00002010B5044C04480A462146FFF726
:101100001DFD204610BD00BFF4280020A4FC0808E7
:1011100010B5044C04480A462146FFF70FFD20464F
:1011200010BD00BFF4280020B0FC0808A84A53688E
:1011300023F4FD4323F07F032DE9F04143F07603D0
:1011400053605368032123F48073536082B01160AD
:1011500010F062FA04460D4610F05EFA001B61EBD7
:101160000501B0F57A7F71F10001F5D310F054FA62
:1011700004460D4610F050FA001B61EB0501B0F576
:101180007A7F71F10001F5D3914C6368002040F241
:10119000FF5543F480734FF4806263604FF0FF317A
:1011A000A563A060E260FFF7C9F8A563074618B120
:1011B000012002B0BDE8F0814FF4D5724FF489638D
:1011C000A5630721A2600820E360FFF7B7F8A563D5
:1011D00028B9804B012283F890204FF080477C4C47
:1011E00040F2FF55002240F27743A5630121A2603F
:1011F0003720E360FFF7A2F8A5630028D8D147F0B5
:1012000000470646804647F4801701E09642CFD05B
:1012100040F27743A5630121C4F808803720E360DA
:10122000FFF78CF8034640F2694203212920A563A9
:10123000002BBDD1A563A760E260FFF77FF8013600
:101240004FF6FF72A5630028B2D16369002BDDDA87
:101250004FF6FF729642ABD0580000F1C180236870
:101260009A07A5D05B4D95F89060042E40F0C080A1
:10127000FFF732F900289BD1554C2B6840F2FF57FD
:10128000A763A36040F24743E36001210720FFF713
:1012900055F8A763636823F4FD4323F07F0363607D
:1012A000002885D1022E83D863699B0180D4002257
:1012B0000023CDE900234FF008084FF48A63A763A9
:1012C0000121C4F808801020E360FFF737F8A76316
:1012D00000287FF46DAF2B68A763A36040F27743CB
:1012E000E36001213720FFF729F8A76300287FF486
:1012F0005FAF394E6662C4F82880E26A40F27343F9
:1013000042F03302E2620121A763A060E360332070
:10131000FFF714F8A76300287FF44AAF626B40F22E
:101320002A410A4008BF334602D00FE0013B0DD0EE
:10133000666B02A8B60200EB820004D5D4F8806088
:1013400040F8086C0132606B0842EFD0204C636BB0
:101350001F073FF52DAF636B9F073FF529AF636B09
:101360009E063FF525AF636B98023FF521AF009BCA
:101370001BBA59037FF51CAF2A6840F2774340F24D
:10138000FF55A5630121A2603720E360FEF7D6FF79
:10139000A56300287FF40CAF022240F24643A56308
:1013A0000121A2600620E360FEF7C8FFA5630028C4
:1013B0007FF4FEAE63681A0508D4084A63681340D8
:1013C00043F40063636063681B05F7D50020F0E613
:1013D000002C0140C81E002000E1F5050081FFFF40
:1013E000274D022685F89060236899073FF4E0AE08
:1013F000244C40F2FF570023A7630221A36040F270
:10140000C243E3600846FEF799FFA76300287FF414
:10141000CFAE63696B61A369AB61E369EB61236A7A
:101420002B62022E1BD9062E19D0164C2B6840F2C7
:10143000FF57A763A36040F2C943E360022109207C
:10144000FEF77CFFA76300287FF4B2AE63696B6090
:10145000A369AB60E369EB60236A2B6108E7094C81
:1014600040F2FF570023A763A36040F24343E360C9
:1014700006210320FEF762FFA7630028D5D097E678
:10148000C81E0020002C014010B5104CD4F81C3AA6
:1014900043B119689A880B691A4203D1002384F872
:1014A000F03910BDFFF742FE0028F7D194F8E43977
:1014B0000133DBB2072B84F8E439EFD8D4F8243AAF
:1014C000C4F8E039012384F8F03910BDC81E0020AB
:1014D000F8B5A04CD4F8200A002800F01D8194F83B
:1014E000F0596B1E082B1ED8DFE803F06B056F1D4B
:1014F0004DB63E1D2600984E236840F2FF57B76355
:10150000B36040F24D43F36001210D20FEF716FF5A
:10151000B76328B97369C3F34323042B00F0C18078
:1015200094F8F0596B1EDBB2022B40F2AD80042D13
:1015300040F0B1800120F8BD874D226840F2FF568F
:1015400040F24D43AE630121AA600D20EB60FEF72F
:10155000F5FEAE6368B96B69C3F34323042B08D16E
:10156000042384F8F039E5E7FFF724F9002840F078
:10157000D680D4F8E039D4F8242AFA339342CFD273
:10158000FFF782FFABE7E66A002E40F0AF80FFF77F
:1015900011F9002800F0B180D4F8D85984F8E46932
:1015A000042384F8F039002DC4D0D4F8DC39D4F801
:1015B000CC29D4F8D0193046A84794F8F0596B1EBE
:1015C000B1E7022384F8F03989E7FEF785FF0028A8
:1015D0005AD194F86420B4F86630A4F8F839A16EB2
:1015E000A36EC4F8EC09090E04201B0C84F8FA2938
:1015F00084F8F009A26E84F8FB1984F8FC39A16E16
:1016000094F86C0094F86D3084F8FE19120A1B09E6
:1016100084F8FD2984F8FF0994F86D2084F8043AD1
:10162000216FB4F87600B4F87630C4F8001A02F0EE
:101630000F02C3F30B1384F8052A43EA1023B4F80E
:10164000762003F00F0303F5FA6302F00F02A4F80B
:10165000063A84F8082A42E7236BE3B9D4F8D8693C
:10166000D4F8243AC4F8E039072584F8F05996B143
:10167000D4F8DC39D4F8CC29D4F8D0190120B047FB
:1016800094F8F0596B1E4EE7D4F8243AD4F8E029C8
:101690009B1AC82B25D8A5F10800B0FA80F04009A4
:1016A000F8BDFEF719FF00287FF43AAF94F89030A8
:1016B000002BA3F10203B3FA83F308BF01255B09F2
:1016C00084F8E65984F8E739FEF706FF00287FF42E
:1016D00057AFD4F88020C4F8F429032384F8F039F4
:1016E000FDE6FFF7D1FE94F8F05920E7D4F8E03991
:1016F000D4F8242A64339342CDD2FFF7C5FED4F840
:10170000D859002D3FF4EBAE0022D4F8DC39D4F8E0
:10171000D0191046A847E2E684F8F009F8BDD4F8DD
:10172000EC390022012B84F8E4290BD9D4F8E829FC
:101730000825013B0132C4F8EC39C4F8E82984F8E3
:10174000F059A8E77FF40CAFFFF73AFB94F8F05993
:101750006B1EE8E6C81E0020002C01402DE9F8436E
:10176000274E8146D6F8247A0A4604E0D6F8243A71
:10177000DB1B322B40D896F82B3B002BF6D1CAB39B
:101780004A4402F1FF3809F1FF39D6F8A030D6F803
:10179000A4200133C3F30A039A421BD1D6F8243A9A
:1017A000DB1B322B28D80FF037FF04460D460FF015
:1017B00033FF001B61EB0501B0F57A7F71F1000189
:1017C000F5D3D6F8A030D6F8A4200133C3F30A032A
:1017D0009342E3D0D6F8A020D6F8A03019F8011F24
:1017E00032440133C3F30A03C14582F82C1BC6F807
:1017F000A030CAD1002000E00220BDE8F88300BF7D
:10180000C81E0020F8B50F4ED6F89C3003B9F8BDBD
:10181000D6F89C30052BFAD10B4B1B78002BF6D059
:10182000002AD6F8247A0D461446F0DD21462846D3
:10183000FFF794FFD6F8243A0028E8D0DB1B322BC0
:10184000F4D9F8BDC81E0020000000202DE9F047A3
:10185000534E1F4606EB80039C68002C00F09B80D3
:1018600004F13E03A36104F59F73E3614FF48073B9
:10187000C4E904332836236866600546E16094F8BD
:101880003D00A36391460BF009FE804694F84402A4
:1018900094F83CA0261D002851D194F8450250BB75
:1018A000D4F840326BBB3A0731D419F0020F49D15A
:1018B00019F0010F5AD1D4F8483294F9471294F82C
:1018C00047221B010029DBB20DDB3649881880F85E
:1018D00000335009012302F01F02934041F82030E9
:1018E0003046BDE8F087304902F00F02114430461F
:1018F0000B76BDE8F08778F0E3FBD4F84032002B9C
:10190000D1D02A4A116B0B4313633A07CDD5013569
:10191000EDB2B8F1000F05D040F2067388F8085018
:10192000A8F80630FB0694F846222FD417F0200FB3
:101930000CBF3221122140460BF074FDBBE778F05A
:10194000BFFBAAE76B1CDBB2B8F1000F05D088F82B
:10195000083040F20653A8F8063094F84622404674
:1019600002210BF05FFD19F0010FA4D050460BF0DF
:1019700095FD0135EDB218B140F20663C3800572E2
:1019800094F8462202210BF04DFD94E702214046D7
:101990000BF048FD8FE726463046BDE8F08700BFD4
:1019A0001052080800E100E0FCEC00E000380240C2
:1019B0002DE9F047038A8489A4B21C4082B047D045
:1019C000814688464FF0004501F14C0701F134068D
:1019D000B4FA84F325FA03F2D24391B2A9F81010B5
:1019E00014401B3BB8F1000F5FD0042B2ED8DFE86A
:1019F00003F052483D320300D8F80C30D9F82CA03F
:101A000033B19B6823B11FFA8AF108F104009847AB
:101A1000D8F8243033B19B6823B11FFA8AF108F15A
:101A20001C009847D8F83C3033B19B6823B11FFAAB
:101A30008AF108F134009847D8F8543033B19B68E4
:101A400023B11FFA8AF108F14C009847002CBFD14E
:101A500002B0BDE8F087D8F80C30D9F834105B68D4
:101A600008F104009847002CB2D1F1E7D8F82430EF
:101A7000D9F838105B6808F11C009847002CA7D1F2
:101A8000E6E7D8F83C30D9F83C105B683046984718
:101A9000002C9DD1DCE7D8F85430D9F840105B68B1
:101AA00038469847002C93D1D2E7042B07D8DFE8BB
:101AB00003F01903140F0A00D9F83C300193019B7D
:101AC000002C85D1C4E7D9F82C300193019BF7E7AE
:101AD000D9F834300193019BF2E7D9F838300193FB
:101AE000019BEDE7D9F840300193019BE8E700BF87
:101AF00010B5044629B990F81121032A0DD0002011
:101B000010BDD0F8E4359B69002BF8D090F8122175
:101B1000032AF4D19847002010BDD0F890230B463B
:101B2000D0F87C138A4219D9521AC0F8902394F83D
:101B300003C0D0F880038A4228BF0A46BCF1010FD7
:101B400092B234D0C4E9E22304F55D71C4F8800395
:101B5000A4F8743320467FF0D7F8D0E7D0F8E43506
:101B60001B691BB190F81221032A1ED000234FF4E9
:101B700080720421C4E94A33C4E94C3384F811115A
:101B8000A4F81C2104F58E7120467FF0BDF8636D2A
:101B90000D4A1A61E278012AB1D104F2CC545C6199
:101BA0004FF0802219681A60A9E79847DEE70844D9
:101BB000C4E9E22304F55D71C4F88003A4F874332A
:101BC000C4F88403C6E700BF1800086038B50446AF
:101BD00049B990F81131022B11D094F81631012B2C
:101BE00039D0002038BDD0F8E4355B69002BF8D03F
:101BF00090F81221032AF4D19847002038BDD0F87C
:101C00003831D0F8242193422FD990F803C09B1A81
:101C1000BCF1010F0D46C0F83831D0F828116ED054
:101C20009BB2C0F830314FF48073C0E94A11C0F85C
:101C3000345100F58E71A0F81C317FF065F8C4E9CD
:101C4000E255C4F8805304F55D71A4F8745320463E
:101C50007FF05AF8C1E73F4B2269D3F83412516044
:101C6000002384F81631002038BDD0F83C31B3FB96
:101C7000F2F502FB15350DBB9A421FD8D0F8402172
:101C800093421BD24FF48073A0F81C3100F58E7183
:101C9000C0E94A55C0E94C557FF036F8E378C4F8FE
:101CA0004051012BC4E9E255C4F88053A4F87453A1
:101CB00008BFC4F8845304F55D71C8E7D4F8E4356F
:101CC000DB681BB194F81221032A15D0E2780023B7
:101CD0000521012A84F81111C4E9E233C4F88033E4
:101CE000A4F8743304F55D7124D020467FF00CF81D
:101CF000636D194A1A6170E720469847E6E79BB280
:101D00001144C0F830314FF48073C0E94A11C0F873
:101D1000345100F58E71A0F81C317EF0F5FFC4E956
:101D2000E255C4F8805304F55D71A4F87453C4F807
:101D300084538CE7C4F8843320467EF0E5FF636D5E
:101D40000548186104F2CC525A614FF080211A689C
:101D5000196042E7C02F00201800086070B52B4CB6
:101D60000025D4F89830D4F894209A4228D0D4F89A
:101D70009820D4F898300133C3F30A03C4F898309C
:101D8000D4F89810D4F8943094F8BC31224492F8E6
:101D9000CC510BB9284670BD0126D4F89830D4F840
:101DA000942003F2FF739B1AC3F30A03802B0DD810
:101DB000002EEFD1D4F89830D4F894209A42D6D19E
:101DC00094F8BC31002BCCD00026E6E7104B93F8FA
:101DD0003B12002201290F4984F8BC214FF040003A
:101DE000C3F8EC254FF00102A3F8D425C3F8E805A9
:101DF00003F62C02A1F5677008BFC3F8E425C3F809
:101E0000E0257EF0E3FF002ED4D0C3E7C81E0020FB
:101E1000C02F002094350020F8B5264C94F82B2BC9
:101E2000012A034603D0022A09D00020F8BD224E21
:101E3000D6F86C588DB984F82B5B0020F8BD0025CE
:101E400040F20112C0E95455C0E95655A0F84421AA
:101E500000F5A2717EF0BAFFEDE7402D20D94027B2
:101E6000D4F8A410154AC3F858710A44C3E954229F
:101E700040F20112A3F844210022C3F85C2103F5CB
:101E8000A27118467EF0A2FFD4F8A4303B44ED1BAB
:101E9000C3F30A03C4F8A430C6F86C580020F8BD98
:101EA000AAB2402A01D02F46DAE7022284F82B2B6F
:101EB000D5E700BFC81E0020C02F0020F429002055
:101EC00001EB810138B500EBC1010E4DB1F88C1367
:101ED00004462846FEF72EFF88B9E378C4F8A853D5
:101EE00001214022012BC4E9EC20A4F89C1308BF77
:101EF000C4F8AC5304F5677120467EF067FF0020FC
:101F000038BD00BFEC370020F8B52A4CD4F8703843
:101F10000E2B04D80133C4F870380020F8BD264DCC
:101F200095F82B3B0022C4F87028002BF5D1D5F88A
:101F3000A420D5F8A0309A42EFD0D5F8A420D5F847
:101F4000A0309A422DD9D5F8A460C6F50066402E7F
:101F50002DD8B3B2402B13BF3746402702230123AD
:101F6000D5F8A42085F82B3B144BC0F858711344C6
:101F7000C0E9543340F20113A0F844310023C0F803
:101F80005C3100F5A2717EF021FFD5F8A4303B440E
:101F9000F61BC3F30A03C5F8A430C4F86C6800202C
:101FA000F8BDD5F8A060D5F8A430F61ACFE7012324
:101FB0004027D5E7C02F0020C81E0020F4290020AC
:101FC00010B5324B93F8802893F894C8D3F87C3836
:101FD000044613B152EA0C0231D00123E06984F8BF
:101FE000463140F20112A4F8442102682849002A2F
:101FF000A8BFC2F380739B0301EA124143F02003A0
:102000000B4363F31F42BCF1020F026000D010BD0E
:10201000E278204BC4F8A8331F200021C4E9EC016A
:10202000012A4FF00101A4F89C1308BFC4F8AC3397
:1020300004F567712046BDE810407EF0C7BE01215F
:102040007EF08EFD0122E06984F8462140F2011302
:10205000A4F84431016800290A460CDBC1F38073FF
:102060000B4C9B0343F0200304EA11410B4363F341
:102070001F42026010BD064B03EA114343F4804344
:1020800043F0200363F31F42026010BDC02F002005
:10209000DFBFFFFF3438002090F848305A1C03445B
:1020A000D2B280F8482083F8341090F849300BB150
:1020B000132A01D97EF03EBF704700BF002280F88E
:1020C00049207EF037BF00BF2DE9F041B0F8CC15B4
:1020D000D0F8CE35B0F8D255B0F8D085C0F8405120
:1020E000012284B080F8112101F01F02012A044668
:1020F00000F2CC56ADF80810C1F3072ECDF80A3027
:10210000ADF80E504FEA134C51D0022A7746C9B2AF
:102110009BB210D0002A55D1BEF1090F4BD8DFE891
:102120001EF08900AD004A00C8004A005C01DF00D3
:102130004A001301330101F0600120295FFA8CF29B
:1021400072D0012F00F0B881032F00F0A181AFBB46
:1021500090F81231022B00F0E381032B2BD11CF0FD
:10216000800F40F0E98102EB820200EBC20393F89A
:102170007623003A18BF0122C24D02234FF480712A
:10218000C4E94E3384F81131C4F83031A4F81C117D
:1021900005F50A630021C4F83411C4E94A3304F593
:1021A0008E712046C5F8A0287EF0AEFD06E090F8BE
:1021B0001231032B0ED020467EF09AFC002004B092
:1021C000BDE8F08101F080017EF0CAFC002004B07F
:1021D000BDE8F0815FFA8CFCBCF1010FEBD8D0F8C0
:1021E000E43502A99B689847BDF80E30002BE5D175
:1021F000C4E94A33C4E94C3304214FF4807284F8B3
:102200001111A4F81C2104F58E7120467EF07CFD8E
:10221000636D9D4A1A61E278012ACFD15E614FF069
:10222000802219681A60C9E7D0F8E43502A99B68D2
:102230009847C3E790F81231023B012BBBD8914B72
:10224000D0F818210021C3F89C1812B10222C3F85B
:102250009C288E4A02234FF480700021C4E94C313F
:10226000A4F81C01C4E94E33C4E94A2284F81131B0
:1022700004F58E7120467EF047FD9FE790F812210D
:10228000023A012A97D8012B98D1D0F8E4350025DD
:102290009B68C0F8185102A9984704224FF4807334
:1022A000C4E94A55C4E94C5584F81121A4F81C31FD
:1022B000A9E7012B00F03B81022B7FF47FAF5FFA8F
:1022C0008CF3002B7FF47AAF03694FEA1C22023AA9
:1022D0005B68032A00F2BD81DFE802F0B6CED2D0FF
:1022E0001E0A022EADF8065000F08A81032E00F07F
:1022F0004E81012E7FF45FAFD0F8EC3580781B68FB
:102300000DF106019847BDF80630002B3FF456AF9B
:10231000BDF80E20002A3FF451AF934228BF134668
:102320004FF480720221A4F81C210022C4E94A0063
:1023300084F81111C4E94E33C4E94C3204F58E71AE
:1023400020467EF0E1FC39E7012D7FF434AF90F8B0
:102350001231022B00F00881032B7FF42CAF4FF4D5
:10236000807200F588730221A0F81C21002280F8F9
:102370001111C0E94E55C0E94A33C0E94C5200F58D
:102380008E717EF0C1FC19E7DDB23E4F012D87F85A
:1023900095583FF610AF90F81231022B00F0D8801C
:1023A000032B7FF408AF002D00F0358190F8101159
:1023B000012910D0D0F8E4355B68984797F8951854
:1023C000D4F8E43584F810111B6820469847D4F8F7
:1023D000E8359B68984700230AE758EA05027FF42E
:1023E000EAAE90F8121103293FF4E5AE03F07F0541
:1023F00080F814510069114663F30A110368194308
:102400000423016084F811314FF48073C4E94A2237
:10241000C4E94C22A4F81C3104F58E7120467EF0EC
:1024200073FC636D184A1A61E278012A06D0002D08
:1024300000F0FC80022384F81231BFE65E614FF0A9
:10244000802219681A60F2E702210E4861F3061330
:102450000022C0F834320423C4E94A22C4E94C22E1
:1024600084F8113101224FF4807304F58E7184F8E1
:102470001621A4F81C31C8E60321E6E70521E4E7AC
:102480000421E2E7C02F0020180008605C3800201B
:1024900090F81211022943D003297FF48CAE23B99E
:1024A000510602D011467EF05BFBD4F8E4359B6800
:1024B00002A9204698478EE790F8121102292FD0E2
:1024C00003297FF478AE002B7FF478AE12F07F0101
:1024D00081D01CF0800F40F0AD8002EB820100EB58
:1024E000C10181F8763381F87533282381F874238C
:1024F00003FB020300EB820193F87723496D0B681D
:10250000023A012A23F400138CBFC3F300720122A4
:1025100062F31C73D4F8E4250B60936802A9C8E742
:1025200053063FF44BAE11467EF01AFB46E6D0F858
:10253000E425C0F81831F0E702F07F0202EB8202D6
:1025400000EBC20393F81E21003A18BF012213E6E4
:10255000002D3FF4A2AE01210322D0F8E43580F82B
:10256000101180F812212FE73B4A80F811314FF407
:1025700080710023A0F81C11C0E94E55C0E94A2221
:10258000C0E94C5300F58E717EF0BEFB16E6DBB25F
:10259000052B3FF610AEDFE803F02B231B130B03D4
:1025A000D0F8EC3580789B690DF106019847AAE6D2
:1025B000D0F8EC3580785B690DF106019847A2E60A
:1025C000D0F8EC3580781B690DF1060198479AE642
:1025D000D0F8EC358078DB680DF10601984792E67B
:1025E000D0F8EC3580789B680DF1060198478AE6B3
:1025F000D0F8EC3580785B680DF10601984782E6EB
:10260000D0F8E43580789B6A0DF106019847467052
:10261000C4F8F00577E60222D0F8E43580F81221FC
:1026200080F810515B682946984736E6012384F804
:102630001231C3E5282202FB010080F81C1104EBD3
:10264000810180F81E3180F81DE190F81F21896911
:1026500055E70121F9E600BF5838002070B50B7826
:1026600013F060020D46044624D0202A04D02046F0
:102670007EF03EFA022070BDCA8848781AB31B0665
:1026800040D5324E3146FEF719FBEB884FF480728D
:102690000221A4F81C21002284F81111C4E94E3350
:1026A000C4E94A66C4E94C3204F58E7120467EF0D6
:1026B0002BFB06E04B780A2B10D00B2B08D0062BF7
:1026C000D5D0002070BD02221144FEF7F7FAF8E7DA
:1026D0008B78BBBB1E4AC2F8A438F2E7022180F80F
:1026E00011114FF48071A0F81C111A490123C0E99F
:1026F0004A11C0E94E33C0E94C3200F58E717EF0CC
:1027000003FBDEE71449154B4860E078C3F8A820C6
:102710000021AC3301284FF00305C4F88C13A4F852
:102720007413C4E9E42284F81151C4F88823C4F86E
:10273000803304F55D7108BFC4F8843320467EF011
:10274000E3FABEE77EF0D4F9BBE700BF741F0020B8
:10275000C02F00206438002000000020C81E002088
:10276000002310B51946044640227EF063FA80210A
:102770002046002340227EF05DFAD4F8E835A078A8
:10278000012284F812215B689847002010BD00BF29
:1027900010B502230446402281217EF04BFA2046E8
:1027A0000223402201217EF045FA2046032308221D
:1027B00082217EF03FFA104B0222A3F85020FEF750
:1027C00063FAE2780D4BC4F8A8334021C4F8B01383
:1027D000012A4FF000004FF00101C4F8B403A4F83F
:1027E0009C13204604F5677108BFC4F8AC337EF033
:1027F000EDFA002010BD00BF00000020EC370020E3
:1028000030B5812183B004467EF0E4F901212046F1
:102810007EF0E0F92A4900250223402281F8285A57
:10282000204681217EF006FA012102234022204623
:102830007EF000FA234BD3F8A82883F89458126846
:10284000284690470095009AE1681F4B42F010021D
:102850000092009A0A610A690092013B02D0009A34
:10286000D006F8D400230193019B43F02003019389
:10287000019A154B012060F38A120192019A0A61B4
:102880000A690192013B02D0019A9206F8D4E278DB
:102890000E4BC4F8A8331F200021C4E9EC01012A23
:1028A0004FF00101A4F89C13204604F5677108BF9E
:1028B000C4F8AC337EF08AFA002003B030BD00BF0C
:1028C000C81E0020C02F0020410D03003438002016
:1028D0002DE9F8433D4F8046894615461C4697F83A
:1028E000F01904290BD0082907D1D7F8E839434556
:1028F00005D0FEF765FA0228F1D0012053E097F8E1
:102900009020C7F8DC490123022A314CC7F8D0894E
:10291000C7F8D859C7F8CC9987F8D4393B6318BFA2
:102920004FEA48280A2640F2FF554FF48B63A5630F
:102930000121C4F808801820E360FDF7FFFC03467E
:102940004FF0000C40F2774201213720A563ABB174
:10295000A563C4F808C0E260FDF7F0FC721EA56331
:1029600060B112F0FF06E0D197F8E5393E63022B23
:102970001BD8013387F8E539012014E001214846CE
:1029800077F00AFB124B134959624FF400729A62B6
:10299000DA6A002042F091020621DA6287F8F01923
:1029A000B86287F8E509BDE8F88387F8E569FEF7BE
:1029B0006BFDD7F8D84934B1D7F8DC39D7F8D0193E
:1029C00032460120A0470320EDE700BFC81E0020CB
:1029D000002C014000E1F5052DE9F04F454E9946E8
:1029E00096F8F03983B0042B01908846924609D0BE
:1029F000082B03D0002003B0BDE8F08FFEF7E0F90C
:102A00000228F7D196F890300122022BF2626ED0A4
:102A1000019B4FEA432B384C0021404677F0BCFA2B
:102A20004FF40072354B6362A262E36A40F2FF57D3
:102A300043F09303E362A763A2604FF48A62E2600B
:102A400001211020FDF77AFC0A25A76340F25142CC
:102A5000A7630121C4F808B01120E260FDF76EFC05
:102A600002464FF0000E40F2774301213720A76362
:102A70002AB3A763C4F808E0E360FDF75FFC013DFB
:102A8000A763E0B115F0FF05E0D196F8E539F562EE
:102A9000022BB06203D8013386F8E539AAE786F83D
:102AA000E559FEF7F1FCD6F8D849002CA2D0D6F8AB
:102AB000DC39D6F8D0192A462846A0479AE70523DC
:102AC00086F8F0390023019AB362C6F8D029D6F807
:102AD000242AC6F8CC890120C6F8D8A9C6F8DC9902
:102AE000C6F8E02986F8E53903B0BDE8F08FDDF8D7
:102AF00004B090E7C81E0020002C014000E1F5055D
:102B00001049114BD1F8882042F4700210B4C1F87A
:102B100088201A680D4C002042F001021A6098606B
:102B20001A6822F0847222F480321A605C601A689B
:102B3000074C22F480221A60D8608C605DF8044B48
:102B4000704700BF00ED00E0003802401030002464
:102B500000000008704700BF2DE9F84345697DB9C2
:102B60000768C7F30D0804460E46B8F1000F0AD0F7
:102B7000D6F80080FDF718FF09283BD06FF001055B
:102B80002846BDE8F883514B9F422AD303F5804382
:102B90009F4224D303F580439F427FD34C4B9F42F7
:102BA0007FD903F580339F427ED903F500339F42DE
:102BB0007DD903F500339F427CD903F500339F4252
:102BC00069D903F500339F4277D903F580239F42EB
:102BD00076D9B7F1016F76D305200EF079FD4FF06D
:102BE0000808FDF7E1FE092821D04FF0FF352846FF
:102BF000BDE8F883374E336923F44073336133699A
:102C000043F400733361336943F001033361C7F860
:102C10000080FDF7C9FE3369092823F00103336101
:102C2000ACD12368043323602846BDE8F883DFF87D
:102C3000A490D9F8103023F44073C9F81030D9F8B3
:102C4000103043F40073C9F81030D9F8103023F075
:102C5000F803C9F81030D9F8103043EA080343F0FC
:102C60000203C9F81030D9F8103043F48033C9F8A2
:102C70001030FDF799FED9F8103023F00203C9F89F
:102C80001030D9F81030092823F0F803C9F81030B3
:102C90003FF46EAFA9E74FF03808A2E74FF01008F5
:102CA0009FE74FF018089CE74FF0200899E74FF096
:102CB000280896E74FF0300893E74FF0400890E778
:102CC0004FF048088DE74FF058088AE700400008A9
:102CD000FFFF0008003C02400148FDF799BA00BF21
:102CE000BC0000200148FDF793BA00BF0803002094
:102CF0000148FDF78DBA00BF540500200148FDF7DB
:102D000087BA00BFA00700202DE9F0410268214DDD
:102D10000746002455F834309A4209D001340E2C6D
:102D2000F8D11D4A0021052005F060FB002013E0CA
:102D30001A4B03EB8408D8F8AC687EB1797901EBC3
:102D4000410306EBC30300221820C3E9032200FB62
:102D500001609F601A750430BDE8F08107216C2086
:102D600005F0CCFB0146C8F8AC0868B131466C22CE
:102D700082F044F8D8F8AC6805EBC405C6E9005603
:102D8000F6617663F664D9E7054A052005F02EFB67
:102D9000CCE700BF6C520808C0FC0808C02F002018
:102DA000E8FC0808704700BF38B5D0E9004007EEDE
:102DB000902A0068324A334B2468D3F8E8392468F3
:102DC000013990428DB210D002F5806290420CD051
:102DD00002F57052904208D002F58062904204D011
:102DE00002F58062904218BF5B0807EE103AF8EED9
:102DF000677AB8EE477ADFED246A87EE270A30EE6D
:102E0000260A7FF00BFF1E492388421E8C4292B295
:102E10009BB21AD01D498C4217D0B4F1804F1FD0FD
:102E2000A1F580318C421BD001F580618C4217D016
:102E300001F580618C4213D015498C4219D1238051
:102E40000123E5622285A38238BD23F45C739BB223
:102E500023800023E562228523860123A38238BDD7
:102E600023F45C739BB223800123E5622285A38255
:102E700038BD08498C42E2D023F440739BB2DEE7B0
:102E800000000140000000200AD7233C000401405C
:102E9000001000400014004070B54268937903F0C0
:102EA000020E13F004033AD175469C469E464FF439
:102EB000807001235479032C30D8DFE804F08E624F
:102EC00002361468704E228C22F480721204120CA6
:102ED0002284228C22F4007212042B43120CA58847
:102EE00042EA0322A38B23F073031B041B0CB4429E
:102EF000ADB243F0600300F09B8006F58066B442FB
:102F000000F09680A580A383E1632284A38B23F045
:102F100008031B041B0C43F00803A38370BD0020AF
:102F200005464FF0040C0346C4E71268564E148C55
:102F300024F480542404240C1484148C24F40054A9
:102F400024042B43240C958844EA0334938B23F404
:102F5000E6431B041B0CB242ADB243F4C04375D030
:102F600006F58066B24271D0958093831164148413
:102F7000938B23F400631B041B0C43F400639383C3
:102F800070BD1468404E228C22F010021204120C04
:102F90002284228C22F0200212042B43120CA588DA
:102FA00042EA0312238B23F4E6431B041B0CB442B6
:102FB000ADB243F4C04359D006F58066B44255D053
:102FC000A5802383A1632284238B23F400631B0445
:102FD0001B0C43F40063238370BD1268148C24F02F
:102FE00001042404240C1484148C968824F0020414
:102FF00024042B43240C1C43138B234D23F0730315
:103000001B041B0CAA42B6B243F0600323D005F5A3
:103010008065AA421FD09680138351631484138B5A
:1030200023F008031B041B0C43F00803138370BD3B
:1030300022F4006242EA0E2222F4806292B225F467
:10304000405542EA0C2245EA00155BE725F480452D
:1030500045EA801588E726F4407606434FF6F3707C
:10306000204040EA0E0040EA0C04D4E722F080023F
:1030700042EA0E1222F0400292B225F4406542EA82
:103080000C1245EA80059BE7000001404268537935
:10309000032B0FD8DFE803F00B080502106840305F
:1030A000704710683C3070471068383070471068BF
:1030B0003430704700207047024B0348D3F8AC18F7
:1030C000FEF776BCC02F00200000014010B5064C72
:1030D0000648D4F8AC18FEF76BFCD4F8CC180448BA
:1030E000BDE81040FEF764BCC02F00200000014086
:1030F0000040014010B5064C0648D4F8AC18FEF765
:1031000057FCD4F8D0180448BDE81040FEF750BC76
:10311000C02F0020000001400044014010B5064CC3
:103120000648D4F8AC18FEF743FCD4F8D418044889
:10313000BDE81040FEF73CBCC02F0020000001405D
:1031400000480140034B4FF08040D3F8B018FEF721
:103150002FBC00BFC02F0020024B0348D3F8B41887
:10316000FEF726BCC02F002000040040024B03489D
:10317000D3F8B818FEF71CBCC02F00200008004090
:10318000024B0348D3F8BC18FEF712BCC02F002036
:10319000000C0040024B0348D3F8C818FEF708BCE7
:1031A000C02F00200004014010B5064C0648D4F89A
:1031B000C818FEF7FDFBD4F8D8180448BDE8104045
:1031C000FEF7F6BBC02F00200004014000180040AD
:1031D00010B5064C0648D4F8C818FEF7E9FBD4F839
:1031E000DC180448BDE81040FEF7E2BBC02F002009
:1031F00000040140001C004010B5064C0648D4F8FD
:10320000C818FEF7D5FBD4F8E0180448BDE8104014
:10321000FEF7CEBBC02F002000040140002000407C
:103220000348D0F8F83913B100F6EC10184770478E
:10323000000000200348D0F8183A13B100F60C2023
:1032400018477047000000200348D0F8383A13B1FF
:1032500000F62C2018477047000000200348D0F8E3
:10326000583A13B100F64C20184770470000002070
:103270000348D0F8783A13B100F66C20184770472D
:10328000000000200348D0F8983A13B100F68C20D3
:1032900018477047000000200348D0F8B83A13B12F
:1032A00000F6AC2018477047000000200348D0F813
:1032B000D83A13B100F6CC20184770470000002020
:1032C0000348D0F8F83A13B100F6EC2018477047DD
:1032D000000000200348D0F8183B13B100F60C3072
:1032E00018477047000000200348D0F8383B13B15E
:1032F00000F62C3018477047000000200348D0F833
:10330000583B13B100F64C301847704700000020BE
:103310000348D0F8783B13B100F66C30184770477B
:10332000000000200348D0F8983B13B100F68C3021
:1033300018477047000000200348D0F8B83B13B18D
:1033400000F6AC3018477047000000200348D0F862
:10335000D83B13B100F6CC3018477047000000206E
:1033600030B44568144CA542144D2C6B0CBF44F48A
:10337000001444F480042C6390F914C0C16012015D
:10338000BCF1000F8361D2B20FDB0D4901EB0C03DE
:103390004FEA5C1083F800230CF01F0C012303FAA2
:1033A0000CF330BC41F820307047064B0CF00F0C8A
:1033B00063441A7630BC7047006002400038024017
:1033C00000E100E0FCEC00E02DE9F047AB48002212
:1033D00042F2043C510143588CEA030313F47C5439
:1033E0000AD00132102AF5D1A54D0023C5F8203AA4
:1033F00085F8F039BDE8F0870144A14D0B7FC5F891
:10340000201A002BF1D18F689E4B9F4202D0483387
:103410009F42EAD19C4A536A43F4006353620EF020
:10342000FBF8064688460EF0F7F8801B61EB0801B2
:10343000B0F57A7F71F10001F5D3934A536A23F412
:10344000006353620EF0E8F8064688460EF0E4F892
:10345000801B61EB0801B0F57A7F71F10001F5D3B3
:10346000DFF82492DFF84882D9F8443043F400634F
:10347000C9F84430D9F8303043F48003C9F830300B
:10348000D9F8303043F00C03C9F830304FF00D0A52
:1034900000260C220E2108F6C420A8F8CAAA88F833
:1034A000CC6A09F0BFFF0C220E2108F52D60A8F8A8
:1034B000D6AA88F8D86A09F0B5FF0C220E2108F6C2
:1034C000DC20A8F8E2AA88F8E46A09F0ABFF0C2235
:1034D0000E2108F6E820A8F8EEAA88F8F06A09F0AC
:1034E000A1FF0C220E2108F6F420A8F8FAAA88F809
:1034F000FC6A09F097FF0C220E2108F62430A8F888
:103500002AAB88F82C6B09F08DFF604BC8F8307B34
:10351000302283F831234FF400325A60D9F830302A
:1035200043F48003C9F83030564B9F425BD0584A71
:103530005849C2F8A060C2F8A8104FF47411D160C5
:103540005549C2F8A0100721C2F8B4104B4A534F96
:1035500033461046114605E00133102B01F12001DE
:1035600000F089808E68BE42F6D14D4901EB4311CF
:103570005B01D1F8F0694B498E426DD0424E316B00
:1035800041F48001316303440D21998343499368D9
:103590008B4225D00134102C02F12002F7D10020FB
:1035A000414900230122FFF7DBFED5F81C3A4BB15D
:1035B00019689A880B691A4204D1002385F8F039FA
:1035C000BDE8F087FDF7B2FD0028F6D1D5F8242A32
:1035D000C5F8E029012385F8F039A5F8E40909E7E1
:1035E00000EB4410DCE72A492A488E65234A086626
:1035F000334629484FF074668E6088650720C86698
:103600001046114604E00133102B01F1200132D0A5
:103610008E68BE42F7D1224901EB43115B01D1F81C
:10362000F06920498E4220D0174E316B41F4800161
:10363000316303440D219983124993688B4211D061
:103640000134102C02F12002F7D100201749002389
:103650000122FFF785FEA8E70B4E316B41F4001104
:10366000316390E700EB4410F0E7074E316B41F413
:1036700000113163DDE700235B68FFDEEC09002009
:10368000C81E0020586402400038024000E100E0FB
:1036900000640240802C01406054A308A0640240F2
:1036A0000000002000600240BD080008F507000887
:1036B000C02F002070B52D4C636BD9051ED54FF47B
:1036C000807340F2FF56A363A663E36B284D23F497
:1036D000414323F03A03E3636B6B9A071FD4012243
:1036E00000236A62AB62214A40F2FF539363D36BBB
:1036F00023F4414323F03A03D36370BD636B98070F
:1037000003D51B4B02229A62EDE7636B190721D4A4
:10371000636B9A0622D5164B06229A62E3E7154B95
:10372000D3F8302B136823F001031360E36A0022FF
:1037300023F00803E3622A636B6BDB07CFD540F20B
:103740004C43A6630121A2600C20E360FCF7F6FD68
:10375000A663C4E7064B04229A62C4E7636BDB06E8
:10376000C1D5034B05229A62BDE700BF002C014082
:10377000C81E0020C02F002002683649002310B464
:1037800022F00102212488420260036043608360CA
:10379000C3600361446138D02F4B98422ED02F4B29
:1037A00098423CD02E4B984240D02E4B984232D07B
:1037B0002D4B984241D02D4B984246D02C4B9842ED
:1037C00017D02C4B98423CD02B4B984216D02B4B09
:1037D000984224D02A4B984228D02A4B98421AD09B
:1037E000294B984229D0294B98422ED0284B9842F9
:1037F00008D14FF03D5243F8AC2C03E04FF4746213
:1038000043F8202C5DF8044B7047224B5DF8044BC5
:103810003D229A607047204A43F8642CF2E74FF447
:1038200074125DF8044B43F8382C70474FF0746203
:103830005DF8044B43F8502C7047184A43F87C2C31
:10384000E0E73D2243F8082CDCE7154A43F8942CC6
:10385000D8E700BF1060024028600240406002408C
:10386000586002407060024088600240A0600240E0
:10387000B860024010640240286402404064024084
:10388000586402407064024088640240A0640240B0
:10389000B8640240006002403D000020400F00205C
:1038A00000003D20214A936803F00C03042B10B460
:1038B0003AD0082B1FD01E4B1C4C0360A1681D4A38
:1038C000C1F30311114491F8CC10CB404360A168BF
:1038D000C1F38221114491F8CC1023FA01F18160E7
:1038E000A1685DF8044BC1F342310A4492F8CC2040
:1038F000D340C36070475368516813F4800F536816
:1039000014BF0D4A0A4AC3F3881301F03F01B2FB0A
:10391000F1F202FB03F3054A5268C2F3014201329D
:103920005200B3FBF2F3C7E7034BC5E70038024090
:103930000024F4001052080800127A0070B5446B9D
:103940008668A38923F400531B041B0CA38185798B
:1039500090F805C02B0303F40051C5F380000CF070
:1039600001032A029B001CF0020F4FEA003002F410
:10397000806218BF43F0080302431A43238A9BB2B4
:1039800023F440530B432382A38923F4B05323F041
:103990000C031B041B0C1343A381A38A23F4407361
:1039A0001B041B0C84B0A3826846FFF77BFF234BEC
:1039B0009C4205D003F580639C4201D0029B00E04D
:1039C000039BA2891E49120403EB83034CBF7600BC
:1039D000B60003EB8303B3FBF6F3A1FB0302A0895C
:1039E00052096426000406FB12334FEA02121CD46B
:1039F0001B013233A1FB0313C3F3431313439BB2E5
:103A000023812A07A38A0AD59BB243F00803A38225
:103A1000A3899BB243F40053A38104B070BD23F08B
:103A200008031B041B0CA382F2E7DB003233A1FB6B
:103A30000313C3F342131343E1E700BF0010014037
:103A40001F85EB512DE9F8431D462E4B9DF8206054
:103A50009DF824909842884617463BD02A4B9842BE
:103A600040D02A4B984245D0294B984221D14B4611
:103A7000324629460520FDF7E9FE04460023C4E945
:103A80000B87C4E90733C4E909336671A56084F87C
:103A900006902046FFF752FFF107626B12D4B3077E
:103AA0000BD493899BB243F4005393812046BDE825
:103AB000F88300242046BDE8F883D36843F08003F0
:103AC000D360EEE74FF6DF731380D36843F0200333
:103AD000D360E4E74B46324629460020FDF7B6FEA8
:103AE0000446CBE74B46324629460120FDF7AEFEA1
:103AF0000446C3E74B46324629460320FDF7A6FE9F
:103B00000446BBE70010014000440040004C004068
:103B100000140140816011E741710FE781710DE7E9
:103B20002DE9F043704F07EBC00985B005464FEA19
:103B3000C00899F8F00B09F0B1FC064699F8F10BB2
:103B400009F0ACFC044699F8F20B76F0B9FA6B1C5C
:103B5000DBB21EB140F60C123372F2801CB123723C
:103B600040F60C23E380304604223A2109F05AFC47
:103B7000042220463A2109F055FC07EB08025B4B72
:103B8000D2F8EC4B9C4200F08E80594B9C4200F0E6
:103B90009580584B9C4200F09C80474497F8F33B3B
:103BA000022B32D0032B7CD05349544F012B08BF3A
:103BB0000F46A6886846FFF775FE26F03F06029B73
:103BC0004F4AB3FBF7F13604A2FB0323360C46EA57
:103BD0009346A680228822F001021204120C228051
:103BE0008AB2C1F30B019B0C09B942F001024FF4F8
:103BF000967101FB03F34349A1FB03139B090133B6
:103C00009BB242F4004223841FE0A6886846FFF777
:103C100049FE26F03F06029A394B3604A3FB0213F5
:103C2000360C46EA9346A680218821F0010109045A
:103C3000090C218034499209A1FB021292099B0CC4
:103C40000133042A238438BF0422A28323882F4A05
:103C50009BB243F001032380238823F4816323F084
:103C600002031B041B0C4FF4804143F48063238048
:103C70002181238823F080031B041B0C23802388CD
:103C80009BB202EB451243F0010323800121002384
:103C900082F8385B82F8391B82F83A3B05B0BDE800
:103CA000F0831B4F85E703F5F2331A6A42F40012E2
:103CB0001A621A6A22F400121A626EE703F5F033F0
:103CC0001A6A42F480021A621A6A22F480021A62A4
:103CD00063E703F5EE331A6A42F400021A621A6AC5
:103CE00022F400021A6258E700000020005400404D
:103CF00000580040005C0040009F2400804F1200EC
:103D000083DE1B43D34D6210632D3E05C02F002080
:103D1000C02709002DE9F047924E90F90010804627
:103D2000807806EBC1050138CC0090B0D5F8EC1BCB
:103D300014282DD8DFE810F04C01200115005500A3
:103D40005F009E00A600C301B6017A0084003C0219
:103D50000402D701C000D0002F003700A301950155
:103D60005401888A0C8B81B27F4841EA0441884320
:103D700000F02081D8E90201101A42F2107263EBC0
:103D80000101904271F1000102D3152388F802303D
:103D900010B0BDE8F08798F813000882C8E9022344
:103DA000122088F80200888A0C8B80B240EA044016
:103DB0006E4C844300F0B28000200E900F900120E2
:103DC0000F910E900E99002900F017820F9914316F
:103DD0000F910F9909684905CCD5142388F8023052
:103DE000D6E798F8110000F0FE000882C8E9022327
:103DF000052088F80200888A0C8B80B240EA0440D3
:103E00005B4C844300F0A1800020009001900120D1
:103E1000019100900099002900F0FB810199143173
:103E20000191019909684F05D7D4A3E798F81100CB
:103E300040F001000882C8E902230B2088F8020044
:103E4000888A0C8B80B240EA04404A4C84436DD08F
:103E50000020049005900120059104900499002908
:103E600000F0D181059914310591059909684D0536
:103E7000B3D47FE798F813000882C8E9022307202B
:103E800088F80200888A0C8B80B240EA0440374CE4
:103E900084435ED0002002900390012003910290A1
:103EA0000299002900F0C18103991431039103990B
:103EB00009684E0591D45DE7088820F4806000040D
:103EC000000C088098F8110000F0FE000882C8E994
:103ED0000223102088F80200888A0C8B80B240EA06
:103EE0000440234C844312D000200C900D900120FC
:103EF0000D910C900C99002900F091810D991431CD
:103F00000D910D99096848053FF567AF32E798F8BC
:103F10001330FF2B06D198F810301BB1132388F80B
:103F2000023035E7112388F8023031E7D8F8140061
:103F3000012800F08F81022800F04382098B0E21B6
:103F4000C8E9022388F8021022E7062388F8023025
:103F50001EE7D8F81400002800F06D81082388F8C7
:103F6000023015E700000020010003008400070074
:103F70008200070002000300088820F400600004AB
:103F8000000C0880088880B240F4806008800888AF
:103F900080B240F480700880032088F80200888A8C
:103FA0000C8B81B2A94841EA04418843C8E9022345
:103FB0007FF4EEAE98F81230002B40F0CE8198F8E6
:103FC0001330FF2B00F03F82042388F80230DFE635
:103FD000098889053FF5CEAE002388F80230D7E680
:103FE000344494F8F00B09F059FA064694F8F10BB2
:103FF00009F054FA964AB2F8983B01339BB28246D4
:10400000A2F8983B16B13368B2881A83BAF1000F50
:1040100004D0DAF80030BAF804201A8311213046AF
:1040200009F0DCF91121504609F0D8F94FF00909DF
:1040300065272EB13368B28819690A4240F023819E
:10404000013F00F01D810DF0E7FA04460D460DF02A
:10405000E3FA001B61EB0501052871F10001F6D3BD
:10406000E7E7088880B240F4007008804FF6FF3020
:1040700088820121C8E9022388F8021088E6D8F86E
:104080001400002800F06D81D8F8184014F8016B76
:104090000E8201381225C8E90504C8E9022388F810
:1040A000025075E6888A0C8B81B2684841EA044167
:1040B00088437FF45FAE0A2388F8023068E60888F8
:1040C00080B240F480700880092088F80200888A55
:1040D0000C8B81B25D4841EA04418843C8E9022360
:1040E0007FF456AEE7E7002401250A940B940B9168
:1040F0000A950A98002800F047810B9814300B901D
:104100000B98006846077FF535AED8F814000328F1
:1041100000F06D81022800F24381088820F480605D
:104120000004000C0880088880B240F40070088009
:10413000098A88F81C40C8E9022388F8025027E65B
:1041400000200124089009900991089408980028FB
:1041500000F0148109981430099009980068470705
:104160007FF508AEEFF31185102080F312880888E0
:1041700080B240F400700880D8F818000E8A471CFE
:10418000C8F81870EDB2067085F311880D8AD8F85A
:1041900018106FF001004E1CC8F818600D70C8E9C7
:1041A0000223C8F8140088F81C4088F80240EFE5A4
:1041B000002006900790012007910690069C002C95
:1041C00000F0E880079C14340794079C2468640678
:1041D0007FF5D0AD0C8AD8F818104D1CC8F81850CF
:1041E0000C70D8F8141088F81C000139C8E90223B3
:1041F000C8F8141088F80200CAE50F9918310F9119
:104200000F990968B6E5059918310591059909686E
:10421000B0E501991831019101990968AAE50D9954
:1042200018310D910D990968A4E50399183103918E
:10423000039909689EE5088880B240F40070088000
:104240000121C8E9022388F80210A1E5010003005A
:10425000C02F0020088820F480600004000C088033
:10426000EFF31184102080F31288088B088880B245
:1042700040F40070E4B2088084F311880C215FE6FA
:1042800016B13368B2885A830DF0C6F904460D465C
:104290000DF0C2F9001B61EB0501052871F1000169
:1042A000F6D316B13368B2881A830DF0B5F9044617
:1042B0000D460DF0B1F9001B61EB0501052871F108
:1042C0000001F6D3B9F101097FF4B2AE16B133683B
:1042D000B2885A830DF0A0F904460D460DF09CF902
:1042E000001B61EB0501052871F10001F6D3BAF15D
:1042F000000F04D0DAF80030BAF804205A830DF029
:104300008BF904460D460DF087F9001B61EB0501A2
:10431000052871F10001F6D316B13368B2881A830B
:104320000DF07AF904460D460DF076F9001B61EBAD
:104330000501052871F10001F6D3BAF1000F04D090
:10434000DAF80030BAF804201A8398F90000441C07
:104350003FF442AEFFF7E4FB3EE60F2388F802305D
:1043600016E5088880B240F4007008800121C8E991
:10437000022388F81C1088F8021009E50999183101
:10438000099109990968F5E40B9918310B910B997A
:104390000968EFE407991831079107990968E9E47A
:1043A000D8F81800098A441CC8F818400170D8F8D9
:1043B0001410C8F808200139C8F81410C8F80C30D7
:1043C000E6E4088880B240F400600880EFF31184CE
:1043D000102080F31288088B088820F48060000485
:1043E000000CE4B2088084F311880D21A8E5088848
:1043F00020F480600004000C0880EFF3118410208A
:1044000080F31288D8F818000D8A461CC8F8186086
:104410000570088880B240F40070E4B2088084F32C
:104420001188D8F81800098A441CC8F8184001708F
:10443000D8F814100C200239C8E90223C8F8141067
:1044400088F80200A4E498F81030002B3FF4BCADCB
:1044500031E600BF38B5184D9DF814E005EB401467
:104460004FEA401C94F8390B00B938BD84F84B2B47
:10447000C4F84C3B01220023490005F6383584F886
:104480004A2B84F8543B049A84F848EB022384F8BE
:10449000491BC4F8502B84F83A3B65440DF0BCF836
:1044A00002460B462846FFF735FC94F83A3B002BB2
:1044B000F4D194F8540B38BDC02F002038B5184DF6
:1044C0009DF814E005EB40144FEA401C94F8390BBA
:1044D00000B938BD490084F84B2BC4F84C3B84F834
:1044E000491B0023049984F848EB022205F638356D
:1044F00084F84A3BC4F8501B84F8543B84F83A2BA8
:1045000065440DF089F802460B462846FFF702FC89
:1045100094F83A3B002BF4D194F8540B38BD00BF0B
:10452000C02F0020F0B589B00023904A0293039376
:10453000136843F48033136003E0029BB3F5A04F8C
:1045400009D0136803F400330393029B01330293F1
:10455000039B002BF1D0854B1B6813F4003318BF6D
:1045600001230393039B012B01D000BFFDE77F4B89
:104570007F491A6C7F4842F080521A640A6842F4FC
:1045800040420A609A689A609A6842F400429A60CF
:104590009A6842F4A0529A6058601A6842F0807299
:1045A0001A601A689001FCD5734A40F205711160D7
:1045B000996821F003019960996841F00201A2F520
:1045C00080629960936803F00C03082BFAD193681A
:1045D00003F00C03042B00F0C680082B00F0AB8026
:1045E000664A624B66499868664D674E674FC0F3EE
:1045F00003100144002491F8DC10CA406449E960CA
:104600006449586FA960596BC6F8E82921F0800108
:104610005963596F604A614841F080715967196B5D
:104620000A431A635A6B5A639A6B9A631A6C5C4911
:104630000A431A64596C5B4A0A435A6448F2FF7190
:1046400023462246CDE900447CF098FC5648234698
:1046500022464FF6FF71CDE900447CF08FFC5348B1
:10466000234622464FF6FF71CDE900447CF086FCDC
:104670004F48234622464FF6FF71CDE900447CF0B7
:104680007DFC4C48234622464FF6FF71CDE900449D
:104690007CF074FC4848234622464FF6FF71CDE972
:1046A00000447CF06BFC4548234622464FF6FF71E0
:1046B000CDE900447CF062FC4148234622464FF697
:1046C000FF71CDE900447CF059FC234622464FF6A9
:1046D000FF713C48CDE900447CF050FC04A8FFF792
:1046E000E1F8D5F8FC200499D6F8E839364842F0CC
:1046F0008072C5F8FC20354AC2F8B00F54601068CB
:1047000040F0010010604FF47A72B3FBF2F3013B0A
:10471000B3F1807F2E4AB1FBF2F2C7F89C2B08D28E
:104720004FF0E022F0215361072385F823109461B4
:10473000136109B0F0BD5168536852684902C2F371
:1047400088124CBF23490D4903F03F03B1FBF3F33B
:1047500003FB02F2054B5B68C3F3014301335B00CB
:10476000B2FBF3F23DE71B4A3BE700BF00380240D3
:104770000070004008544007003C02400024F40050
:104780001052080800ED00E000000020C02F0020BB
:104790000003FA0500000008FF91670000000240D6
:1047A000FFC9FE1033570700000402400008024012
:1047B000000C0240001002400014024000180240A9
:1047C000001C02400020024055CEACC5001000E0A5
:1047D00040420F0000127A0082B0064B0022019284
:1047E0000193019B03EB80030193019B196002B0CD
:1047F000704700BF5028004010B51C2008F04EFE46
:104800001121044608F0EAFD4CB12368A2885A83BE
:10481000C8200CF02FFF2368A2881A8310BDBDE8C2
:104820001040C8200CF026BF704700BF704700BF83
:10483000704700BF10B5104C94F8423223B90F4BAB
:104840004FF480225A6110BD4FF0E022D2F8103DA3
:1048500023F00603C2F8103DFEF752F9D4F84832AF
:104860009B68DB07EBD5D4F84423136823F00301DE
:1048700061F307031360E2E7C02F0020003C014012
:104880002DE9F04FA34CD4F844325A69D5078BB0C8
:1048900002D50BB0BDE8F08F5A699B6912EA03019B
:1048A000F7D0C1F307430803019300F1E180019BB6
:1048B0005D073FD48807CEB203D5D4F84432022234
:1048C0005A610029C0F248820A05C1F3072500F1A8
:1048D0009981370708D5904B9048D3F8103C9847FA
:1048E000D4F8443208225A61F60600F10D82E80637
:1048F00000F1BE81A80600F11781019BDA0609D5F7
:10490000854B8648D3F8203C9847D4F844324FF47E
:1049100080125A61019B9B06BBD57F4B7F48D3F821
:10492000243C9847D4F844324FF400125A610BB03B
:10493000BDE8F08FD4F848329E69DB691E40B6B2FC
:10494000002EB7D0754D4FF0000B05F118080F463B
:10495000F00740F18280D4F84812D8F800200869A6
:104960004B6B23FA0BF3DB01DBB20343906803408C
:1049700013F00109D8B200F00D824B6B012000FA50
:104980000BF023EA00034B6301239360624B6348FF
:10499000D3F8083C5FFA8BF1984794F83B32012B2F
:1049A00000F07C8219F0800F57D0D5E94CC1D5F8C2
:1049B0002431D8F800E0ACEB01029342DEF8180095
:1049C00028BF134680B20333B0EB930F45D9D4F818
:1049D000483294F83B92CDE9026BBA4667469C4652
:1049E000B94237D2D5F82431781A984228BF1846F0
:1049F00000F1030BD5F828314FEA9B0BB9F1000FFA
:104A000010D182B203329210D8F8B8600AD0494669
:104A1000013153F8047B37608A42F9D1D5E94C71F2
:104A2000D5F82831014403448F42C5F82831C5F830
:104A30003411DEF818300AD195F81C01012202FA6F
:104A400000F0DCF8342022EA0002CCF834209BB2DB
:104A50009B45C5D3DDE9026B574676080BF1010B88
:104A600005F1280508F104087FF472AF394621E703
:104A7000D4F848329D69DB691D402D0C3FF417AF17
:104A800004F50E78DFF890B0029104F52376002744
:104A90004FF00109C24608E06D0807F1010706F171
:104AA000040608F1280800F08F81EA07F4D5306881
:104AB000D4F84812836849690B40D9B2DB0740F14A
:104AC0006E8194F83B32C0F80890012B07D1016940
:104AD000D8F87C33C1F312015B1AC8F88C33DBF8C9
:104AE000043CF9B25046984794F83B32012BD3D19D
:104AF000002FD1D194F84933052BCDD1D4F88C3285
:104B0000074919610749596119684FF080211960F7
:104B1000C2E700BFC02F002000000020F8310020B5
:104B200018000860C4370020D4F84852D4F8502246
:104B3000AB68C3F34103022B136814BF00210321A8
:104B400061F30A0313606B6843F4807306A86B601B
:104B5000FEF7A8FED4F84422079ED36823F47053CE
:104B6000D360A86810F0060FC0F3410100F03A814D
:104B70009E499F483144814240F2AC819D48A6F550
:104B80007401A1F51051814240F2A8819A499B48D5
:104B900031448142C0F0A6819948A6F18C71A1F5FB
:104BA0004341814240F2A281964997483144814273
:104BB000C0F0A0819549964831448142C0F09E8161
:104BC0009448A6F1B771A1F558518142C0F09E8179
:104BD0009149924831448142C0F094819048914972
:104BE0003044884234BF062005204025012160F36F
:104BF0008D23D3604FF4005384F83A12A4F83C524A
:104C000053617AE600238DF8133094F84A338DF817
:104C10001330854B8548D3F8183C9847D4F8483270
:104C2000D4F84422986894F842324FF400615161FC
:104C3000002B3FF44EAEC3077FF54BAE94F84D33D7
:104C4000012B7FF446AE9DF81330032B7FF441AE69
:104C5000D4F8443376491A6842F001021A601A689F
:104C600042F003021A600B6943F006030B6130E661
:104C7000D4E991167368002723F001037360059748
:104C8000059B43F020030593059B67F38A13059367
:104C9000059B0B61674BBC460A690592013B02D03C
:104CA000059A9206F8D494F8392252B1624B03EB7C
:104CB000820EFF2253F8040F8260D86B7345826026
:104CC000F8D10B2363F3070763F3070C4FF0FF33AF
:104CD000B3614FF00113F3617761C6F810C0336818
:104CE000564823F4FE63336094F83B22D4F88C32A8
:104CF000012A18616FD04FF480534B614A4B4B48E7
:104D0000D3F8143C9847F5E5D4F844329A6922F078
:104D100010029A611A6AC2F34340022802F00F019E
:104D200000F09080062812D101EB810104EBC10153
:104D3000D4F80863D1F8C405C2F30A1210443268EB
:104D4000C4F804283268C4F80828C1F8C4059A6970
:104D500042F010029A61CAE594F842323BB1D4F8AD
:104D60004423136823F0030060F307031360D4F8AF
:104D700048222D4B2D48D3F81C5C5368029123F038
:104D800001035360A847D4F8443202994FF000421F
:104D90005A6199E5010707D5082393605DE68A0704
:104DA00007D50223836077E6C3060FD510239360EF
:104DB00053E60B077FF570AEDBF80C3C5046984786
:104DC00033680821996067E6029970E5410679D554
:104DD0004023936041E61A4A5A611A684FF08022D4
:104DE0001A6088E74FF40075092000E7401E1BFF9A
:104DF0003F420F00DFC810002013FBFE20D6130037
:104E0000FF69180000D3CEFE40771B00C05BB3FEE5
:104E1000C091210040AC2700C01D6AFE40E1330074
:104E2000803C36FEE09C410000000020F83100206C
:104E300000ED00E0410D03000C3200201800086076
:104E4000C437002047F6F070104280D0C2F30A1237
:104E500001EB810004EBC00002F1030C5FEAAC0C33
:104E6000D0F8B865D4F808E34FEA810818BF0020ED
:104E700006D00130DEF8007046F8047B8445F8D196
:104E8000414404EBC101D1F8B8051044C1F8B8059C
:104E9000D1F8C4051044C1F8C40558E7BBF1000FB0
:104EA0007FF480AD94F84933042B7FF47BADD4F8C4
:104EB0008C32184A1A61184A5A611A684FF08022D7
:104EC0001A606FE5830758BF81467FF56BAD0223FB
:104ED0009360C2E5012140250E2088E6012140258E
:104EE0000D2084E6012140250C2080E6012140258B
:104EF0000B207CE6012140250A2078E6012140258F
:104F0000092074E601214025072070E60121402593
:104F100008206CE618000860C43700200278436857
:104F2000022A11D00C490269D1F8180210B41840B5
:104F3000D1F81042D1F80C12931E400A04FB030072
:104F400008445DF8044B7047034AD2E9802102EB24
:104F5000410202EB532070479C5B00202DE9F04F8B
:104F600012F0020A884E83B09B4601D000286FD011
:104F7000D6F80852002D58D14FF0FF3C834C844F97
:104F8000CDF804C0E046E646002300922268A57BE7
:104F9000904200F09E80002D40D003F58179012DD4
:104FA00007EB09190AD199F80750EA0706D415F05A
:104FB0007E0F03D1ED0900F090809E460133082B4F
:104FC00004F11004E2D1BCF1000F009A04DABEF142
:104FD000000FC0F29280F4466D4CD6F8983004EB86
:104FE0000C1741F2180E013347F80E0041F21C0E67
:104FF0000CF5817547F80E302F01C6F89830E35153
:1050000004EB051300275F6004EB05139B79042B69
:105010007AD8DFE803F02940194043009C46013369
:10502000082B04F11004B1D1CDE7D6E9833404FB99
:1050300005339842A0D396F8B43113B9012386F80A
:10504000B431534B01225A70002003B0BDE8F08FF9
:1050500096F8B431A6F58054002B59D001230220D4
:10506000637003B0BDE8F08F12F0010776D104EB56
:105070000513D01093F807E0BBF1030F60F3C71ED0
:1050800083F807E068D94FF6FF735B4528BF5B469E
:1050900004EB05108380BAF1000F49D1500705D504
:1050A00004EB0510C37943F00103C371D30608D59F
:1050B00004EB0515EB79C3F34502013262F34603B5
:1050C000EB71344B012003EB4C230B6003B0BDE8C4
:1050D000F08F009A05BB9C467EE7A568019A954231
:1050E00038BF984603F1010338BF2A46082B0192C6
:1050F00004F110047FF44AAF65E7B8F1000FA8BFD0
:10510000C446BFF669AF9FE796F8B431002BA5D12E
:10511000012386F8B431A1E7D6F898701C4C03F54A
:1051200081759C462B010137E750C6F898706BE7F4
:10513000D6F89830D6F89C0001330130C6F8983084
:10514000C6F89C0004EB0C1041F21C06835104EBE2
:10515000051304209871A1E73B4699E70E4BD3F85D
:10516000A03B002B3FF470AF0A495E680B4A01EB8D
:105170004C210023B04700283FF466AF04EB05152F
:105180000223AB7160E700BF9C5B0020B45B002092
:105190009C4B0020B44B0020C02F0020710E000853
:1051A00070B5104E3378022B0F4B0BBF020AC0F3C1
:1051B000D412C4B200F07F04D3F8000282B01044CD
:1051C0000D460023032201A9FFF7C8FE012807D1DD
:1051D0003378019A022B0CBF22F8145042F8245065
:1051E00002B070BD9C4B00209C5B00202DE9F04F6D
:1051F000DFF820910D4699F800102B68032985B03F
:10520000164640D0022966D14FEA132A5FFA83F886
:105210004FF4807B421E012A24D801249E421CD9CF
:1052200001288CBF00220122394F0192D7F8782142
:105230001AB1D7F89411994250D0D7F80002002340
:105240005044092203A9FFF789FE012824D002282F
:1052500015D020B12B689E42E8D82E60032005B0FF
:10526000BDE8F08FB8F1000F14D0294B93F8B421AA
:1052700012B9012283F8B421012389F801300220F8
:1052800005B0BDE8F08F4FF0800BC3F3D41A03F0E4
:105290007F08BFE75C46C1E799F80010022916D0E5
:1052A0000329ECD1039B53F8282022F07042019B84
:1052B000D5F800C0B2FA82F252099A4220D0A04436
:1052C0000CEB0403D8452B601DD20229EAD1039BC5
:1052D00033F81820EBE74FF4807BD6E7D7F81012AD
:1052E000013A02EB41224902B2FBF1F21344B3FB53
:1052F000F4F204FB12320AB123449B1A2B60AAE792
:105300006645ACD8A9E70AF1010A4FF00008A2E708
:105310009C5B00209C4B00202DE9F04FDFF8509162
:105320000B6899F800C0174609F58052BCF1020FCE
:10533000D2F8005283B08B46824640F08180DEB2C4
:10534000A6EB030805EB1325B8444FF48072904494
:10535000BB4208F1FF38B8FBF2F843D2A844BCF1D5
:10536000030F06EB0704A4EB030414BF4FF4807291
:1053700080229442A8EB050328BF1446B6BB944292
:1053800034BF0B220A2201A92846FFF7E7FD0128B6
:1053900029D199F800C0DBF80000BCF1020F00F140
:1053A000010325D0A64210D2019906F18042013AAC
:1053B00001EB8202043901EB840142F8043F8A4286
:1053C00003F10103F9D1DBF80000A31B0344BAF198
:1053D000010FCBF8003023D09F4205F101054FF0BB
:1053E0000006BCD8012003B0BDE8F08F0B22CAE74D
:1053F000A642EAD2019906F10042013A01EB4202CB
:10540000023901EB440122F8023F8A4203F1010311
:10541000F9D1A31B0344BAF1010FCBF80030DBD163
:10542000BB42D9D1BCF1020F019B18D004F18044DA
:10543000013C4FF0FF3243F82420DBF80030CBE78B
:1054400003F07F06C3F3D412BCF1030FA6EB0308ED
:105450001544B84414BF4FF48072802277E704F1FA
:105460000044013C4FF6FF7223F814200120BAE7F4
:105470009C4B002030B50446C06983B010B90120B0
:1054800003B030BD0D460023032201A9FFF766FDDE
:105490000128F5D1B4F92020002A19DB019B012D48
:1054A0004FEA421103EB421203D0022D1BD1E5203B
:1054B0005854A368D3612378032B04D100231377B6
:1054C00053779377D377636A53831B0C9382D6E722
:1054D000064A92F8B41109B982F8B401044B0122CA
:1054E0005A700220CCE7E368E4E700BF9C5B002031
:1054F0009C4B00202DE9F043814683B00E4699F87D
:105500003C30042B00F28980DFE803F02F03704F5A
:105510003F00434DDFF810814FF6F77705F58054D3
:1055200018E0BA4260D874F065FB01284FF0000122
:1055300038D1D9F83000FFF733FE012832D1019A73
:10554000D4F81412C9F83020531E8B4228BF0B46E2
:10555000C4F814322A78D9F83030032A01A9184641
:105560009AB2DED14345DED93EE0710001F0FE0182
:105570004846FFF77FFF012843D1D9F83430002B8C
:1055800018BF022089F83C00B9E799F82830042BAD
:1055900004BF002389F82830D9F838300BB14846C9
:1055A0009847012003B0BDE8F0831E48D9F82C20AD
:1055B000D0F89431C0F894219B1AD0F8102202FB45
:1055C00003F3D0F8782102EB4322C0F87821D0F819
:1055D0007C2102EB4322C0F87C21002100F5B87049
:1055E000FFF748FF01280CD10420CBE7D9F834207D
:1055F00009F130010020FFF78FFE012801D10320BF
:10560000C0E70228CED199F82830042B04BF00232C
:1056100089F8283003B0BDE8F0830220F3E700BF2B
:105620009C4B00209C5B0020F7FFFF0F38B5044621
:1056300094F83430052B58D8DFE803F0372B2319C2
:10564000100394F82830082B04BF002384F8283076
:10565000274B012283F8B521022038BD94F8283069
:10566000082B04BF002384F82830012038BD002116
:105670002046FFF7FFFE012837D1042084F83400CC
:10568000D6E7D4E90B01FFF78BFD01282DD10320CC
:10569000F4E7206B4FF0FF31FFF782FD012824D1A2
:1056A000E36A002BF3D00220E8E7114DD5F8082279
:1056B00004F1300101200232FFF798FD012805D0E6
:1056C0000238C0B2012810D80520D7E7E368D5F822
:1056D0001012226BC5F8142203EB4123C4E90332F4
:1056E000E36A002BCAD16262C8E7002038BD00BF60
:1056F0009C5B002070B5044694F83830032B4BD8DF
:10570000DFE803F01F170B0200212046FFF7B2FE6F
:10571000431EDBB2012B40D970BD626B04F1300136
:105720000120FFF7F9FD0128F2D1032384F8383076
:10573000E2E71F480021FFF79DFE0128E8D1022380
:10574000F4E71C4AE56802F580531278D3F810128A
:10575000D3F89401032A14BF4FF48072802202FB15
:1057600001F105EB4125C4E90350D3F87851A5EBCD
:105770004125C3F87851D3F87C51861AA5EB412115
:105780000244C3F89421C3F87C11E36AC4E90C0213
:105790005BB960620123C9E7022094F82830062B28
:1057A00004BF002384F8283070BD2663F2E700BFF1
:1057B0000C5D00209C4B00202DE9F0434368C3F3AF
:1057C00008020A44B2F5007F83B005460C4605D2B4
:1057D00023446B60012003B0BDE8F08390F91A20E8
:1057E000501C0AD0464902F5817201EB0212D179B0
:1057F00021F00101D171FF22AA7695F91B20511CDD
:1058000016D03F4E02F5817206EB021106EB021232
:10581000C979D079C1F34501012986BF01F1FF3172
:1058200001F03F010021FF2661F34600D071EE76C2
:105830002A78022ACCD0324E06F58058D8F81022A9
:10584000B4EB422F4FEA42292BDCD8F818721F40E4
:105850007A42A24225DCE2194A45286913D32A7EFE
:10586000120729D5D8F89421411C8A421BD300D1B4
:1058700000214B44DB1BA4EB0909686109EB070419
:1058800029616B6008460028A4D03278032A31D001
:1058900080B24FF6F77290429CD81A4614446C605E
:1058A00098E7002097E798F8B42102BB012388F815
:1058B000B43173706B68DCE701A974F09BF90128BF
:1058C000EFD16B68297828696861A4EB09049944D1
:1058D000A9EB070301986B6002293C4428611A4632
:1058E000D1D1D8F82012B3EB412FD7D372E70122E0
:1058F0007270BEE7034A90423FF66CAFCDE700BF3F
:105900009C4B0020F7FFFF0F2DE9F047044682B0C3
:1059100094F83830032B00F2AB80DFE803F09A17DD
:105920000C02236C002084F8280003B19847022061
:1059300002B0BDE8F087236C002284F828200BB168
:1059400020469847012002B0BDE8F08723786668BA
:10595000484F022B1CBF474BD3F81832204618BFC4
:105960001E40FFF7DBFAC6F34F26361A0546B6B2DD
:10597000A7F5805811E0D7F810325A1E914557D23A
:10598000FFF71AFF40B997F8B43113B9012387F82C
:10599000B431012388F80130013506EB050C0222F1
:1059A00001A9002328461FFA8CF9FFF7D7FA01282E
:1059B0004FF400724FF00001BAD101987FF01EFA47
:1059C000E3694FF400712046002BD4D06368002BAC
:1059D000D1D1019B4FF020324FF02E0C4FF0100E22
:1059E000C3F80120C3F80520A3F8092083F800C0FC
:1059F00042F62E6AD4F824C0A3F820A083F80BE066
:105A0000C3F82220C3F8262083F82A20E26BA3F8EB
:105A10001AC05A872CFA0EFC22FA0EF283F82BE0F9
:105A20009A86A3F814C0D7F810325A1E9145A7D30E
:105A3000C3EBC353590201F500712046FFF7BCFECA
:105A400028B997F8B4317BB10B4B01225A70022070
:105A500007E02046FFF7EAFD012802D0022807D11F
:105A6000032084F8380053E7012387F8B431EBE7CB
:105A700000205DE79C5B00209C4B00202DE9F0415D
:105A8000B1F904300F2B82B00E460446174632D0CF
:105A90002046FFF743FA94F91B80B8F1FF3F3BD053
:105AA0005C4B41F2180203EB08118A58904211D165
:105AB000183303EB4825B38801331BB205EB4315BC
:105AC000B38020463D60FFF729FA3060012002B024
:105AD000BDE8F08103F5805292F8B41100295CD042
:105AE00001225A702378022B4CD02269002A60D1FF
:105AF00000233B60EAE74FF40071FFF75DFE0028EA
:105B000047D04FF6FF73B3802046FFF707FA94F9AA
:105B10001B80B8F1FF3FC3D12378022B41D022690B
:105B2000002AE5D03B4B1B78032B69D093B24FF68C
:105B3000F7718B4294BF00230123002BD6D138B9D3
:105B4000354B93F8B421002A4DD0324B01225A70C4
:105B50000023112201A9FFF701FA012810D1019DAC
:105B60002E4BEB1A48BF03F2FF13B3F5805F4FEAE9
:105B700063222DD24FFA82F884F81B80002D9AD12F
:105B80002378B0E7244A6368D2F82022B3EB422F8F
:105B9000AED2002002B0BDE8F081012182F8B4113C
:105BA0009EE71D4BD3F820226368B3EB422FC6D388
:105BB0009EE7184B1B78032B19D093B24FF6F77260
:105BC000934294BF00230123002B91D10020E1E7F1
:105BD000114B93F8B42112B9012283F8B4210D4B73
:105BE00001225A70C8E7012283F8B421ADE70C4BBB
:105BF0009A4294BF00230123002B7FF479AFE5E79D
:105C0000074B9A4294BF00230123002B7FF46EAF11
:105C100095E700BF9C4B00209C5B0020B44B00200C
:105C2000F7FFFF0F2DE9F043044689B094F83030B8
:105C3000042B11D8DFE803F0501361035A00237ED0
:105C40009A0640F1FA80E0690023112204A9FFF7C7
:105C500085F9012800F0F18009B0BDE8F083C64D58
:105C600003AE04F11C07324639462846FFF706FF0B
:105C7000012800F0FD800228EED1C04901F58055D1
:105C800095F9D2315A1C0AD003F5817301EB031345
:105C9000DA7922F00102DA71FF2385F8D23195F921
:105CA000D3315F1C16D003F5817301EB031201EBB6
:105CB0000313D279D979C2F34502012A86BF02F1D2
:105CC000FF3202F03F02002262F34601FF22D97147
:105CD00085F8D321042306E0A74874F0B3FA4FF601
:105CE000FF720123228484F830309FE70020E36AAA
:105CF000207009B0BDE8F0431847A14D95F8E03198
:105D0000002BA9D104F11C0703AE05F5DC7832465F
:105D100039464046FFF7B2FE012840F01A81039B46
:105D2000002B00F0F4801A78E52A01D0002AEED189
:105D30009449591A48BF01F2FF11B1F5805F4FEA4B
:105D4000612280F050818D4912018F480244907B7E
:105D500004280CD0D5F898000130C5F898005060A0
:105D600004209073D5F89C200132C5F89C2095F949
:105D7000D221561C0AD002F5817201EB0212FF20DB
:105D800085F8D201D07920F00100D07195F9D321A6
:105D9000501C18D002F5817001EB001201EB0011CC
:105DA000D279C2F34502012A4FF0FF0088BF02F109
:105DB000FF3285F8D301C8798CBF02F03F02002280
:105DC00062F34600C8711846202200217FF016F8C1
:105DD000D4F83120D4F8351041600260B4F839208D
:105DE00094F83B1081720281627EC272019005A814
:105DF00002F0BCFE019B002800F0DE809DF816003A
:105E00009DF817209DF8191042EA4012BDF81400C1
:105E1000A0F2BC7042EA40229DF81A00490141EA12
:105E200050019DF8180041EAC02192B288B2D98190
:105E30001A821A83D882032355E7204674F002FAA7
:105E40002369002B00F08A80237E03F0F70213F011
:105E50000403227640F09A80122A00F0B080E36AB0
:105E60000022204684F8282009B0BDE8F0431847F6
:105E7000DDF80C80B8F1000F00F0C18098F8003018
:105E8000002B00F0BC8098F80B9019F0080F7FF4FD
:105E9000EAAE0B2204F1310140467EF0F3FF002808
:105EA0007FF4E1AE637E89EA0303D90640F1E68020
:105EB000324901F5805595F9D2315A1C0AD003F5C3
:105EC000817301EB0313FF2285F8D221DA7960F3A5
:105ED0000002DA7195F9D321571C3FF4FBAE02F5AD
:105EE000817201EB021301EB0212DB79D179C3F36A
:105EF0004503012B86BF03F1FF3303F03F0300236B
:105F000063F34601FF23D17185F8D331E2E695F8BA
:105F1000B831022B4FF009023FF4DCAE95F8E031C6
:105F2000002B7FF4D7AEC5E97D3385F8F03185F8D5
:105F3000EC31D5F8CC31C5F8E4310F48D5F814323E
:105F400085F8E021C5F8E831FFF7DEFC01283FF4D1
:105F5000DEAE02287FF480AE0423C4E6237E1B0756
:105F60007FF57DAF064B93F89821002A7FF474AE3D
:105F7000072283F8982172E7545D00209C4B002093
:105F80009C5B0020B44B0020B45B0020A568E66A4F
:105F9000002384F8283029462046FFF70DFC00280E
:105FA00066D194F82830002B7FF456AE0223C4E962
:105FB0000B6584F828304FE644F2817238E7626A54
:105FC000E16AA163042084F828002046C4E90B227A
:105FD000C4E9023384F83C306363636209B0BDE80E
:105FE000F04374F02FB995F8B42112B9012285F865
:105FF000B421454901224A706FF00F02A5E64249DB
:1060000001F5805595F9D2315F1C0AD003F58173F3
:1060100001EB0313DA7922F00102DA71FF2385F82C
:10602000D23195F9D3315E1C16D003F5817301EBA3
:10603000031201EB0313D279D979C2F34502012A85
:1060400086BF02F1FF3202F03F02002262F34601F6
:10605000FF22D97185F8D321237ED8067FF53AAE89
:106060002A4874F0EFF84FF6FF72022322843AE6D2
:10607000002E3FF4F1AD204633463AE6B8F814203E
:10608000B8F81A30224D43EA02436362D5F8102271
:10609000D8F81C30A3605202B3FBF2F102FB1131BD
:1060A00009B113445B1AE36084F8199095F9D23171
:1060B00015495E1C0AD003F5817301EB0313DA79ED
:1060C00022F00102DA71FF2385F8D23195F9D3214C
:1060D000501C3FF4B0AE02F5817201EB021301EBEC
:1060E0000212DB79D179C3F34503012B86BF03F19B
:1060F000FF3303F03F03002363F34601FF23D17115
:1061000085F8D33197E600BF9C4B0020545D0020FA
:106110009C5B002070B50378017E023B012B044696
:1061200002D911F0060F68D18D0643D494F91A30C4
:10613000581C0AD0374A03F5817302EB0313FF2082
:10614000DA7922F00102DA71A07694F91B305A1C38
:1061500016D0304803F5817200EB021300EB0210F9
:10616000DB79C279C3F34503012B86BF03F1FF330B
:1061700003F03F03002363F34602FF23C271E3767B
:106180000B070ED5244B93F89821072A06D093F8D5
:10619000B421002A38D01F4A01215170002283F80F
:1061A0009821E26A0023237084F8283022B3BDE8E6
:1061B0007040104700231948E5691A01825895423A
:1061C00006D00133082BB1D01A0182589542F8D17C
:1061D000104803F5817300EB0312D279C2F3450234
:1061E000012A15D9013A02F03F0200EB0313D879D6
:1061F00062F34600D87199E770BD0121FFF73AF9C3
:106200000128F9D1217E8FE7012283F8B421C2E76A
:106210000022EAE79C4B00209C5B0020B45B00203E
:1062200038B5184D05F58054014694F8E00120B9C1
:1062300061B191F8283013B138BD002038BD04F5A4
:10624000DC7044227EF096FD012038BD44220E48C9
:106250007EF0D4FD2B78D4F81C12C4F8DC11032294
:106260004FF6FF70022B18BF1346A4F8D20184F832
:10627000D021054884F8B831102284F8D12173F078
:10628000E1FFE1E79C4B0020545D00204FF0FF3C14
:106290002DE9F041344A354D6446002304E00133D2
:1062A000082B02F1100216D010780428F7D103F55C
:1062B000817005EB0010C179CE07F0D4601C52F854
:1062C0000A1C01D08C45EAD91C460133082B8C46A8
:1062D00002F11002E8D1002C02DA0120BDE8F081C1
:1062E000224DDFF8948004F5817705EB0713998838
:1062F000D8F8A03BF9B92601D8F8A03BDFF87C809C
:106300002E4441F2180208EB4421B058EBB1DC688E
:10631000174A0023A047C0B102280AD108F6E8783E
:1063200005EB0715D8F89C300122013BC8F89C30DA
:10633000AA710020D2E705EB041041F218022601F1
:10634000805813B19B689847D6E70A4BD3F89C2036
:1063500005EB07150320013A0121C3F89C20A87121
:1063600083F8A010E5E700BFC25B00209C4B002033
:10637000E50E00089C5B0020C02F0020B44B0020DD
:106380002DE9F04390F82830013B83B00446082BF8
:106390000BD8DFE803F0393D1F24052A0A2F34000B
:1063A0000121FFF7A7F8012802D003B0BDE8F08370
:1063B0002378216C002284F82820002BF5D0D4E922
:1063C000010383424FF0030238BF0346A36084F801
:1063D0002820E162204603B0BDE8F0439AE60021A0
:1063E00003B0BDE8F043FFF785B803B0BDE8F04364
:1063F000FFF780B903B0BDE8F043FFF717B903B06A
:10640000BDE8F043FFF780BA03B0BDE8F04309E40C
:10641000534F4368D7F81852026BD7F8101290F810
:1064200000C01D4005EB020EBEEB412F4FEA412696
:10643000184645D3A7F580594FF6F778BCF1020FFF
:1064400014D02169084600295ED16068A368E26A19
:10645000834238BF03460021A36084F82810002A35
:10646000A3D0204603B0BDE8F04310476068D7F8DA
:106470002012B0EB412F68D22069217E090735D563
:10648000D7F8941100F1010E71452BD297F8B41191
:1064900000294BD1012387F8B43189F8013094F8F1
:1064A00000C06368226B921B2A4433445B1B9642F4
:1064B000C4E904E06360226318464FF00005BDD9CB
:1064C000BCF1020F41D021690029BFD0254B1B78B8
:1064D000032B40D089B24FF6F7739942B6D81044D7
:1064E0006060B3E7DFD14FF0000EDCE701A973F085
:1064F00081FB01287FF459AF2069DDF804E094F8AE
:1065000000C06368226BCEE799F800E0BEF1030F8C
:1065100012D01FFA81FEC64594BF4FF0000E4FF017
:10652000010EBEF1000FA8D06068CDE7012189F807
:10653000011094F800C0B6E7DFF82CE0714594BF75
:106540004FF0000E4FF0010EEBE7D7F82032B0EB22
:10655000432FC4D37AE7044B99423FF677AFBEE7A7
:106560009C5B00209C4B0020F7FFFF0F70B5194D7E
:10657000194BC5F8A43B194B85F8B01B002683F8CE
:10658000286A05F6A433C0E954330D23C0F8583106
:1065900040F201130446C0F85C6100F5A271A0F856
:1065A00044317AF013FC1F23C4E9EC36E37801226E
:1065B00005F674059342C4F8A853A4F89C2308BFB9
:1065C000C4F8AC5304F567712046BDE870407AF01A
:1065D000FDBB00BFC02F002055534253C81E0020F2
:1065E000F0B50B7813F0600283B004462BD0202A5C
:1065F00030D14A78FE2A39D0FF2A2DD14A88002A84
:106600003BD1CA88002A38D11F0636D46148624B74
:1066100080F8282AC4F8B423E278012183F894187A
:10662000A4F89C1303F674031F21012AC4F8B013C5
:10663000C4F8A83304F5677108BFC4F8AC3320462A
:106640007AF0C4FB06E04B780A2B1AD00B2B08D04B
:10665000012B2AD0002002E07AF04AFA022003B08F
:10666000F0BD4D4B4A8883F8B52BF3E74F8827B927
:10667000CD88012D01D11B0642D420467AF038FA8C
:10668000ECE7022180F811114FF48071A0F81C1181
:1066900042490123C0E94A11C0E94E33C0E94C32F6
:1066A00000F58E717AF030FBD4E78B88C0681E0647
:1066B000DDB244D40192019A394B42F010020192AA
:1066C000019A026102690192013B02D0019AD2064D
:1066D000F8D4314E294620467AF07CFA294696F8BD
:1066E00094580223402220467AF0A4FA022DB1D118
:1066F000812120467AF034FA002386F89438A9E7FD
:10670000254ED6F8A8389B699847C0B286F8B40BD6
:106710000028B2D0022306F6B43684F811314FF4C3
:106720008073C4E94E55C4E94A66C4E94C57A4F8DD
:106730001C3104F58E7120467AF0E6FA8AE7009261
:10674000009A174B42F020020092009A65F38A12D9
:106750000092009A026102690092013B02D0009A05
:106760009106F8D40C4E294620467AF033FA294691
:1067700096F894580223402220467AF05BFA022DC4
:10678000B6D0012D3FF466AF01212046FFF7EEFEA3
:1067900060E700BFC81E0020C02F0020753B00200E
:1067A000410D030010B50D4B93F8283A022B07D08A
:1067B000033B012B02D80021FFF7D8FE002010BDBB
:1067C000074B93F88118044672F084FE0028F5DA2E
:1067D00001212046FFF7CAFEF0E700BFC81E0020D7
:1067E000C02F0020F8B53F4C94F8286A05467EB1CA
:1067F000012E01D00020F8BD3B4B93F8811872F0B8
:1068000069FE0028F6DA31462846FFF7AFFEF1E7C9
:10681000354FB0F8B433D7F87C28C7F8AC2B1F2B12
:10682000D7F87828C7F8A82B08D1304BD7F87428A8
:106830009A4203D197F88118012919D997F8B63BE4
:106840005A1CD2B207EBC303042A18BF164605220E
:1068500083F8B82B4FF400522846C3F8BC2B022310
:1068600087F8B66B87F89438FBF7AAFB0020F8BDD1
:1068700097F88238013B0F2BE0D872F02BFE0028EE
:1068800027DB94F8283A013B022BB3D9B7F8D83B61
:106890001BB3042284F8282A154AC5F85C61C5E9AF
:1068A0005422D7F87C2887F8B06B934228BF134650
:1068B000D7F8AC2BC5F8583140F20111A5F84411B6
:1068C000D21A05F5A2712846C7F8AC2B7AF07EFAE9
:1068D00090E72846FBF774FB8CE719462846FFF73C
:1068E00045FE87E7C81E0020C02F002055534243B5
:1068F0009C3B002038B5084B1B6853B1DB6914463C
:106900000D4698474FF4007302682A600020236008
:1069100038BD1B68FFDE00BF603B002008B5054B9B
:106920001B6823B11B699847013840B208BD4FF07E
:10693000FF3008BD603B00200020704700207047FA
:10694000704700BF704700BFD0ED007AD0ED036AFA
:1069500030EE677AE6EE877AB0EE670AC0ED007A2D
:10696000704700BF90ED017AB5EE407AF1EE10FA73
:10697000F0EE407A09D19FED0D7A60EE870AF7EECE
:10698000006A86EEA07A80ED017A31EE077A90ED0A
:10699000000A80ED021AC1EE076A77EEC07AC0EDF8
:1069A000036AA6EEA70A80ED000A7047DB0FC94014
:1069B000D0ED056AD0ED017A90ED066AD0ED025A6D
:1069C00090ED035AC0ED066AB0EE407A26EEA70AB3
:1069D000D0ED007A80ED057AA7EE870AD0ED077A30
:1069E000A5EE860A90ED086AD0ED045AC0ED087A4B
:1069F000A5EE670AA5EEC60A80ED070A704700BF3C
:106A0000F0EE406AD0ED007A90ED050A90ED037A41
:106A100090ED016AD0ED025AA7EEA60AD0ED047AF5
:106A200027EE407A67EEC07AA6EE267AE5EEA67AE1
:106A300090ED066AC0ED067A36EE076A80ED056ACB
:106A4000704700BF03685A1C02601970704700BF8E
:106A50002DE9F04FD0E90031856889B04A1C00EB80
:106A600081045918F1EE407A0591002D92FBF3F163
:106A700003FB1122426000F1800A84ED200AC4ED7C
:106A8000407A00F5807240F38780691C012603F18B
:106A9000FF3B06914FF002090795B6460599A1EB19
:106AA000090090FBF3F103FB1100411C91FBF3F48F
:106AB00003FB14110AEB800802EB800CF14501EB9B
:106AC0000E00D8ED006A90FBF3F49CED006AA3EB96
:106AD000090603FB140055DDCDE90198CDE903C695
:106AE00037460D46044641E0AB420AEB840902EB0F
:106AF000840804F1010441DD0AEB850C02EB8506F4
:106B00000135DCED007AD8ED005A96ED007AF4EE0E
:106B1000E67AF1EE10FA0FDD99ED005AF4EEC57A3F
:106B2000F1EE10FA08DDB4EEE65AF1EE10FA58BFB5
:106B3000F0EE456ACCED006AB4EEC67AF1EE10FADA
:106B40000DDDB4EEE57AF1EE10FA08DDF4EEC65A8A
:106B5000F1EE10FA58BFB0EE656A86ED006A0137B3
:106B60005F4530DAB0EE476AF0EE676AA342BBDCFD
:106B7000AB429046D1464FF00104BDDC1646D446E8
:106B80000125BEE706990EF1010E714509F10209D2
:106B90000BF1FF3B82D1079D0599491B91FBF3F057
:106BA00003FB10130AEB830102EB830391ED000A50
:106BB00093ED007A30EE470AF6EE007A20EE270ACF
:106BC00009B0BDE8F08FDDE90198DDE903C698ED75
:106BD000006ADCED006A41E08B420AEB800C02EBBC
:106BE000800700F1010041DD0AEB810502EB810421
:106BF0000131D5ED007AD7ED005A94ED007AF4EE2C
:106C0000C67AF1EE10FA0FD59CED005AF4EEC57A73
:106C1000F1EE10FA08D5B4EEC65AF1EE10FAD8BF6C
:106C2000B0EE456A85ED006AB4EEE67AF1EE10FA50
:106C30000DD5B4EEE57AF1EE10FA08D5F4EEE65A89
:106C4000F1EE10FAD8BFF0EE656AC4ED006A0136C5
:106C50005E4597DAF0EE476AB0EE676A8342BBDCC6
:106C60008B421746D4464FF00100BDDC1446554612
:106C70000121BEE703685A1C02601970704700BF0B
:106C8000024B186803681B68184700BFC05D0020EE
:106C9000007970470079C0F34010704700794009CF
:106CA000704700BF90F83C20034602F0FF0012B18D
:106CB000002283F83C2070474FF480538381704753
:106CC0004FF40063838170474FF400638381704702
:106CD0004FF40063838170474FF4006383817047F2
:106CE0004FF40063838170474FF4006383817047E2
:106CF000074B10B403F11001002453F8042B824217
:106D000008BF43F8044C8B42F7D15DF8044B704741
:106D1000C45D002070B5374C608CA38AB4F92C5048
:106D2000B4F92660B4F91AC01B1A208C00FB03F3D7
:106D3000B4F92A0005EBE335C00290FBF5F000EB57
:106D4000E330A0F57A6EB4F9243020630EFB0EF523
:106D50002D1305FB06F605FB03F3B4F91C500EFBDF
:106D60000CFC0EFB05F51B1403EB65334FEAEC2C12
:106D7000B4F918500CEBE62C0CEB850C0233B4F98B
:106D80003450A66BE48B9B1003F500430CFA05FC12
:106D900004FB03F30CF1020C4CF25034A6EBAC0CE8
:106DA0002C4104FB0CF4002C4FEAD333ABBF64003E
:106DB000B4FBF3F3B4FBF3F35B0089B11C120E4D8B
:106DC00004FB04F440F6DE3606FB04F403FB05F591
:106DD000241404EB254404F6CF6403EB24130B6066
:106DE0002AB100EB80004000083000111060012043
:106DF00070BD00BFC05D002043E3FFFF012070476E
:106E0000012070472DE9F04F734DE86BB5F8403025
:106E1000B5F94CE0B5F948C0B5F84680B5F94E6013
:106E200085B0C3EB2014009204FB04F4B5F94420B0
:106E3000CDF80CE0241302FB04F45B00B5F942200A
:106E40000296C3EBE00302FB03F3A41304EBE32479
:106E5000EB6D0193A4F5FA30B5F94A30AC6580FBCF
:106E600000EA4FEAE37B03FB0AF98CFB00C20EFB4E
:106E70000B99A3FB0E3BCB4412031B0A42EA1C52A4
:106E800043EA0B634FEA0C3C13EB0C0342EB2B225F
:106E9000A3FB083C02F5004208FB02CC4FEAEC736E
:106EA0004FEA6C0953EA6C0C0F46B5F9501000F02C
:106EB0009180029E019A86FB0008C2F5801C01FBAE
:106EC0000AFA4A464FEA48484FEAE17948EAD03898
:106ED0000EFB09A94004A1FB0E1E4118F14449EB29
:106EE000080900200CF00048039E411848EA5C089D
:106EF0004FEACC7CBCEB010C09EBC60968EB090836
:106F00001CEB0C0E48EB08011EEB0C0E48EB0101CC
:106F100088014FEA8E1940EA9E601EEB090E41EB94
:106F20000001890041EA9E714FEA8E0E1EEB0C0EA5
:106F300048EB01014FEA8E00890010EB0C0041EA9A
:106F40009E7148EB01017AF081FFB5F956304FEAA6
:106F500061384FEA503E4EEAC14EDA1703FB08F99A
:106F600084460EFB0299B5F95400B5F95220A3FBF3
:106F70000E35A94403FB08F50EFB0955A3FB0E3E95
:106F800075445B0E43EAC51313EB0C0341EB6565D7
:106F90004FEAE07E00FB01F10EFB0C11A0FB0C0C94
:106FA0006144C00C40EA41301B1845EBE1451B0A27
:106FB00043EA056303EB02130FB11B0A3B60009B1E
:106FC00023B104EB8404803424121C60012005B03A
:106FD000BDE8F08F0023EFE7C05D0020012070477F
:106FE000012070472DE9F04FC54C83B0B4F8640020
:106FF000236ECDE90012B4F86620A3EB002394F9C8
:107000006800A2FB0326A3FB0335C71700FB05F5A9
:10701000B60446EA923603FB07559204A0FB03032D
:1070200080182B4443EB0603002B02DA013843F1AE
:107030000003009ADF17C4E92037002A00F00C8112
:1070400003FB07F0A3FB032E0EEB400E4FEA921951
:1070500049EA8E694FEAAE1609FB07F003FB06000A
:10706000A9FB03968019D4F8885000F143814FEAB8
:10707000192949EA00694FEA202B94F96E004FEA7A
:10708000E07C00FB0BF609FB0C66A0FB090C16EB81
:107090000C0600F12B81B4F96980B4F96BC040098A
:1070A00040EAC6600146A8F5804894F96D004FEAB1
:1070B000883808EB66184FEAE07A00FB0EF602FB10
:1070C0000A66A0FB02A00644B6004FEA8A00ACF5AF
:1070D000804C46EA9A76081848EB06084FEAEC7AA4
:1070E0000CFB07F603FB0A66ACFB03CA56447605A5
:1070F00046EADC264FEA4C5C10EB0C0048EB060637
:10710000002EC0F2EC8094F974C00CFB0BF84FEA2F
:10711000EC7A09FB0A88ACFB09C9000E18EB0908D8
:1071200040EA06204FEA266600F1D48094F9739075
:10713000B4F871A009FB0EFE4FEAE97B02FB0BEEEF
:10714000A9FB0229CE444FEA5C1C4FEA0E1E4EEA10
:10715000127E4CEAC86C12011CEB020CB4F86F20D2
:107160004FEAC23202EB681848EB0E08AAFB03E2B2
:107170000AFB0722920542EA9E224FEA8E5E1CEB32
:107180000E0C48EB0208B8F1000FC0F29E804FEAE7
:107190009C0C94F97720B4F975E04CEA887CA0FB4C
:1071A00005091CEB000C05FB069040EBA80002FB58
:1071B00007F64FEAE27803FB0866A2FB0328464481
:1071C0004FEA0E4812EB080246EBEE7EA2FB0526C4
:1071D00005FB0E66002E71DB520B42EAC642A2FB93
:1071E000052E761305FB06E6002E60DB520A94F9A5
:1071F00078E042EAC6521CEB020440EB6620A5FB95
:10720000052C4FEAEE7602FB06F60EFB0C66A2FB9F
:107210000E2E16EB0E0643D4120C42EA0642A2FBD7
:10722000052C361405FB06C5002D35DBD20942EAD4
:107230004562121940EBE510941840EB0005A418C4
:1072400040EB0505ED0045EA5475E400A41840EB59
:107250000500009A000C1060019A9AB1DA1847EB09
:107260000701D21847EB0101C90041EA5271D2006F
:10727000D21847EB0107002F08DB019B920B42EA73
:1072800087421A60012003B0BDE8F08F43F6FF7318
:10729000D21847F10007F0E77F3245F10005C5E756
:1072A0004FF6FF7C12EB0C0246F10006B4E740F209
:1072B000FF1E12EB0E0246F1000697E741F6FF7E35
:1072C00012EB0E0246F1000686E71CF1030C48F1B2
:1072D00000085CE71CF11F0C48F1000826E76FF07E
:1072E0007F4C10EB0C0046F100060CE71F3046F116
:1072F0000006D0E619F1FF0940F10000B7E600BF33
:10730000C05D002031B10A4BD3ED2A7AFDEEE77A59
:10731000C1ED007A52B1064B9FED067AD3ED2B7A80
:1073200067EE877AFDEEE77AC2ED007A01207047BA
:10733000C05D00200000C8422DE9F04F614DB5F856
:10734000BE30D5F8B000B5F8BCE0B5F8BA40B5F835
:10735000C06085B01B02C01A67EB0707B5F8B830EC
:107360000191AEFB001C0EFB07CCC9091B0441EACE
:107370004C61C9189346A4FB003EB5F8B62004FB47
:1073800007EE4FEA13234FEAC23243EA0E634FEA95
:10739000EC1C4CF1000C9B18A6FB002406FB0744D8
:1073A0004FEAD25242EA44224FEA2E2E4EF1000E0C
:1073B000E41512F5FA6944F10006B9F5FA6F029680
:1073C00076F1000632DAA2FB02A802FB04F603946F
:1073D00008EB46044FEA84084FEA8A0616EB0A06D1
:1073E00048EA9A7844EB08084FEA560A4AEAC87A0B
:1073F000B608B1EB0A0A46EA8876334C6CEB680CA7
:107400009E1B3346029E6EEBA80EA1454FF0FF3443
:10741000A641514627DB00FB07F7A0FB000202EB69
:107420004702C00F40EA4200B9EB0009019C8CB151
:10743000D5F8C400A0FB033200FB0E225B0D43EA2B
:10744000C2235B1A4FEA625262EB0C02DB0B43EA87
:1074500042432360BBF1000F01D0CBF80090012024
:1074600005B0BDE8F08F40F6AC56039C921944F18C
:10747000000402FB04F4A2FB026202EB44024FEAA6
:10748000C208F400341B48EA567862EB0808641816
:107490004CEB080C2146B41942EB0208A41942EB4C
:1074A00008084FEA880848EA9478A400A41B68EB0F
:1074B0000208620842EAC8729A1A6EEB680E134616
:1074C000A9E700BFC05D002024FAFFFF012070473C
:1074D00010B40F4B0F4C1B68D4F8C8001B1AFA2BC2
:1074E0000BD811B1D4F8D0300B6012B1D4F8D4302D
:1074F000136001205DF8044B7047074A13680020B1
:1075000023F0040384F8CC0013605DF8044B70474B
:10751000EC280020C05D0020000000100120704712
:10752000064B00220021C3F8D820C3F8DC20C3F8A2
:10753000E020C3F8E4100120704700BFC05D0020C8
:10754000104B114A1B68D2F8E4105B1AFA2B16D8BC
:10755000D2ED366A92ED377AD2ED387AFDEEE66AF0
:10756000BDEEC77A16EE903AFDEEE77AC38617EEC7
:10757000103A038717EE903A4387012070470020A6
:10758000704700BFEC280020C05D002030B50F4AD6
:1075900083B092F8E8500191B5B9D2F8EC509DB1A2
:1075A0002B681A6882B19B6873B1044628469847D5
:1075B00050B12B68019922461C6828460B4621468B
:1075C00003B0BDE83040084703B030BDC05D0020C7
:1075D0000B4B70B5D3F8F0608EB133681A6872B196
:1075E0009B6863B1054630460C46984738B133680E
:1075F0002A46196830462346BDE87040084770BDEA
:10760000C05D00202DE9F041DFF888801F4FD8F8D9
:10761000D8203B68B8F8DC10118343B39B699847C6
:1076200028B300263B6813B11B69984790B9B6F59B
:107630007A7F21D009F0F0FF013604460D4609F0AB
:10764000EBFF001B61EB0501B0F57A7F71F10001E2
:10765000F5D3E7E7D8F8D830B8F8DC205A83B6F588
:107660007A7F4FF0FF3018BF0020BDE8F081084B53
:107670003B601B689847D4E7D8F8D830B8F8DC20CE
:107680005A834FF0FF30BDE8F08100BF603B00201F
:10769000300C0020A43800202DE9F84FDFF8BCA002
:1076A000DAF89C009046BAF8A0204283002B45D01F
:1076B0009B46294F8946C34441F289363A6852B104
:1076C0000023546849461A464046A047A0B93B6883
:1076D0000BB11B699847013E34D009F09DFF044669
:1076E0000D4609F099FF001B61EB0501B0F57A7FAB
:1076F00071F10001F5D3E1E741F289363B6813B13E
:107700001B69984780B9013E1CD009F085FF0446EB
:107710000D4609F081FF001B61EB0501B0F57A7F92
:1077200071F10001F5D3E9E708F10108D84509F541
:107730000079C1D1DAF89C00BAF8A02002830020B9
:10774000BDE8F88FDAF89C30BAF8A0201A834FF021
:10775000FF30BDE8F88F00BF603B0020A438002058
:107760002DE9F84FDFF8C0A0DAF89C009046BAF88F
:10777000A0204283002B48D09B462A4E8946C34412
:107780003268FAB141F289370023D46849461A4673
:107790004046A0473368B0B10BB11B699847013F21
:1077A00037D009F039FF04460D4609F035FF001BBC
:1077B00061EB0501B0F57A7F71F10001F5D3326814
:1077C000002AE1D1002341F2893713B11B699847A0
:1077D00088B9013F1DD009F01FFF04460D4609F08E
:1077E0001BFF001B61EB0501B0F57A7F71F1000111
:1077F000F5D33368E9E708F10108D84509F50079C0
:10780000BED1DAF89C00BAF8A02002830020BDE8BF
:10781000F88FDAF89C30BAF8A0201A834FF0FF30C6
:10782000BDE8F88F603B0020A438002038B514462E
:10783000002944D0344BDFED355AD3ED3D7AB3F90E
:10784000102193ED400AB8EEE77A05EE102AC7EE54
:10785000256AB3F90C210D46D3ED3E7A06EE102AC7
:10786000F8EEE77AB3F90E21C7EEA54A05EE902AA5
:10787000B3F90A2107EE102AF8EEE55AB3F9082108
:10788000B8EEC77A07EE902AA6EEA57AB8EEC55AEA
:10789000B8EEC66AF8EEE77AA6EE856AE6EE877A73
:1078A00093ED417AB8EEC77AB8EEC00AA6EE867AB2
:1078B000A6EE870AA4EEA70A7BF0B0F928600CB305
:1078C000114B9FED126AD3ED3E7AB3F9FE20B3F966
:1078D000FC30F8EEE76A07EE102A86EE860A07EE1D
:1078E000903AB8EEC77AF8EEE77A20EE070AB6EEDD
:1078F000006AA7EE860ADFED066A20EE260A7BF014
:107900008DF92060012038BDC05D00200000F04AE4
:107910000000C8422DE9F0410446D0E9003013448C
:1079200083421DD80D4601EB0208B2B104F10C07E9
:10793000002601E0A84510D023695A1C2261234487
:1079400015F8011B1973042AF4D139462046FBF7B8
:1079500003F9A845C4E90460EED16069BDE8F0818F
:107960004FF0FF30FAE700BF2DE9F0410C4E3568CB
:1079700073691D4011D0DFF82C800127B5FA85F41A
:10798000C4F11F0408EB840307FA04F4D3F81401CC
:1079900003689847A5437461F0D1BDE8F08100BF4A
:1079A000003C0140C05D002010B54FEA511E02446A
:1079B00000EB8E0C624529D901F01F034FF0FF3414
:1079C00050F82E1004FA03F30B4093FAA3F3B3FA22
:1079D00083F3DBB2202B16D10CF104018A4202D8CA
:1079E00017E08A4212D98C460431DCF8003093FA51
:1079F000A3F3B3FA83F3DBB2202BF2D0ACEB000C91
:107A000003EBCC0010BD03EB4E1010BD4FF0FF3068
:107A100010BD204610BD00BF0369416890ED067A95
:107A2000F0B4C56A394E876853EA010204BF316871
:107A300041606A1C30EE077A0133012A80ED067A34
:107A40000361C26240D090ED075AD0ED096A3468F4
:107A500007EE902A70EE455AB8EEE76A611AC5EE55
:107A6000867AB94277EE857A30EE670AC0ED087AF9
:107A7000E5EE806AC0ED077AC0ED0A6AC0ED096ADA
:107A800001D8F0BC7047012A29DD07EE905AF8EEC4
:107A9000E77A86EEA76AB5EEC06AF1EE10FA1EDB51
:107AA000F1EEC67AF4EE677AF1EE10FA17D6D0ED61
:107AB000056AF4EEE76AF1EE10FA13D5037BEBB139
:107AC0000323F0BC03707047326880ED080A521A35
:107AD000BA424FF0000180ED070A4162D1D9DFEDD3
:107AE0000C7AE4E707EE903AF8EE677A0223C7EEE5
:107AF000276AF0BC0370C0ED066A704731684160C8
:107B0000002203618261C362BBE700BFEC28002052
:107B100000000000DFED4F4A10B5844600F1480E2A
:107B20000346B1EC017AD3ED067ADA6A77EE877A0A
:107B30000132012AC3ED067ADA6254D093ED075A76
:107B400093ED096A07EE902A77EE455AF8EEE77A48
:107B5000C5EEA76A76EE857AF0EE466A37EE677A6A
:107B6000C3ED087AE5EE876AC3ED0A6AC3ED077ACA
:107B7000C3ED096A18337345D3D1374C4168226885
:107B80000369521A816801338A4203612AD990ED50
:107B9000056A00F1300EDCF82C20DCED0A6A012ABF
:107BA00002F1FF3126DD07EE901AF8EEE77A86EE55
:107BB000A77AB5EEC07AF1EE10FA1BDBF1EEC77AC8
:107BC000F4EE677AF1EE10FA14D6E645B4EEE76A01
:107BD0000CF1180C16D0F1EE10FADCD5037B6BB368
:107BE0000323037010BDF0EE477AF0EE646A83ED74
:107BF000087ABBE7DFED177AE645B4EEE76A0CF1E9
:107C0000180CE8D1F1EE10FAE8D407EE903AD0ED76
:107C1000066A90ED0C7AD0ED125AF8EE677A0223DC
:107C200086EEA76A0370C7EE276A85EEA77A80ED15
:107C3000066AC0ED0C6A80ED127A10BD0022216840
:107C4000416003618261C362026343648264C3650D
:107C500010BD00BF00000000EC280020B0EEC06A9C
:107C6000F0EEE05AF4EEC65AF1EE10FAF0EE407A79
:107C70000EDCB5EE400AF1EE10FA4BD0F4EEC65A27
:107C8000F1EE10FAF0EE466A50D5B0EE655A03E018
:107C9000F0EE656AB0EE465A85EE267A9FED252A0B
:107CA0009FED253A9FED254ADFED254ADFED252A98
:107CB000DFED253ADFED256AA7EE023AE7EE223A3C
:107CC000A7EE034AB7EE005AE7EE044AA7EE235A9E
:107CD000E7EE246AF4EEC65AB1EE667A87EE050A3C
:107CE000F1EE10FA48BF9FED1A7AF5EEC00A48BFD0
:107CF00037EE400AF1EE10FA48BF9FED167AF5EE26
:107D0000C07A48BF37EE400AF1EE10FA48BFB1EE34
:107D1000400A7047DFED107A9FED100AF5EEC00AB9
:107D2000F1EE10FA58BFB0EE670A7047B0EE465A4F
:107D3000B2E700BF39094E3DE3B59EBE88FA16BED4
:107D400045FE7FBF99FB243F69A2163EA7DFA8B47A
:107D5000DB0FC93FDB0F4940A7DFA834DA0F4940EA
:107D600091ED007AD0ED047A90ED054AD0ED064A07
:107D700090ED075AD0ED085A90ED096AD0ED0A6AE5
:107D8000E7EE077AF7EE003AC0ED047A91ED007A5B
:107D9000D1ED017AA7EE274A90ED0B7A80ED054AE6
:107DA00091ED024A91ED003AD0ED0C7AE3EE044AEF
:107DB000C0ED064AD1ED004A35EE245A80ED075A4F
:107DC000D1ED014A91ED005AE4EE855AC0ED085A12
:107DD000D1ED015AA5EEA56A80ED096AD1ED015AEF
:107DE00091ED026AE5EE866AC0ED0A6AD1ED016A9C
:107DF00037EE267A80ED0B7AD1ED026A91ED007AAA
:107E0000E6EE877AC0ED0C7A91ED026AD1ED016A57
:107E1000D0ED0D7A90ED0E7A90ED0F4AD0ED104A2C
:107E200090ED115AD0ED135AE6EE267A75EEA35A6C
:107E3000C0ED0D7AD1ED026AD0ED127A90ED006AB4
:107E4000A6EEA67AD0ED016A80ED0E7A91ED027A67
:107E500034EE074A90ED027A80ED0F4A91ED004A28
:107E600074EE844AC0ED104AD1ED014A35EE245A31
:107E700080ED115A91ED025AC0ED135A77EE857AD2
:107E8000C0ED127AD1ED017AD1ED005A91ED025A8E
:107E900067EEA77AE5EEA57AE5EE057AA5EEA76A84
:107EA00080ED006A91ED016AE6EE276AC0ED016A95
:107EB000D1ED026AA6EEA77A80ED027A90ED037A00
:107EC00077EE277AC0ED037A704700BF2DE9F04FB7
:107ED0004FF0000989B0864600F1100506460346BA
:107EE00000F13008074648462C46CDF80CE08B469A
:107EF0009C46B24600283CD10CF1040CA445FBD1B1
:107F0000032800F1010151D09C46AA46029398B182
:107F1000DCED047A0192AAEB0903B6467246F3EC53
:107F2000016A92ED007AE6EEC77A53450EF1100E23
:107F3000CCED047AF2D1019ADCED046A15ED047AF5
:107F4000C6EE877A0CF1100CC4450AF1100ACCED8C
:107F5000007ADCD1029B04361433084608F1040889
:107F600014351034103709F104099C46B246002834
:107F7000C2D0DCED007A0192D64639467246F1EC69
:107F8000016A92ED007AE6EEC77A99420EF1100E80
:107F9000CCED007AF2D10CF1040CA445019A0AF15F
:107FA000040AE6D1032800F10101ADD1DDF80CE0AF
:107FB0000023594604930593069307937646774624
:107FC00004AD0020F2EC017AE5EC017AB0B104AC2A
:107FD0003B46B4EC017AF3EC016AE6EEC77AB342B1
:107FE00045ED017AF5D1013004280BD0F2EC017A8D
:107FF00010371436E5EC017A0028E8D11037143632
:108000000120DFE708AD75ED017A10310EF1400E69
:1080100004287446A1F1040241ED017A1ED0734692
:10802000F3EC016AB1EC017AE6EEC77AA342C2ED45
:10803000007AF5D15EED016A87EEA67A013882ED0D
:10804000007A17D0AEF1140E103C114675ED017A8E
:108050000428A1F1040241ED017AE0D15EED016A4C
:1080600087EEA67A103CAEF1140E032001ED017AE2
:108070001146EBE709B0BDE8F08F00BFDFED297ACC
:10808000B4EEE70AF1EE10FA28DD9FED277A30EE24
:10809000470AB4EEE70AF1EE10FAF8DCDFED237AD6
:1080A000B4EEE70AF1EE10FA2FDD30EE670A37EE94
:1080B000C00A60EE007A9FED1E7A9FED1E6ADFED2A
:1080C0001E6AA7EE876A9FED1D7AE7EE866A60EE6C
:1080D000275AA7EEA67AA5EE870A7047DFED187A31
:1080E000B4EEE70AF1EE10FAD8D59FED0F7A30EE34
:1080F000070AB4EEE70AF1EE10FAF8D4DFED0B7AD6
:10810000B4EEE70AF1EE10FACFDC9FED0E7AB4EE92
:10811000C70AF1EE10FA44BF30EE270A37EE400AE4
:10812000C7E700BFDB0F4940DB0FC940DB0FC93F8A
:108130009A7C2E36FAAF4FB93587083CA4AA2ABEDE
:10814000DB0F49C0DB0FC9BF10B5404CB4FBF2F4E4
:10815000A14219D3DFED3E7AF7EE005AB0EE677A0E
:10816000B0EE676AF0EE676A0023C0ED005AC0ED1A
:10817000017A80ED027A80ED036AC0ED046A8361C2
:1081800043610362C36110BD07EE902AB8EE677ABF
:10819000DFED307A27EE277AB7EE006AC6EE076A7F
:1081A00007EE901A9FED2C7AF8EE677AB0EE405AFF
:1081B00067EE877AC7EEA64AFDEEE47A17EE902ABC
:1081C0002032402A3FD8B0EE640AFFF757FFB0EEE6
:1081D000404ADFED227A34EEA70AFDEEC07A17EEB0
:1081E000902A2032402A29D8FFF748FFF8EE006A8B
:1081F00060EE266A012B1CD0B7EE006A36EE406AAC
:10820000F6EE004A66EE244A35EE055AF7EE007A9D
:1082100084EE057A77EE275A37EEC75A84EEA57AB0
:10822000C6EE257A86EEA56AC5EE256AF0EE475AB7
:108230009AE7B0EE666AF7EE004AE5E7DFED086A16
:108240009FED030AD6E79FED024AC2E720A107008F
:1082500000000000BD378635DB0FC940DB0FC93F8A
:1082600000000080DFED077A30EE270AFDEEC07ACD
:1082700017EE903A2033402B00D8FFE69FED020A1C
:10828000704700BFDB0FC93F000000002DE9F84F29
:10829000DDF82CB09DF828408946002C1BF8011B06
:1082A0000CBF4FF020084FF030081C1E0546174643
:1082B00008463ADB00295CD0002C55D04FF0000A6C
:1082C0005B4600E064B313F8016B013C002EF9D16A
:1082D000BAF1000F2FD1264644B14D4541462846FC
:1082E00000D2B847013CF8D10B9B18780146A0B1E9
:1082F0004FF0FF344FF0000A00E09B464D45284602
:1083000000D2B8475B4613F8011B0029F5D10B9B3F
:10831000F61A5E44BAF1000F10D13046BDE8F88F6E
:10832000BAF1000F1BD15646E0E7634229B31C4661
:108330004FF0010AC4E70028E0D10646002C04F102
:10834000FF3AEADD54464D454146284600D2B8473B
:10835000013CF8D2013656443046BDE8F88F064657
:108360000028DAD02646C9E72646A2464FF0FF3459
:10837000C4E72646002CB0D1CFE76FEA040A0E46C8
:10838000E0E700BF0FB430B583B006AB0A4C53F83A
:10839000042B0193D4E9DD0171F09AFF05462068B2
:1083A00003685B6998470028F9D0284603B0BDE808
:1083B000304004B0704700BFC05D00200EB410B55F
:1083C00083B005AB044653F8042B0749009301A87A
:1083D000019471F07DFF019B00221A7003B0BDE88B
:1083E000104003B0704700BF756C00080CB4F0B5C6
:1083F0003D4CD4F87C33ADF5277D002B6FD094F83D
:10840000843399420BD9D4F8882301238340134243
:1084100005D10DF5277DBDE8F04002B07047334B24
:10842000334A1B68A2FB030292094FF47A7101FBE5
:10843000123306A82F49FFF7C1FF06AB03442E49AC
:10844000AC9A01930646ADAB01A8009371F040FFD2
:10845000019B0A22591C01911A70019B0022591C90
:1084600001911A70D4F87C53BDB12B685B6A2BB1B3
:10847000284698470028CCD0D4F87C539DF8181093
:108480000029C6D00DF119042B6828461B689847AF
:1084900014F8011B0029F7D1BBE7D4F88073002F33
:1084A000B7D0304426AB841CFD2206A9ADF81020BD
:1084B00018462246CDF81250ADF816507CF05AFC02
:1084C00002220346044402A93846CDE902343AF0B8
:1084D00025FE0DF5277DBDE8F04002B07047D4F8C9
:1084E0008033002B8BD194E7C05D0020EC28002066
:1084F000D34D621010FD0808456A0008184A10B5EF
:10850000D2F88C43033004EB9003B3F5007F18D806
:1085100002EB8101C2F88C3302F5647202EB840431
:10852000D1F8902B20F003001044C3F50073C1F87C
:10853000900B0C4A9B0004210020FFF757FF2046B8
:1085400010BD00210846084AFFF750FF074AD2F83D
:10855000B030002443F00073C2F8B030204610BDA4
:10856000C05D00201CFD080840FD08080000001048
:1085700038B50568EB690446F3B1987800B938BDA1
:10858000B3F90A2007EE902AF8EEE77A0120C4ED4D
:10859000057AB3F90C2007EE902AF8EEE77AF1EEAF
:1085A000677AC4ED047AB3F90E3007EE903AF8EE2C
:1085B000E77AC4ED067A38BD09211420FFF79EFF43
:1085C0000346E861D9E700BF38B50568EB690446A2
:1085D000E3B1987800B938BDB3F9042007EE902ACA
:1085E000F8EEE77A0120C4ED047AB3F9062007EE2D
:1085F000902AF8EEE77AC4ED057AB3F9083007EE71
:10860000903AF8EEE77AC4ED067A38BD09211420D5
:10861000FFF774FF0346E861DBE700BF38B5056884
:10862000EB690446E3B1987800B938BD9A88D2BAAC
:1086300007EE902AF8EEE77A0120C4ED047ADA8892
:10864000D2BA07EE902AF8EEE77AC4ED057A1B89D4
:10865000DBBA07EE903AF8EEE77AC4ED067A38BD59
:1086600009211420FFF74AFF0346E861DBE700BF5A
:1086700038B50468E3690D467BB1987800B938BD18
:108680005B89094ADBBA82FB0312DB17C3EB2213B7
:1086900003F26D132B80012038BD09211420FFF750
:1086A0002DFF0346E061E8E7797878782DE9F0411D
:1086B00003EB4306964602EB460612F9067B86B0AC
:1086C0000346754692F80080A3EB0804A3EB070C61
:1086D000002CB8BF6442BCF1000FB8BFCCF1000C55
:1086E0006445B8BF154602F10602B8BF4FFA88F7D5
:1086F000B242E7D16A889EF80000B842144614D10D
:10870000BEF80200A1EB0008A1EB020CB8F1000FCB
:10871000B8BFC8F10008BCF1000FB8BFCCF1000C25
:10872000E045BEBF7546024604460EF1060E76458C
:10873000E1D16A7904922A79CDE902422878054A82
:10874000CDE9001003210120FFF750FE284606B0B6
:10875000BDE8F08150FD08084B1EDBB2062B98BF28
:108760002D4AF0B596BF02EB43034FF480761E8A84
:108770002A4C431E012B87B039D9B4F83839B4F8E4
:10878000305983B304F6381704F5136404F1100E5E
:10879000A6EB050CF21ABCF1000FB8BFCCF1000C2F
:1087A000002AB8BF52429445C4BF3C461D46774696
:1087B0003EF8083B002BEBD10128258821D0022868
:1087C00013D1174BA2790592A2880492A2780120B6
:1087D000CDE90252CDE90016124A0321FFF706FE49
:1087E000204607B0F0BD04F513640F4BEAE7B4F878
:1087F000E038B4F8D85833B104F50E6704F6D8045D
:10880000C4E70A4BDEE7094B054A04F6D804012801
:1088100018BF1346D6E700BF08530808300C0020E5
:1088200094FD0808A4FD08089CFD08088CFD0808B4
:1088300003685A1C02601878704700BF03681A4624
:10884000591C016012F8021B0260587841EA0020AE
:10885000704700BF10B402681346511C016013F842
:10886000021B0360D31C5478036093781B0443EA13
:108870000423141D0460D0785DF8044B0B4343EAD5
:108880000060704712B370B50446864604E0981B3A
:1088900017D114EB0C0C15D01EF8013BA3F14100CD
:1088A000192811F8010BA0F1410598BF2033192DAB
:1088B000A2EB0E0C00F12006E9D91B1A04D1002806
:1088C000E7D170BD604670BD184670BD1046704758
:1088D00010B402888378174C02F0030101EB4101C8
:1088E000013B03EB810304EB4303C1781B8CA2F52E
:1088F000FA62920840F2B55404FB02334A1E134454
:10890000017942798479008903EB430301EBC301C8
:10891000C1EB0111084B02EB8102C2EB02122344AE
:1089200003EB820300214FF47A72C3FB02015DF86E
:10893000044B70470853080880436D38F8B5164655
:108940001F460446394630464FF47A72002379F0C8
:108950007DFA3B4D3B4B054483FB05602844E917FA
:10896000C1EB601183FB01030B44374EC817C0EB0A
:10897000631086FB003CC317344EC3EBAC0386FB8D
:1089800003764FEAE37ECEEBE61EC1EB0116A5EBC4
:10899000860CC0EB0015A1EB8501617103EB43016F
:1089A000A0EBC10040F2B55101FB1E33B3F5896F56
:1089B00084F806C020714FEA8E0635DA40F2DA21DB
:1089C0008B4237DCB3F5B77FB4BF4FF0000E4FF0EA
:1089D000010E1F490EEB4E0001EBC0017546C88E1B
:1089E0004FEA4E071B4907EB0E0C01EBCC0C0CF1C8
:1089F000160C0B2101E03CF8020D984211DD013903
:108A0000F9D11349774401EBC701088C01210133E7
:108A100006F5FA6E1B1A7544A170E3702281258059
:108A2000F8BD0131C9B2F2E7032540F29650AE46D7
:108A30000627D7E7022540F22940AE460427D1E7B2
:108A400080BC92C789888888ABAAAA2A73B06D16A1
:108A5000085308082853080830B52F4C86460D46A1
:108A60000FCC8DB0EC46ACE80F000FCCACE80F009B
:108A700094E80F001EF0030F8CE80F000FD1274B76
:108A8000274A03FB0EF3B2EBB30F43D3254AB2EBF5
:108A9000331F34BF01220022C2F11D0200E01C225C
:108AA0000EF1FF33002B019240F26D12194602FBCA
:108AB0000EF2B8BF0EF1020102EBA1021A491B4CE3
:108AC00081FB0301DB17A3EB61100244C3EBE1134D
:108AD0001A44253284FB02311144D317C3EBA1039E
:108AE000C3EBC303D31AADF10402EE4602EB8501DA
:108AF0005EF8040FC21884FB023C9444D317C3EB06
:108B0000AC03C3EBC3037145A2EB0303F0D1C01A5E
:108B10000DB030BD1D22C3E788530808295C8FC201
:108B2000285C8F020AD7A3001F85EB51932449923A
:108B30000C4B10B553E9024354EA030209D1014634
:108B400040F201130020C1F80230887108800881CA
:108B500010BD054A1268121943F10003FFF7EEFE3B
:108B6000012010BDE0690020EC28002030B5144D34
:108B7000D5F8181CD5F81C3C51EA030283B0044612
:108B800009D1002040F201132080C4F80230A07106
:108B9000208103B030BD0B4A1268521843F1000324
:108BA000FFF7CCFEB5F8203CADF8063020460DF1BD
:108BB0000602214670F07EFF012003B030BD00BFE9
:108BC000C05D0020EC28002088422DE9F0414FF0E4
:108BD00001043DD301FB04F4B0FBF4FC8C45F9D255
:108BE0003CB3002616E0BCF1090F274698462C46F8
:108BF00023DD002A0CBF4FF0570E4FF0370EF44420
:108C0000B94288F800C003F1010306F1010610D84B
:108C1000B0FBF5FCB4FBF1F504FB1C00002EE2D127
:108C2000BCF1000FDFDCA1420AD90CF1300C03F8D3
:108C300001CB00221A70BDE8F0814FF0300EDEE764
:108C4000B0FBF5FC2C4605FB1C00B5FBF1F5E7E796
:108C50008446C6E72DE9F04104469442154608468D
:108C600009D2B4FBF2F6154B05FB16441B5D00F868
:108C7000013BBDE8F081B4FBF2F69642B6FBF2F799
:108C80000CD20E4B05FB176705FB1644DA5D00F8A6
:108C9000012B1B5D00F8013BBDE8F081BA42B7FB38
:108CA000F2F807D9054B05FB187813F8082000F8EF
:108CB000012BE7E74046FFF7CDFFF3E7ECFD08089F
:108CC000B5EEC00ADFED347AF1EE10FACCBF30EE2B
:108CD000270A30EE670ADFED317A20EE270A30B539
:108CE000FDEEC07A87B017EE904A054684EAE4703C
:108CF000002303A9A0EBE470CDE90033029371F0E7
:108D00003FFA002CB4BF2D23202303A88DF8003098
:108D100078F0E0FA012829D0022833D003281DD0AA
:108D200003A968467CF072F8684678F0D3FAC41E4E
:108D3000E4B22246694628467CF01CF800232B55F5
:108D4000284678F0C7FA2E232B5401300DEB04018E
:108D500028447CF0E2F8284607B030BD302303A950
:108D600068468DF801307CF051F8DDE743F23002BF
:108D7000302303A96846ADF801208DF803307CF05C
:108D800045F8D1E743F2300303A96846ADF8013056
:108D90007CF03CF8C8E700BF6F12033A00007A4449
:108DA0000278202A034600F10100F9D0092AF7D001
:108DB0002D2A29D02B2A03BF5A78B7EE000A034682
:108DC000B7EE000AA2F13001C8B20928DFED4C7AF3
:108DD00010D8F2EE046A07EE101AB8EEC77A13F84C
:108DE000012FA7EEA67AA2F13001C8B20928F0EE51
:108DF000477AF0D92E2A49D0197801F0DF014529A8
:108E000007D020EE270A70475A78BFEE000A0346C3
:108E1000D8E710B459782D2962D02B2954D0A1F16C
:108E20003002092A03F1010355D80024002202EB85
:108E3000820201EB420213F8011FA1F13000092860
:108E4000A2F13002F3D9B2F59A7F134628BF4FF44E
:108E50009A73072A50D9DFED2B6A1A46B7EE007ACB
:108E6000083A072A27EE267AFAD803F007032BB12F
:108E7000F2EE046A013B27EE267AFBD16CB3C7EE13
:108E8000877A5DF8044B20EE270A70475978A1F1E4
:108E90003002D0B2092803F10103AED8F2EE046A21
:108EA000F0EE665A07EE102AB8EEC77A13F8011FE3
:108EB00087EE266AA1F13002D0B2092866EEA56AD3
:108EC00077EE867AEED998E79978A1F13002092AEF
:108ED00003F10203A9D9B7EE007A67EE877AD0E7EB
:108EE0009978A1F13002092A03F1020388BFB7EE95
:108EF000007AC4D8012499E7B7EE007AB7E700BF3B
:108F00000000000020BCBE4C0378202B024600F17C
:108F10000100F9D0092BF7D02D2B08BF5378A3F10E
:108F20003001CBB206BF02464FF0FF3C4FF0010CC0
:108F3000092B4FF0000000D9704712F8013F00EBF9
:108F4000800001EB4000A3F13001CBB2092BF4D932
:108F50000CFB00F0704700BF70B5344D2B787E2BB2
:108F600001D0002070BD08224FF4FC4341F22100E3
:108F700019B200294FEA4303B6BF80EA41019BB210
:108F80008BB2013AF4D1B5F8011069B32848294CE5
:108F9000A042E6D206384618A642E2D241F2210C9F
:108FA0000529DED9864214D0013806F1FF3E10F8BB
:108FB000012F082183EA02231AB2002A4FEA430351
:108FC000B6BF8CEA42029BB293B20139F4D170452C
:108FD000EDD1318849B1B21DA242C2D27218A2426B
:108FE0003046BED21646DBE7134E741E41F2210016
:108FF000A44614F8012F082183EA02231AB2002A9A
:109000004FEA4303B6BF80EA42029BB293B20139F2
:10901000F4D16645ECD17288D01A084A331D5B1B27
:10902000B0FA80F04009A2F8243C70BD00000E08A0
:1090300007000E080000100801000E08C05D0020A7
:109040002DE9F04FB24BB34A93F8543102EB43038E
:109050008FB05B7813B1012007F034FAAE4EAF4BFE
:109060004FF0030AF31A03934FF00009D346374633
:10907000AA4B0793039BAA4ACDE90A99CDE90C991B
:10908000CDE908731369002BC0F2D981A44BF322F8
:10909000DA60A44ACDF830900123BA428DF834301A
:1090A00000F2BE810B937E238DF8283008214FF407
:1090B000FC4341F221001AB2002AABBF5B0080EAF8
:1090C00042029BB293B20139F5D1974AADF8123002
:1090D000964B934280F0D4819846904B0297394644
:1090E00041F221051A46B8F80200B8F800308DF8B0
:1090F0001990C0F30B06B41DADF81440C3F30B0474
:109100001B0B8DF818300304ADF8164000F11081E8
:1091100006328A4200F2838105AF0DF11A0A3C46FD
:1091200001E0A24513D00B9B14F8011B03F1380298
:109130006A440133042B02F8101C0B93F1D10AA9E5
:1091400007A8F9F709FDA245CDE90B90EBD10C9BDF
:10915000002BC0F26481BDF8124017F8013B0822D1
:1091600084EA032423B2002BABBF640085EA4303E7
:10917000A4B29CB2013AF5D15745EED1D8F804A07B
:109180003246514607A8FEF7C5FB0028C0F24781CA
:109190000AEB0600824513D00AF1FF31013811F8BD
:1091A000013F082284EA032423B2002BABBF6400F2
:1091B00085EA4303A4B29CB2013AF5D18142EED1D3
:1091C000ADF81240DDE90740574B08F11408984507
:1091D0002246014687D3029F234602330026994246
:1091E000ADF81460C0F01C8105ADA8460DF1160461
:1091F000AA4601E0544513D00B9B1AF8011B03F15A
:1092000038026A440133042B02F8101C0B93F1D18D
:109210000AA907A8F9F7A0FC5445CDE90B60EBD1EA
:109220000C9B002BC0F2FC80BDF8123041F22100F3
:1092300018F8012B082183EA02231AB2002AABBFD7
:109240005B0080EA42029BB293B20139F5D1A0459E
:10925000EED1ADF81230079B089A0233934200F228
:10926000DF800E460DF1120401E0AC4213D00B9BDF
:1092700014F8011B03F138026A440133042B02F88D
:10928000101C0B93F1D10AA907A8F9F765FCAC42B1
:10929000CDE90B60EBD10C9C002CC0F2C1800B9887
:1092A000002800F0D880079B089A0344934200F2FC
:1092B000B7800AABC0F10402002118447BF09EFD88
:1092C0000AA907A8F9F748FC002804460C90C0F248
:1092D000A7809DF83430002B40F0BD80BBF1010B1E
:1092E00000F0BF80002C7FF4C3AE094B094A93F80D
:1092F000543102EB43035B7813B1204607F0E2F8E8
:10930000FFF72AFE002800F097800FB0BDE8F08F2D
:10931000C05D0020085308080000100800000E0877
:10932000003C024001000E08408009088C7A0908C0
:1093300000231F469A46CDF804B00AF1010A931D96
:109340005FFA8AFA8B428DF819A066D80DF1140CD9
:109350000DF11A0B6446CDF800C001E05C4514D055
:109360000B9B14F8010B03F138020DEB02010133E2
:10937000042B01F8100C0B93F0D10AA907A8F9F7F8
:10938000EBFB5C45CDE90B90EAD10C9BDDF800C00E
:10939000002B42DBBDF812401CF8013B082284EA96
:1093A000032423B2002BABBF640085EA4303A4B2BD
:1093B0009CB2013AF5D1E345EED1D8F8041001EBA7
:1093C000070B3246594607A8FEF7A4FA002824DB0B
:1093D0000BEB0600834513D00BF1FF31013811F878
:1093E000013F082284EA032423B2002BABBF6400B0
:1093F00085EA4303A4B29CB2013AF5D18142EED191
:10940000ADF81240DDE90740BAF1030F37442246B8
:10941000014692D1DDF804B0D6E6DDF804B0029F33
:10942000BBF1010B7FF424AE174B184A93F854316B
:1094300002EB43035B7843B9052008F049F9144B6C
:10944000536003F18833536020E6584607F03AF83A
:10945000052008F03DF90F4A136943F000431361FA
:109460003CE7094B094A93F8543102EB43035B781C
:1094700013B1584607F026F8002C3FF441AFDBE764
:10948000054B3946A9E600BFC05D00200853080817
:1094900023016745003C024000000E0870B5458876
:1094A0000B460446C5F30B052A46002118467BF0FF
:1094B000A5FC0A4A21699142034606D3084A914213
:1094C00006D3BDE87040184608470029F9D170BDA1
:1094D0002A46BDE870407BF04DBC00BF40800908C3
:1094E0007785090810B50446C06900B110BD09218F
:1094F0001420FFF703F8E06110BD00BF10B5174C52
:1095000004EB8000406830B300EB400004EB8003C4
:1095100093F929CCBCF1FF3F1ED093F8310CD0B1A8
:1095200004EB0C0293F8300C92F87CEC8C231421A1
:1095300003FB0CFC00220CEB000304EB430301399A
:10954000B3F8803C704412FA83F2F4D1044BA3FBCD
:109550000230C0F30F1010BD002010BDC05D002010
:10956000CDCCCCCC844610B5BCF80EE000230EF474
:109570007F4401200EF00F0EACF80E4019464A1041
:109580003CF81220002A18BF002011F0010F1ABF6A
:10959000D2B2534083EA1223082213F4004F18BFBB
:1095A00083F4C053013A4FEA4303F6D10131102945
:1095B000E5D14EEA0404ACF80E4038B9C3F30333E6
:1095C000B3EB0E0018BF4FF0FF3010BD4FF0FF306F
:1095D00010BD00BF70B5104B104CA3421AD2054607
:1095E00002E00C33A34215D293F805C08C45F8D1A4
:1095F00093F804C0AC4501D0002DF2D1D879904247
:10960000EFD1186890F804E0E645EAD106689E427A
:10961000E7D170BD002070BD7885090894870908DE
:109620000379022B00D0704710B490F910201D4828
:109630001D4C83B002EB82020831694400EB8202C8
:109640000094D2F8902911F8084C18498A4225D084
:10965000A1F578418A4223D001F580618A4219D16F
:10966000118821F04001090403EB8303090C1180E8
:1096700000EB83001388D0F89C1923F0380331F8ED
:1096800024101B041B0C0B43138013889BB243F064
:109690004003138003B05DF8044B70470023DFE7FD
:1096A0000123DDE7300C00200001020300300140FF
:1096B000034690F910002DE9F041244C00EB8000A6
:1096C00016469A6804EB80009207D0F8908909D575
:1096D000404677F0FDFC3146404677F0F9FC01202A
:1096E000BDE8F0815D69084615B12B68AA885A83E8
:1096F000174B184F1C68184B7A684FEAC40CA3FB31
:109700000C3C4FEA9C1C7B689B1A9C45FBD2014693
:10971000404677F0DDFC3146404677F0D9FC0E4BF1
:1097200078680C494FF4FA7204FB02F2A3FB023290
:1097300092094B681B1A9A42FBD2002DCFD02B689E
:10974000AA881A830120BDE8F08100BF300C0020F8
:109750005C3B0020001000E0D34D621010B503798F
:10976000012B84B08E460DD0022B02D0002004B015
:1097700010BD8368DB0758BF01F07F0104B0BDE86E
:10978000104095E7144682688DF80F4002F0010200
:1097900001920DF10F020092417C90F91000724687
:1097A000FAF758FE04B010BD2DE9F041076882B009
:1097B0008046B6227E213846FFF7D0FF642607F0A8
:1097C0002BFF04460D4607F027FF001B61EB050148
:1097D000B0F57A7F71F10001F5D3013EEFD102219E
:1097E0003846FFF71DFF7B6913B11A689B885383C6
:1097F00007F012FF04460D4607F00EFF001B61EB59
:109800000501B0F57A7F71F10001F5D37B6913B1E1
:109810001A689B8813830A2607F0FEFE04460D464D
:1098200007F0FAFE001B61EB0501B0F57A7F71F1DC
:109830000001F5D3013EEFD132467C213846FFF7D7
:109840008DFF07F0E9FE04460D4607F0E5FE001B1C
:1098500061EB0501B0F57A7F71F10001F5D30022CB
:1098600059213846FFF77AFF07F0D6FE04460D4629
:1098700007F0D2FE001B61EB0501B0F57A7F71F1B4
:109880000001F5D397F910308E4A03EB830302EB06
:109890008303BA68D3F890495E2192078DF80710C8
:1098A00040F1E48001230DF107020021204677F00A
:1098B000BFFB4FF4A473844A2046002177F0B8FB25
:1098C000BB689B0740F1E5800A2607F0A5FE044629
:1098D0000D4607F0A1FE001B61EB0501B0F57A7F94
:1098E00071F10001F5D3013EEFD101225921384633
:1098F000FFF734FF07F090FE04460D4607F08CFE9C
:10990000001B61EB0501B0F57A7F71F10001F5D321
:109910008C2240213846FFF721FF07F07DFE0446E8
:109920000D4607F079FE001B61EB0501B0F57A7F6B
:1099300071F10001F5D3032241213846FFF70EFFF4
:1099400007F06AFE04460D4607F066FE001B61EB59
:109950000501B0F57A7F71F10001F5D35B4CD8F8C1
:10996000382098F83500B4FBF2F2032391B2584A3C
:10997000FEF79CFE4388B4FBF3F4C8F8404002793C
:10998000422142F0C0023846FFF7E8FE07F044FEED
:1099900004460D4607F040FE001B61EB0501B0F5E3
:1099A0007A7F71F10001F5D3082243213846FFF791
:1099B000D5FE07F031FE04460D4607F02DFE001BD4
:1099C00061EB0501B0F57A7F71F10001F5D3042256
:1099D00058213846FFF7C2FE07F01EFE04460D462A
:1099E00007F01AFE001B61EB0501B0F57A7F71F1FB
:1099F0000001F5D30A2253213846FFF7AFFE07F0E6
:109A00000BFE04460D4607F007FE001B61EB050147
:109A1000B0F57A7F71F10001F5D300227C21384640
:109A2000FFF79CFE07F0F8FD04460D4607F0F4FD35
:109A3000001B61EB0501B0F57A7F71F10001F5D3F0
:109A400006227D213846FFF789FE07F0E5FD044632
:109A50000D4607F0E1FD001B61EB0501B0F57A7FD3
:109A600071F10001F5D302B0BDE8F0817B6913B15B
:109A70001A689B885383174B17491A68174B486815
:109A8000D200A3FB023292094B681B1A9A42FBD206
:109A900008E7104B10491A68104B48684FF4FA74E5
:109AA00004FB02F2A3FB023292094B681B1A9A4292
:109AB000FBD27B69002B3FF407AF1A689B881383A6
:109AC00002E700BF300C0020B853080840420F00E6
:109AD000005508085C3B0020001000E0D34D6210E8
:109AE0002DE9F041836B07685A4A5B4DB5FBF3F1F2
:109AF0000446062389B290F83500FEF7D7FD002111
:109B00004388B5FBF3F5804625643846FFF788FDAA
:109B100080226B213846FFF721FE642607F07CFD8A
:109B200004460D4607F078FD001B61EB0501B0F51A
:109B30007A7F71F10001F5D3013EEFD10322682154
:109B40003846FFF70BFE642607F066FD04460D4617
:109B500007F062FD001B61EB0501B0F57A7F71F142
:109B60000001F5D3013EEFD101226B213846FFF70A
:109B7000F5FD0F2607F050FD04460D4607F04CFD9D
:109B8000001B61EB0501B0F57A7F71F10001F5D39F
:109B9000013EEFD118221B213846FFF7DFFD0F26CB
:109BA00007F03AFD04460D4607F036FD001B61EB59
:109BB0000501B0F57A7F71F10001F5D3013EEFD1D7
:109BC00018221C213846FFF7C9FD0F2607F024FD97
:109BD00004460D4607F020FD001B61EB0501B0F5C2
:109BE0007A7F71F10001F5D3013EEFD198F804209E
:109BF0001A213846FFF7B2FD0F2607F00DFD044687
:109C00000D4607F009FD001B61EB0501B0F57A7FF9
:109C100071F10001F5D3013EEFD198F8052019212B
:109C20003846FFF79BFD642607F0F6FC04460D4618
:109C300007F0F2FC001B61EB0501B0F57A7F71F1D2
:109C40000001F5D3013EEFD138460321BDE8F041D4
:109C5000E6E400BF1455080840420F002DE9F0412A
:109C6000836B0768654A664DB5FBF3F1044606232E
:109C700089B290F83500FEF719FD00214388B5FB45
:109C8000F3F5804625643846FFF7CAFC80226B2135
:109C90003846FFF763FD642607F0BEFC04460D4618
:109CA00007F0BAFC001B61EB0501B0F57A7F71F19A
:109CB0000001F5D3013EEFD1072268213846FFF7B6
:109CC0004DFD642607F0A8FC04460D4607F0A4FCF1
:109CD000001B61EB0501B0F57A7F71F10001F5D34E
:109CE000013EEFD132466B213846FFF737FD64263F
:109CF00007F092FC04460D4607F08EFC001B61EB5A
:109D00000501B0F57A7F71F10001F5D3013EEFD185
:109D100001226B213846FFF721FD0F2607F07CFC5E
:109D200004460D4607F078FC001B61EB0501B0F519
:109D30007A7F71F10001F5D3013EEFD118221B218A
:109D40003846FFF70BFD0F2607F066FC04460D466C
:109D500007F062FC001B61EB0501B0F57A7F71F141
:109D60000001F5D3013EEFD118221C213846FFF740
:109D7000F5FC0F2607F050FC04460D4607F04CFC9E
:109D8000001B61EB0501B0F57A7F71F10001F5D39D
:109D9000013EEFD198F804201A213846FFF7DEFC87
:109DA0000F2607F039FC04460D4607F035FC001B72
:109DB00061EB0501B0F57A7F71F10001F5D3013E49
:109DC000EFD198F8052019213846FFF7C7FC642623
:109DD00007F022FC04460D4607F01EFC001B61EB59
:109DE0000501B0F57A7F71F10001F5D3013EEFD1A5
:109DF00038460321BDE8F04112E400BF14550808BD
:109E000040420F002AE700BFF8B57822074600213C
:109E10000068FFF7A3FC052607F0FEFB04460D468D
:109E200007F0FAFB001B61EB0501B0F57A7F71F1D9
:109E30000001F5D3013EEFD1386820220121FFF760
:109E40008DFC052607F0E8FB04460D4607F0E4FB11
:109E5000001B61EB0501B0F57A7F71F10001F5D3CC
:109E6000013EEFD1324638680221FFF777FC6426C5
:109E700007F0D2FB04460D4607F0CEFB001B61EB5A
:109E80000501B0F57A7F71F10001F5D3013EEFD104
:109E90000120F8BD70B52422044641210068FFF777
:109EA0005DFC90B9052607F0B7FB04460D4607F0A8
:109EB000B3FB001B61EB0501B0F57A7F71F1000186
:109EC000F5D3013EEFD1012070BD20682022302162
:109ED000FFF744FC0028E5D0206806223121FFF777
:109EE0003DFC0028DED0206800223421FFF736FC3C
:109EF000D8E700BFF8B5072207460A210068FFF738
:109F00002DFC052607F088FB04460D4607F084FB70
:109F1000001B61EB0501B0F57A7F71F10001F5D30B
:109F2000013EEFD1386824224121FFF717FC0526B6
:109F300007F072FB04460D4607F06EFB001B61EB59
:109F40000501B0F57A7F71F10001F5D3013EEFD143
:109F50003868C0224221FFF701FC052607F05CFBB0
:109F600004460D4607F058FB001B61EB0501B0F5F8
:109F70007A7F71F10001F5D3013EEFD10120F8BDE8
:109F800010B50446002221210068FFF7E7FB206896
:109F9000FC222021FFF7E2FB206840222421FFF76A
:109FA000DDFB20680C222321FFF7D8FB206800226C
:109FB0002221FFF7D3FB012010BD00BFF8B501221D
:109FC000074610210068FFF7C9FB00B9F8BD142649
:109FD00007F022FB04460D4607F01EFB001B61EB59
:109FE0000501B0F57A7F71F10001F5D3013EEFD1A3
:109FF0003868A022BDE8F8401121FFF7AFBB00BFD1
:10A00000F0B5046883B0074600212046FFF708FB3F
:10A010000C2225212046FFF7A1FB0A2226213868C1
:10A02000FFF79CFB002263213868FFF797FB386835
:10A0300081222721FFF792FB142607F0EDFA044650
:10A040000D4607F0E9FA001B61EB0501B0F57A7FD8
:10A0500071F10001F5D3013EEFD10C2225213868C2
:10A06000FFF77CFB0A2226213868FFF777FB0F22D7
:10A0700063213868FFF772FB386881222721FFF7D8
:10A080006DFB0A2607F0C8FA04460D4607F0C4FA2D
:10A09000001B61EB0501B0F57A7F71F10001F5D38A
:10A0A000013EEFD1032301AA102138466EF030FDA6
:10A0B0000A2607F0B1FA04460D4607F0ADFA001B78
:10A0C00061EB0501B0F57A7F71F10001F5D3013E36
:10A0D000EFD19DF804009DF805109DF806202C4B4B
:10A0E000803080318032A3F8C80FA3F8CA1FA3F8CC
:10A0F000CC2F25210C223868FFF730FB0A222621BD
:10A100003868FFF72BFB324663213868FFF726FBE0
:10A11000386881222721FFF721FB0A2607F07CFA05
:10A1200004460D4607F078FA001B61EB0501B0F517
:10A130007A7F71F10001F5D3013EEFD10DF10302F9
:10A140000123022138466EF0E3FC01230DF10302E6
:10A15000092138466EF0DCFC38680C222521FFF717
:10A16000FDFA38680A222621FFF7F8FA3868122229
:10A170006321FFF7F3FA812238682721FFF7EEFA0F
:10A1800038680321FFF74CFA012003B0F0BD00BF8F
:10A19000C05D00202DE9F041802207460B210068B8
:10A1A000FFF7DCFA1E26804607F036FA04460D4615
:10A1B00007F032FA001B61EB0501B0F57A7F71F10F
:10A1C0000001F5D3013EEFD1B8F1000F02D100201C
:10A1D000BDE8F081386806222921FFF7BFFA002880
:10A1E000F5D0386808220B21FFF7B8FA0028EED026
:10A1F0003868CF22BDE8F0410A21FFF7AFBA00BFAF
:10A2000010B5044694220B210068FFF7A7FA2068D6
:10A2100071220121FFF7A2FA206800220421FFF732
:10A220009DFA2068C8220521FFF798FA20680022CD
:10A230000621FFF793FA2068C8220721FFF78EFA5C
:10A24000206800220821FFF789FA2068C822092126
:10A25000FFF784FA012010BD00680379012B0BD0B1
:10A26000022B01D0002070478368DB074FF0F0021B
:10A2700019D5FF21FFF71CBA00B5826890F910C00C
:10A28000417C85B002F0010201920DF10F020092B3
:10A290006046FF224FF0F00C8DF80FC0FAF7DAF8A5
:10A2A00005B05DF804FB7F21FFF702BA006803796F
:10A2B000CA4341EA0211012BCAB209D0022B01D0D4
:10A2C000002070478368DB0717D5D221FFF7F0B96C
:10A2D00000B585B090F910C08DF80F208268417CE0
:10A2E00002F001020DF10F00CDE90002D22260461A
:10A2F000FAF7B0F805B05DF804FB5221FFF7D8B9C2
:10A3000000680379012B0BD0022B01D0002070478D
:10A310008368DB074FF0B40219D5FF21FFF7C8B9F6
:10A3200000B5826890F910C0417C85B002F001024E
:10A3300001920DF10F0200926046FF224FF0B40C23
:10A340008DF80FC0FAF786F805B05DF804FB7F21A1
:10A35000FFF7AEB900680379012B0AD0022B01D0B8
:10A36000002070478368DB070A4617D5A521FFF751
:10A370009FB900B5826890F910C085B002F0010263
:10A380008DF80F10417C0DF10F00CDE90002A522E0
:10A390006046FAF75FF805B05DF804FB2521FFF78A
:10A3A00087B900BF00680379012B0BD0022B01D0C5
:10A3B000002070478368DB074FF0960219D5FF2114
:10A3C000FFF776B900B5826890F910C0417C85B07E
:10A3D00002F0010201920DF10F0200926046FF228D
:10A3E0004FF0960C8DF80FC0FAF734F805B05DF811
:10A3F00004FB7F21FFF75CB900680379012B0AD0C9
:10A40000022B01D0002070478368DB070A4617D56E
:10A410008721FFF74DB900B5826890F910C085B06B
:10A4200002F001028DF80F10417C0DF10F00CDE913
:10A43000000287226046FAF70DF805B05DF804FBCC
:10A440000721FFF735B900BF00680379C901012B67
:10A45000CAB206D0022B01D0002070477821FFF746
:10A4600027B900B585B090F910C08DF80F2082682B
:10A47000417C02F001020DF10F00CDE900027822CB
:10A480006046F9F7E7FF05B05DF804FB0068037963
:10A49000012B0BD0022B01D0002070478368DB0713
:10A4A0004FF0550219D5A521FFF702B900B5826812
:10A4B00090F910C0417C85B002F0010201920DF1CB
:10A4C0000F0200926046A5224FF0550C8DF80FC088
:10A4D000F9F7C0FF05B05DF804FB2521FFF7E8B8E8
:10A4E00000680379012B0BD0022B01D000207047AC
:10A4F0008368DB074FF02E0219D5F421FFF7D8B897
:10A5000000B5826890F910C0417C85B002F001026C
:10A5100001920DF10F0200926046F4224FF02E0CD2
:10A520008DF80FC0F9F796FF05B05DF804FB7421B4
:10A53000FFF7BEB8154B00689A8E0379920134324A
:10A54000012BD2B209D0022B01D0002070478368C2
:10A55000DB0717D5F421FFF7ABB800B585B090F94C
:10A5600010C08DF80F208268417C02F001020DF1CD
:10A570000F00CDE90002F4226046F9F76BFF05B049
:10A580005DF804FB7421FFF793B800BFC05D0020A5
:10A5900000B500680379012B85B012D0022B03D0DF
:10A5A000012005B05DF804FB8368DB074FF0310242
:10A5B0004CBFF4217421FFF77BF8012005B05DF852
:10A5C00004FB826890F910C0417C02F00102019204
:10A5D0000DF10F0200926046F4224FF0310C8DF81D
:10A5E0000FC0F9F737FF012005B05DF804FB00BF8D
:10A5F00000680379012B07D0022B01D0002070479F
:10A6000013221B21FFF754B800B5826890F910C0DF
:10A61000417C85B002F0010201920DF10F0200921F
:10A6200060461B224FF0130C8DF80FC0F9F712FF94
:10A6300005B05DF804FB00BF00680379012B07D06B
:10A64000022B01D00020704701225821FFF730B8BB
:10A6500000B5826890F910C0417C85B002F001021B
:10A6600001920DF10F020092604658228DF80F30D2
:10A67000F9F7F0FE05B05DF804FB00BF0068037950
:10A68000012B07D0022B01D0002070470122482166
:10A69000FFF70EB800B5826890F910C0417C85B014
:10A6A00002F0010201920DF10F0200926046482271
:10A6B0008DF80F30F9F7CEFE05B05DF804FB00BF52
:10A6C00000680379012B07D0022B01D000207047CE
:10A6D0001A460821FEF7ECBF00B5826890F910C059
:10A6E000417C85B002F0010201920DF10F0200924F
:10A6F000604608224FF0020C8DF80FC0F9F7AAFE51
:10A7000005B05DF804FB00BF00680379012B07D09A
:10A71000022B01D00020704701220821FEF7C8BF9C
:10A7200000B5826890F910C0417C85B002F001024A
:10A7300001920DF10F020092604608228DF80F3051
:10A74000F9F788FE05B05DF804FB00BF10B50446BC
:10A7500000680379012B84B012D0022B02D00020B4
:10A7600004B010BD01220B21FEF7A2FF0028F6D095
:10A7700020681D22092104B0BDE81040FEF7EEBF9D
:10A78000826890F910C0417C8DF80F3002F0010210
:10A7900001920DF10F02009260460B22F9F75AFE6A
:10A7A000E4E700BF2DE9F04105461F4695F910305A
:10A7B000244803EB830300EB8300AB68D0F8908957
:10A7C00016469A070ED5404676F082FC3B46324646
:10A7D0000021404676F02CFCAB689B0718D5012081
:10A7E000BDE8F0816B6913B11A689B885383164BDF
:10A7F000164A1B684FEAC30E154BA2FB0E2E5A6871
:10A800004FEA9E1E5C68A4EB020CE645FAD2DAE73A
:10A810000D4B0F491A680D4B4FF4FA7000FB02F212
:10A82000A3FB0232486892094B681B1A9A42FBD27A
:10A830006B69002BD3D01A689B8813830120BDE875
:10A84000F08100BF300C00205C3B0020D34D621033
:10A85000001000E030B50579012D83B08E460DD093
:10A86000022D02D0002003B030BD8468E40758BF39
:10A8700001F07F0103B0BDE8304093E714468268E1
:10A88000009402F00102417C90F91000019272469E
:10A89000F9F7E0FD03B030BD2DE9F04105461F4654
:10A8A00095F91030244803EB830300EB8300AB6879
:10A8B000D0F8908916469A070ED5404676F008FCE7
:10A8C0003B4600223146404676F0B2FBAB689B0720
:10A8D00018D50120BDE8F0816B6913B11A689B8817
:10A8E0005383164B164A1B684FEAC30E154BA2FB47
:10A8F0000E2E5A684FEA9E1E5C68A4EB020CE645D9
:10A90000FAD2DAE70D4B0F491A680D4B4FF4FA7083
:10A9100000FB02F2A3FB0232486892094B681B1A43
:10A920009A42FBD26B69002BD3D01A689B881383A1
:10A930000120BDE8F08100BF300C00205C3B00200E
:10A94000D34D6210001000E030B50579012D83B0C1
:10A950008E460DD0022D02D0002003B030BD846899
:10A96000E40758BF41F0800103B0BDE8304093E7F1
:10A9700014468268009402F00102417C90F91000B4
:10A9800001927246F9F79AFD03B030BD2DE9F0430C
:10A99000836B0768804A814CB4FBF3F185B0804635
:10A9A000062389B290F83500FDF780FE0021438828
:10A9B000B4FBF3F48146C8F840403846FEF730FE59
:10A9C00080226B213846FEF7C9FE962606F024FE4B
:10A9D00004460D4606F020FE001B61EB0501B0F5B4
:10A9E0007A7F71F10001F5D3013EEFD10322682196
:10A9F0003846FEF7B3FE962606F00EFE04460D46D8
:10AA000006F00AFE001B61EB0501B0F57A7F71F1DB
:10AA10000001F5D3013EEFD103226B213846FEF74A
:10AA20009DFE06F0F9FD04460D4606F0F5FD001BFF
:10AA300061EB05010F2871F10001F6D310226A21A4
:10AA40003846FEF78BFE06F0E7FD04460D4606F09D
:10AA5000E3FD001B61EB05010F2871F10001F6D346
:10AA600000226C213846FEF779FE06F0D5FD04463B
:10AA70000D4606F0D1FD001B61EB05010F2871F1B9
:10AA80000001F6D399F8052019213846FEF766FE35
:10AA900006F0C2FD04460D4606F0BEFD001B61EB4C
:10AAA00005010F2871F10001F6D318221B21384649
:10AAB000FEF754FE06F0B0FD04460D4606F0ACFD70
:10AAC000001B61EB05010F2871F10001F6D318227C
:10AAD0001C213846FEF742FE06F09EFD04460D4658
:10AAE00006F09AFD001B61EB05010F2871F10001D2
:10AAF000F6D399F804201A213846FEF72FFE06F007
:10AB00008BFD05460C4606F087FD8C4208BF85424A
:10AB1000F9D003213846FEF783FDD8F8000006235C
:10AB2000432102AAFFF710FF28B3BDF80810BDF8B3
:10AB30000A30BDF80C20C9BA07EE901ADBBAD2BAB7
:10AB4000F8EEE76A07EE102A07EE903AB8EEC77AF9
:10AB5000F8EEE77AC8ED076AC8ED087A88ED097A59
:10AB6000FDEEE77ACDED017A9DF90430013305D091
:10AB700005B0BDE8F083D8ED087AF1E7D8ED077AA3
:10AB8000FDEEE77ACDED017A9DF904300133EFD186
:10AB9000062006F09DFD00BF1455080840420F0036
:10ABA00008B500680379022B0BBF114A114A07232D
:10ABB00006230421FFF7C8FE0F4B93F8D31F93F829
:10ABC000D2CF93F8D62F090441EA0C2193F8D1CFC4
:10ABD00041EA0C0193F8D5CFC3F88810120442EA79
:10ABE0000C2293F8D4CF42EA0C0201201A6608BD69
:10ABF000906D0020916D0020C05D002010B50446CE
:10AC00000068037982B0022B0CBF43210321062385
:10AC10006A46FFF799FE68B1BDF80010BDF8022042
:10AC2000BDF8043049BA52BA5BBAE186628723871D
:10AC300002B010BDC4F83600608702B010BD00BF7E
:10AC40002DE9F047164F97F8D93F824689466BB9F0
:10AC5000DAF8000097F8DA3F00244A46492187F8DD
:10AC6000D94FFFF771FE0120BDE8F08706F0D4FC54
:10AC7000D7F8E03FC51AC5F5FA55002DE8DD06F016
:10AC8000CBFC4FEAE57804460E4606F0C5FC001BF7
:10AC900061EB0601A84271EB0801F6D3D8E700BFCB
:10ACA000C05D00202DE9F041624C0546D4F8E80F64
:10ACB000C5F8360094F8D83FB4F8EC2F6A87012B1A
:10ACC00082B076D0022B0FD0002B69D10122022155
:10ACD00028466FF013FD012394F8EE6F84F8D83FF7
:10ACE000304602B0BDE8F08194F8D93F05F136084E
:10ACF00004F6E877002B6ED169462846FFF7A0FFDF
:10AD00009DF80630064600284AD01B0748D4B4F800
:10AD1000C82FBDF8003013FB02F3474A93427DDB96
:10AD2000B3F5000F6FDA002BB8BFFF331B125B4285
:10AD30001BB2B4F8CA2FEB86BDF8023013FB02F346
:10AD40003D4A93426EDBB3F5000F6FDA002BB8BFBC
:10AD5000FF3343F30F23B4F8CC2F2B87BDF8043017
:10AD600013FB02F3344A93425ADBB3F5000F5BDA6C
:10AD7000002BB8BFFF331B125B421BB2D5F8360065
:10AD8000C4F8E80F6B87B8F80430BB8000220123B9
:10AD9000304684F8D82F84F8EE3F02B0BDE8F08149
:10ADA0000026304684F8D86F84F8EE6F02B0BDE814
:10ADB000F08194F8D93F94F8EE6FD3B969462846EC
:10ADC000FFF73EFF9DF8003008B19A071DD1002320
:10ADD00084F8D83F84E706F01FFCD4F8E03FC01A9F
:10ADE000B0F5FA5F88DA94F8EE6F304602B0BDE84D
:10ADF000F08106F011FCD4F8E03FC01AB0F5FA5F1C
:10AE0000FFF66EAFDAE70D4B93E7072203212846E2
:10AE10006FF074FC022384F8D83F61E7084B88E7A1
:10AE2000074BABE7064B96E7044BA7E747F6FF73E4
:10AE300091E700BFC05D002001FF7FFF0180FFFFA1
:10AE40000080FFFF70B50668F46982B00546002CEB
:10AE50003FD03379012B04F104022DD0022B26D1EF
:10AE6000B36813F0010F4FF00C03304614BF1946BE
:10AE70008C21FFF711FDA070D8B1B4F9043007EEB2
:10AE8000903AF8EEE77AC5ED077AB4F9063007EEA6
:10AE9000903AF8EEE77AC5ED087AB4F9083007EE93
:10AEA000903AF8EEE77AC5ED097A02B070BD00235A
:10AEB000A370002002B070BDB368717C96F91000D9
:10AEC000009203F0010301930C231A46F9F7F6FAF6
:10AED000D1E709211420FDF711FBF06104462E682B
:10AEE000B7E700BF70B50668F46982B00546002C6C
:10AEF0003FD03379012B04F103022DD0022B26D150
:10AF0000B36813F0010F30464FF00D0314BF0C214E
:10AF10008C21FFF7C1FCA070D8B1B4F90A3007EE5C
:10AF2000903AF8EEE77AC5ED077AB4F90C3007EEFF
:10AF3000903AF8EEE77AC5ED087AB4F90E3007EEEC
:10AF4000903AF8EEE77AC5ED097A02B070BD0023B9
:10AF5000A370002002B070BDB368717C96F9100038
:10AF6000009203F0010301930C220D23F9F7A6FAD6
:10AF7000D1E709211420FDF7C1FAF06104462E68DB
:10AF8000B7E700BF10B500680379012B84B00C4609
:10AF90001AD0022B02D0002004B010BD836813F039
:10AFA000010F03AA4FF0030314BF2221A221FFF7D0
:10AFB00073FC0028EFD0BDF90D3003EB83031B12A7
:10AFC000E633238004B010BD8368417C90F9100003
:10AFD00003F00103019303AB009322220323F9F74B
:10AFE0006DFAE6E710B5044600680379012B84B0DA
:10AFF0002DD0022B01D0002027E0836813F0010F31
:10B0000002AA4FF0060314BF1F219F21FFF744FC43
:10B010000028F0D0BDF80810BDF80A20BDF80C30AB
:10B02000C9BA07EE901AD2BAF8EEE76A07EE902A8C
:10B03000DBBAB8EEE77A07EE903AF8EEE77AC4EDBD
:10B04000046A84ED057AC4ED067A04B010BD836805
:10B05000417C90F9100003F00103019302AB0093CF
:10B060001F220623F9F72AFAD2E700BF10B50446DB
:10B0700000680379012B84B02DD0022B01D0002071
:10B0800027E0836813F0010F02AA4FF0060314BFF4
:10B090002521A521FFF700FC0028F0D0BDF80810FD
:10B0A000BDF80A20BDF80C30C9BA07EE901AD2BA22
:10B0B000F8EEE76A07EE902ADBBAB8EEE77A07EE19
:10B0C000903AF8EEE77AC4ED076A84ED087AC4EDA9
:10B0D000097A04B010BD8368417C90F9100003F038
:10B0E0000103019302AB009325220623F9F7E6F949
:10B0F000D2E700BF10B500680379012B84B00C467D
:10B1000025D0022B01D000201FE0826812F0010F31
:10B1100018BF1D2103AA08BF9D21FFF7BDFB002812
:10B12000F1D0BDF80C309FED116ADFED116ADBBA8A
:10B1300007EE903AB8EEE77AC7EE067A77EEA67A8F
:10B14000FDEEE77A17EE903A238004B010BD8368D5
:10B15000417C90F9100003F00103019303AB0093CD
:10B160001D220223F9F7AAF9D9E700BFCFF753410F
:10B1700000007A4370B50668F46982B00546002C79
:10B180003FD03379012B04F104022DD0022B26D1BC
:10B19000B36813F0010F30464FF00E0314BF3B218C
:10B1A000BB21FFF779FBA070D8B1A389DBBA07EE0A
:10B1B000903AF8EEE77AC5ED077AE389DBBA07EE55
:10B1C000903AF8EEE77AC5ED087A238ADBBA07EE03
:10B1D000903AF8EEE77AC5ED097A02B070BD002327
:10B1E000A370002002B070BDB368717C96F91000A6
:10B1F000009203F0010301933B220E23F9F75EF95D
:10B20000D1E709211420FDF779F90446F061B8E788
:10B2100000B500680379012B85B011D0022B01D055
:10B2200000200AE003AAF621FFF736FB0028F7D03A
:10B23000BDF80C30094A5BBA938205B05DF804FB97
:10B240008368417C90F9100003AA03F00103CDE963
:10B2500000230223F622F9F731F9E7E7C05D002069
:10B2600000B500680379012B85B01ED0022B01D0F8
:10B27000002017E0032303AAF621FFF70DFB0028A7
:10B28000F6D09DF80D309DF80CC00F499DF80E20AA
:10B290001B0243EA0C431343B1F93420C2F1080204
:10B2A000D3408B6305B05DF804FB8368417C90F963
:10B2B000100003AA03F00103CDE900230323F622C3
:10B2C000F9F7FCF8DBE700BFC05D002000B50068BF
:10B2D0000379012B85B033D0022B0AD01F49D1F856
:10B2E000F03FD1F8F42FCA630020CB6505B05DF8BC
:10B2F00004FB062302AAF721FFF7CEFA0028EDD0BF
:10B300009DF809309DF808C09DF80C209DF80A10A2
:10B310009DF80BE01B0143EA0C3312019DF80DC0B0
:10B3200043EA111342EA0E320C4942EA1C12C1F8F8
:10B33000F03FC1F8F42FCA63CB6505B05DF804FB9C
:10B340008368417C90F9100002AA03F00103CDE963
:10B3500000230623F722F9F7B1F8CFE7C05D0020FC
:10B3600000B500680379012B85B01ED0022B10D0E8
:10B370009DF80D309DF80C009DF80E10124A1B022E
:10B3800043EA00430B430120C2F8B03005B05DF83A
:10B3900004FB836813F0010F03AA4FF0030314BFEB
:10B3A00000218021FFF778FAE2E78368417C90F979
:10B3B000100003AA03F00103CDE9002303230022B8
:10B3C000F9F77CF8D4E700BFC05D002000B5006845
:10B3D0000379012B85B01ED0022B10D09DF80D30C3
:10B3E0009DF80C009DF80E10124A1B0243EA004320
:10B3F0000B430120C2F8C43005B05DF804FB83683C
:10B4000013F0010F03AA4FF0030314BF00218021A2
:10B41000FFF742FAE2E78368417C90F9100003AA43
:10B4200003F00103CDE9002303230022F9F746F8D6
:10B43000D4E700BFC05D002010B500680379012B80
:10B4400084B029D0022B01D0002023E0836813F0C0
:10B45000010F4FF0030303AA14BF19468321FFF71E
:10B460001BFA0028F0D09DF80C309DF90C109DF8C7
:10B470000D209DF80EC01B04002943EA0223A8BF3B
:10B4800000210C4AB8BF4FF07F4143EA0C030B4345
:10B49000C2F8F83004B010BD8268417C90F9100009
:10B4A00002F0010203AC0323CDE900421A46F9F78A
:10B4B00005F8D6E7C05D002000B500680379012BD0
:10B4C00085B02AD0022B01D0002023E0836813F03E
:10B4D000010F03AA4FF0030314BF00218021FFF7DF
:10B4E000DBF90028F0D09DF80C309DF90C109DF888
:10B4F0000D209DF80EC01B04002943EA0223A8BFBB
:10B5000000210D4AB8BF4FF07F4143EA0C030B43C3
:10B51000C2F8F43005B05DF804FB8368417C90F913
:10B52000100003AA03F00103CDE900230323002246
:10B53000F8F7C4FFD5E700BFC05D002010B5044692
:10B5400000680379012B84B043D0022B07D000227E
:10B5500013461046C4F83620638704B010BD8368D4
:10B5600013F0010F02AA4FF0060314BF112191211D
:10B57000FFF792F90028EAD0BDF90820BDF90A309A
:10B5800006EE902A5B42BDF90C2007EE103AF8EE69
:10B59000E66AB7EE086A07EE902A66EE866AB8EEAB
:10B5A000C77AFDEEE66A27EE067AF8EEE77A16EE3F
:10B5B000903A67EE867ABDEEC77AFDEEE77AE386CB
:10B5C00017EE103A238717EE903A1BB2638704B048
:10B5D00010BD8368417C90F9100003F001030193D2
:10B5E00002AB009311220623F8F768FFC2E700BF01
:10B5F00010B5044600230068C4F836306387037929
:10B60000012B84B022D0022B01D000201CE08368E3
:10B6100013F0010F02AA4FF0060314BF0321832188
:10B62000FFF73AF90028F0D0BDF90A30BDF808104C
:10B63000BDF80C205B4201EB410103EB430302EB3D
:10B640004202E1862387628704B010BD8368417C93
:10B6500090F9100003F00103019302AB0093032261
:10B660000623F8F72BFFDDE710B504464FF0000C7A
:10B670000068C4F836C0A4F83AC00379012B84B03E
:10B6800018D0022B01D0002012E0836813F0010FC4
:10B6900002AA4FF0060314BF61468021FFF7FCF8B1
:10B6A0000028F0D0029ABDF80C30C4F83620638729
:10B6B00004B010BD836890F910E0417C03F00103F1
:10B6C000019302AB0093624606237046F8F7F6FE3C
:10B6D000E6E700BF10B584B000230446006802937B
:10B6E000CDF80B300279012A1ED0022A19D18368C5
:10B6F00013F0010F02AA4FF0070314BF4E21CE2111
:10B70000FFF7CAF8BDF80910BDF80B20BDF80D30E1
:10B71000C9BAD2BADBBA0120E1862287638704B0B6
:10B7200010BD1A461946F6E7836890F910C0417CAF
:10B7300002AA03F00103009201934E220723604600
:10B74000F8F7BCFEDEE700BF70B50446234894F965
:10B75000103003EB830300EB8300A368D0F89069FB
:10B7600015469A070DD5304675F0B2FC012300222C
:10B770002946304675F05CFCA3689B0716D501206E
:10B7800070BD636913B11A689B885383144B154AC3
:10B790001B6850684FEAC30C134BA3FB0C3C4FEAE9
:10B7A0009C1C53681B1A9C45FBD2DCE70C4B0D49D3
:10B7B0001A680D4B4FF4FA7000FB02F2A3FB023241
:10B7C000486892094B681B1A9A42FBD26369002BA6
:10B7D000D5D01A689B881383012070BD300C0020DF
:10B7E0005C3B0020001000E0D34D621010B50379DF
:10B7F000012B82B08E460DD0022B02D0002002B069
:10B8000010BD8368DB0758BF41F0800102B0BDE87E
:10B81000104099E714468268009402F00102417CCE
:10B8200090F9100001927246F8F748FE02B010BD80
:10B8300070B505682B79012B84B004460E4616D0EE
:10B84000022B02D0002004B070BDAB68E122DB0700
:10B850004CBF114661212846FDF72AFF0028F1D090
:10B8600020683246FF2104B0BDE87040BEE7AA68F8
:10B87000697C95F9100002F001020DF10F050192AB
:10B880000095E1228DF80F20F8F7E4FDE6E700BF10
:10B8900070B505682B79012B84B004460E4617D08D
:10B8A000022B02D0002004B070BDAB68DB074FF064
:10B8B000C3024CBFE12161212846FDF7F9FE0028B3
:10B8C000F0D020683246FF2104B0BDE870408DE71B
:10B8D000AA6895F91000697C02F0010201920DF14D
:10B8E0000F020092C3228DF80F20E122F8F7B2FD7B
:10B8F000E5E700BF70B505682B79012B84B00446DD
:10B900000E461CD0022B02D0002004B070BDAB68E4
:10B91000DB074FF0F0024CBFE12161212846FDF723
:10B92000C7FE0028F0D02246FF2152F8040BFFF793
:10B930005DFF0028E8D02379337004B070BDAA6899
:10B9400095F91000697C02F0010201920DF10F02DD
:10B950000092F0228DF80F20E122F8F77BFDE0E75E
:10B96000F0B5046883B0002107462046FDF758FE75
:10B9700015227E212046FDF7F1FE642605F04CFEDF
:10B9800004460D4605F048FE001B61EB0501B0F5CD
:10B990007A7F71F10001F5D3013EEFD138681122B1
:10B9A0007E21FDF7DBFE052605F036FE04460D463A
:10B9B00005F032FE001B61EB0501B0F57A7F71F1F5
:10B9C0000001F5D3013EEFD138680DF107020321E4
:10B9D000FFF70CFF9DF8073003F03C03142B40F0F9
:10B9E0009B800C2240213868FDF7B8FE05F014FE5C
:10B9F00004460D4605F010FE001B61EB0501B0F595
:10BA00007A7F71F10001F5D3BB6B454C454AB4FB1D
:10BA1000F3F197F83500092389B2FCF747FE034696
:10BA200042215A88B4FBF2F43C641A793868FDF775
:10BA300095FE05F0F1FD04460D4605F0EDFD001BF9
:10BA400061EB0501B0F57A7F71F10001F5D30822B1
:10BA500041213868FDF782FE05F0DEFD04460D4603
:10BA600005F0DAFD001B61EB0501B0F57A7F71F19D
:10BA70000001F5D3002243213868FDF76FFE05F081
:10BA8000CBFD04460D4605F0C7FD001B61EB05012B
:10BA9000B0F57A7F71F10001F5D310225121386899
:10BAA000FDF75CFE05F0B8FD04460D4605F0B4FD5B
:10BAB000001B61EB0501B0F57A7F71F10001F5D350
:10BAC0000A2253213868FDF749FE05F0A5FD04461A
:10BAD0000D4605F0A1FD001B61EB0501B0F57A7F75
:10BAE00071F10001F5D3802256213868FDF736FE4A
:10BAF00005F092FD04460D4605F08EFD001B61EB3E
:10BB00000501B0F57A7F71F10001F5D338680321A2
:10BB1000FDF786FD03B0F0BD062005F0D9FD00BF9E
:10BB200040420F00385508082DE9F04F836B076835
:10BB3000A74AA84CB4FBF3F185B08046052389B22F
:10BB400090F83500FCF7B2FD00214388B4FBF3F414
:10BB50008146C8F840403846FDF762FD0022762154
:10BB60003846FDF7FBFD0F224E213846FDF7F6FD66
:10BB70000F2605F051FD04460D4605F04DFD001B56
:10BB800061EB0501B0F57A7F71F10001F5D3013E5B
:10BB9000EFD1DFF844A299F805209AF8F8BFABF18D
:10BBA0000103B3FA83F35B0902F00F0242EA431286
:10BBB0004F215B0138460193FDF7D0FD0F2605F0BC
:10BBC0002BFD04460D4605F027FD001B61EB05012A
:10BBD000B0F57A7F71F10001F5D3013EEFD199F80C
:10BBE0000520019B02F00F0213431A4650213846EC
:10BBF000FDF7B4FD0F2605F00FFD04460D4605F0D8
:10BC00000BFD001B61EB0501B0F57A7F71F10001BE
:10BC1000F5D3013EEFD1FF2252213846FDF79EFDBC
:10BC20000F2605F0F9FC04460D4605F0F5FC001B57
:10BC300061EB0501B0F57A7F71F10001F5D3013EAA
:10BC4000EFD198F8351007293FD05846FCF784FD0E
:10BC50000446012276213846FDF780FDA2780C21AA
:10BC60003846FDF77BFD22790D213846FDF776FD3C
:10BC7000A279A388120142EA1322D2B20E213846D9
:10BC8000FDF76CFD4FF480719AF8F80FFCF764FD36
:10BC90000446022276213846FDF760FDA278520064
:10BCA000032102F0FE023846FDF758FD22790421F7
:10BCB0003846FDF753FDA279A388120142EA132208
:10BCC0000521D2B23846FDF749FD002276213846DB
:10BCD000FDF744FD032214213846FDF73FFD0F26F2
:10BCE00005F09AFC04460D4605F096FC001B61EB3E
:10BCF0000501B0F57A7F71F10001F5D3013EEFD176
:10BD0000324663213846FDF729FD642605F084FCA0
:10BD100004460D4605F080FC001B61EB0501B0F503
:10BD20007A7F71F10001F5D3013EEFD10822652140
:10BD30003846FDF713FD64210DF10F023846FFF779
:10BD400055FD9DF80F2022F0100242F060026421A0
:10BD500038468DF80F20FDF701FD0F2605F05CFC3D
:10BD600004460D4605F058FC001B61EB0501B0F5DB
:10BD70007A7F71F10001F5D3013EEFD10DF10E0292
:10BD80004D213846FFF732FD9DF80E2002F03F02AC
:10BD900042F040024D2138468DF80E20FDF7DEFCC2
:10BDA0000F2605F039FC04460D4605F035FC001B56
:10BDB00061EB0501B0F57A7F71F10001F5D3013E29
:10BDC000EFD103213846FDF72BFC05B0BDE8F08F1D
:10BDD0007055080840420F00C05D0020F0B583B0E8
:10BDE00015460DF107021C4606460F46FFF7FEFCFE
:10BDF0009DF8072005EA0203A34201D103B0F0BD7C
:10BE000022EA050222433946304603B0BDE8F0403D
:10BE1000FDF7A4BC10B582B004466A46006808214C
:10BE2000FFF7E4FC9DF80030DB0602D4002002B0EE
:10BE300010BD206806236A460021FEF785FD002814
:10BE4000F4D09DF801309DF800109DF802209FED80
:10BE50004A6A1B0203EB01439DF804101C029DF883
:10BE600003401A444FEA01219DF8053001EB0441DB
:10BE700048BF02F17F420B4407EE902A090248BFF7
:10BE800003F17F43B8EEE77A07EE903AF8EEE77AEF
:10BE9000C7EE066A394BB3F99820B3F99E1093F8B0
:10BEA000FC4F112CC7EE863A07EE102A93ED256A57
:10BEB000B3F99A20D3ED247AF8EEC65A06EE102A8A
:10BEC000B3F99C2005EE102AB3F9A02004EE901AD5
:10BED00004EE102AB8EEC77AF8EEE77AB8EEC66A32
:10BEE000B8EEC55AF8EEE44AB3F9A210B3F9A420AB
:10BEF000B8EEC44A27EE237A26EEA32A23D0A6EE74
:10BF0000845AA6EEA46AE5EE265AE5EEA67A77EE06
:10BF1000877AE6EE027AB3F98E2007EE102AB3F99B
:10BF20008C20C3ED2A7A06EE902AB8EEC77AF8EE96
:10BF3000E66A27EE237AB6EE006AA6EE867A83EDED
:10BF40002B7A02B010BD03EE102AF8EEC32A03EEDE
:10BF5000101AA6EEA24AB8EEC33AA4EE265AE6EEAE
:10BF6000834AE5EE265AA4EEA66AE5EEA67A77EEB7
:10BF7000877AE6EE027ACEE700007848C05D0020BE
:10BF8000F0B5002283B007460A210068FDF7E6FB02
:10BF9000142605F041FB04460D4605F03DFB001B51
:10BFA00061EB0501B0F57A7F71F10001F5D3013E37
:10BFB000EFD138680F220A21FDF7D0FB0A2605F0E1
:10BFC0002BFB04460D4605F027FB001B61EB05012A
:10BFD000B0F57A7F71F10001F5D3013EEFD13868F9
:10BFE000032301AA1021FEF7AFFC0A2605F014FB7B
:10BFF00004460D4605F010FB001B61EB0501B0F592
:10C000007A7F71F10001F5D3013EEFD19DF8042054
:10C010009DF805009DF80610194B80328030803164
:10C0200023F8F82C23F8F60C324623F8F41C386871
:10C030000A21FDF793FB0A2605F0EEFA04460D46A9
:10C0400005F0EAFA001B61EB0501B0F57A7F71F1AA
:10C050000001F5D3013EEFD10DF103023868022152
:10C06000FFF7C4FB0DF1030238680921FFF7BEFB9F
:10C07000386811220A21FDF771FB012003B0F0BDE1
:10C08000B86E0020F0B5002283B007460A21006890
:10C09000FDF764FB142605F0BFFA04460D4605F0D3
:10C0A000BBFA001B61EB0501B0F57A7F71F100016D
:10C0B000F5D3013EEFD138680F220A21FDF74EFB80
:10C0C0000A2605F0A9FA04460D4605F0A5FA001B5C
:10C0D00061EB0501B0F57A7F71F10001F5D3013E06
:10C0E000EFD13868032301AA1021FEF72DFC0A26A0
:10C0F00005F092FA04460D4605F08EFA001B61EB3E
:10C100000501B0F57A7F71F10001F5D3013EEFD161
:10C11000324638680A21FDF721FB0A2605F07CFA31
:10C1200004460D4605F078FA001B61EB0501B0F5F9
:10C130007A7F71F10001F5D3013EEFD10DF10302D9
:10C1400038680221FFF752FB0DF10302386809211C
:10C15000FFF74CFB386801220A21FDF7FFFA0120A6
:10C1600003B0F0BD30B5002385B00446C0F83630CA
:10C1700043870DF1070200680221FFF737FB18B172
:10C180009DF80730DB0703D40025284605B030BDF5
:10C19000062302AA03212068FEF7D6FB20680DF1D2
:10C1A00007020921FFF722FB05460028ECD09DF885
:10C1B000073013F00C0FE7D1BDF80820BDF80C30A4
:10C1C000BDF80A102068C2EB8232C3EB83339B00B8
:10C1D00092008900E2862187638701220A21FDF708
:10C1E000BDFA284605B030BDF0B583B00023074640
:10C1F0008DF80230142605F00FFA04460D4605F0BE
:10C200000BFA001B61EB0501B0F57A7F71F10001BB
:10C21000F5D3013EEFD131460DF102023868FFF748
:10C22000E5FA0DF1020280213868FFF7DFFA4FF4DA
:10C23000F842ADF8042038688DF80660032301AA9F
:10C240006021FEF707FB142605F0E6F904460D46CB
:10C2500005F0E2F9001B61EB0501B0F57A7F71F1A1
:10C260000001F5D3013EEFD131460DF103023868EC
:10C270008DF80360FFF7BAFA4CF26243ADF8043070
:10C2800004238DF806303868032301AA6021FEF7E5
:10C29000E1FA142605F0C0F904460D4605F0BCF994
:10C2A000001B61EB0501B0F57A7F71F10001F5D358
:10C2B000013EEFD131460DF1030238688DF803607D
:10C2C000FFF794FA4FF4E853ADF8043008238DF8E3
:10C2D0000630386801AA03236021FEF7BBFA142652
:10C2E00005F09AF904460D4605F096F9001B61EB3E
:10C2F0000501B0F57A7F71F10001F5D3013EEFD170
:10C300000DF10302314638688DF80360FFF76EFACD
:10C3100038680DF102021E21FFF768FA012003B010
:10C32000F0BD00BFF0B5044683B00D461746061DAC
:10C3300020680379012B1AD0022B02D0002003B011
:10C34000F0BD8368DB0732464FF0FF015CBF324629
:10C35000FF21FFF7F9F90028F0D015B12379DB07A9
:10C36000E6D4002FEBD023793B7003B0F0BD826898
:10C37000417C90F9100002F00102CDE90062FF2239
:10C38000F8F79CF8E7E700BF30B50446051D2068C4
:10C390000379012B83B017D0022B02D0002003B009
:10C3A00030BD8368DB072A464FF0FF015CBF2A4699
:10C3B000FF21FFF7C9F90028F0D02379DB07EED57C
:10C3C00020680379012BE7D18268417C90F9100045
:10C3D00002F00102CDE90052FF22F8F76FF8EAE718
:10C3E00030B50246044652F8040B0379012B83B0A2
:10C3F0000ED0022B01D0002008E0FF21FFF7A4F9A6
:10C400000028F8D02079C04300F0010003B030BD0F
:10C410008568417C90F91000009205F001050195B6
:10C42000FF22F8F74BF8EBE730B5B42283B00446AF
:10C43000FF210068FDF792F910B9002003B030BD6C
:10C4400020680379012B04F1040514D0022BF4D1E8
:10C450008368DB072A464FF0FF015CBF2A46FF21B5
:10C46000FFF772F90028E8D02379DB07E6D52068CA
:10C470000379012BEAD18268417C90F9100002F027
:10C480000102CDE90052FF22F8F718F8EAE700BFF1
:10C4900030B50A4683B00446A5210068FDF75EF971
:10C4A00010B9002003B030BD20680379012B04F1DE
:10C4B000040514D0022BF4D18368DB072A464FF021
:10C4C000FF015CBF2A46FF21FFF73EF90028E8D0B4
:10C4D0002379DB07E6D520680379012BEAD182684E
:10C4E000417C90F9100002F00102CDE90052FF22D8
:10C4F000F7F7E4FFEAE700BF70B582B0CDE90023AB
:10C500000446FFF791FF10B9002002B070BD20680B
:10C510005522A521FDF722F90028F5D0251D206818
:10C520002A46FF21FFF762F90028EDD02379DB07C7
:10C53000F5D40DF1FF350DF1070615F8011F204662
:10C54000FFF7A6FF0028DFD0B542F6D1DDE700BF38
:10C55000002A35D0F0B5044683B00E468F18051D6D
:10C5600016F8012B2068A521FDF7F8F890B90020F6
:10C5700003B0F0BD8268417C90F9100002F0010226
:10C58000CDE90052FF22F7F799FF0028EFD0237979
:10C59000DB0710D520680379012BEBD0022BE6D105
:10C5A0008368DB072A464FF0FF015CBF2A46FF2164
:10C5B000FFF7CAF8E9E7B742D2D1012003B0F0BDD6
:10C5C0000120704770B5962282B004460E4600687E
:10C5D000FF21FDF7C3F810B9002002B070BD251D82
:10C5E00020680379012B1FD0022BF5D18368DB076C
:10C5F0002A464FF0FF015CBF2A46FF21FFF7A4F84F
:10C600000028E9D02379DB07EAD4E122206811462B
:10C61000FDF7A4F80028DFD020683246FF2102B0E1
:10C62000BDE87040FFF7E2B88268417C90F91000E5
:10C6300002F00102CDE90052FF22F7F73FFFDFE7EA
:10C64000002A43D0F0B5044683B00E468F18051D6E
:10C6500020689622FF21FDF781F890B9002003B0F1
:10C66000F0BD8268417C90F9100002F00102CDE932
:10C670000052FF22F7F722FF0028EFD02379DB07D3
:10C6800010D520680379012BEBD0022BE6D183680B
:10C69000DB072A464FF0FF015CBF2A46FF21FFF768
:10C6A00053F8E9E7E12220681146FDF757F8002822
:10C6B000D4D020683246FF21FFF798F80028CDD06B
:10C6C0000136B742C4D1012003B0F0BD012070474C
:10C6D00070B505460B460446164655F8040B82B065
:10C6E00087211A46FDF73AF820680379012B1AD002
:10C6F000022B02D0002002B070BD8368DB072A46FF
:10C700004FF0FF015CBF2A46FF21FFF71DF800280C
:10C71000F0D02379DA07E7D4002EECD0C3F340132E
:10C72000337002B070BD8268417C90F9100002F055
:10C730000102CDE90052FF22F7F7C0FEE7E700BF94
:10C7400070B5782182B00446164600680022FDF7D5
:10C7500005F810B9002002B070BD251D20680379CE
:10C76000012B14D0022BF5D18368DB072A464FF04A
:10C77000FF015CBF2A46FF21FEF7E6FF0028E9D053
:10C780002379DA07EAD45B09337002B070BD82689E
:10C79000417C90F9100002F00102CDE90052FF2225
:10C7A000F7F78CFEEAE700BF30B5CC2283B0044631
:10C7B000A5210068FCF7D2FF10B9002003B030BDFE
:10C7C00020680379012B04F1040514D0022BF4D165
:10C7D0008368DB072A464FF0FF015CBF2A46FF2132
:10C7E000FEF7B2FF0028E8D02379DB07E6D5206802
:10C7F0000379012BEAD18268417C90F9100002F0A4
:10C800000102CDE90052FF22F7F758FEEAE700BF28
:10C8100030B5B42283B00446FF210068FCF79EFFC8
:10C8200010B9002003B030BD251D20680379012B0D
:10C8300022D0022BF5D18368DB072A464FF0FF0197
:10C840005CBF2A46FF21FEF77FFF0028E9D023794D
:10C85000DA07EAD4CC212046FFF71AFE0028E0D000
:10C8600002E02379DB07DDD520682A46FF21FEF7A9
:10C87000BDFF0028F5D1D4E78268417C90F9100013
:10C8800002F00102CDE90052FF22F7F717FEDCE7C4
:10C890002DE9F04F8BB0CDE907230446002004902A
:10C8A0008A460390251D049B079A2046DE0002EB72
:10C8B000C30BFFF7B9FD20B935E0237913F001026E
:10C8C00007D020682A46FF21FEF790FF0028F4D108
:10C8D00029E005929A07099040F1D880F02120467E
:10C8E000FFF7D6FDF8B1079BDDF81480083E33440E
:10C8F000012606933746BAF1000F54D0082F52D8BC
:10C9000007F1FF394AFA09F909F0010920684FEAED
:10C91000C9127821FCF722FF28B120680379012B86
:10C9200050D0022B06D00020089B049A1A700BB03E
:10C93000BDE8F08F8368DB072A464FF0FF015CBF3C
:10C940002A46FF21FEF700FF0028ECD0237913F0E0
:10C950000102E2D1C3F3801CD9099B0646D5BCF184
:10C96000000F60D1BAF1000F5AD0082F58D889456E
:10C9700040F08880B9F1000F48D01BF808303343ED
:10C980000BF808307600013716F0FF06FFB2B2D17F
:10C9900008F101085FFA88F8B8F1080F43D00126C2
:10C9A000BAF1000FAAD1049BC3B1039BBB4215D9B6
:10C9B000069B13F808301E4214BF4FF001094FF0D8
:10C9C0000009A3E78268417C90F9100002F001029F
:10C9D000CDE90052FF22F7F771FDB5E7039BA3EB0A
:10C9E0000709B9FA89F94FEA59198FE7BAF1000F27
:10C9F00013D0082F11D8894596D1B9F1000FBCD1B9
:10CA0000059BBCF1000F08BF3B4605931BF808309F
:10CA100023EA06030BF80830B4E70029ADD1EFE7AD
:10CA20000029AAD1F2E7402F06D8089B049A1B7868
:10CA300093423FF638AF77E79BF807700BF1FF366C
:10CA40000BF1060B16F801CF082182EA0C0343F321
:10CA50000003013923F0730383EA520211F0FF014E
:10CA6000D2B24FEA5C0CF0D1B345EBD19742DCD1A6
:10CA7000049B0133DBB20493059B002B3FF454AFBE
:10CA80000393D2E7DDF8248040464DE780464046D8
:10CA90004AE700BF30B5044600680379012B85B032
:10CAA00062D0022B03D00025284605B030BD826835
:10CAB00002AD12F0010F18BF19462A4608BF8221A5
:10CAC000FEF742FE0028EED09DF80830DA07EAD5DE
:10CAD0002A46206807230321FDF736FF0546002874
:10CAE000E1D0206811220A21FCF738FE9DF80E30B3
:10CAF0001B07D8D42A49BDF8083031F8F82C13FBAD
:10CB000002F3284A93423FDBB3F5000F3ADA002BD9
:10CB1000B8BFFF331B125B421BB2BDF80A20E3868D
:10CB200031F8F63C12FB03F31E4A934230DBB3F5B7
:10CB3000000F31DA002BB8BFFF3343F30F22BDF8EB
:10CB40000C3031F8F41C2287164A13FB01F3934290
:10CB50001CDBB3F5000F1DDA002BB8BFFF331B122F
:10CB60005B421BB263879FE7826890F910C0417CEB
:10CB700002F0010202AD0192009560460222F7F731
:10CB80009DFC9FE7084BC8E7084BC6E7074BE9E762
:10CB9000064AD4E7044BE5E747F6FF72CFE700BF4C
:10CBA000B86E002001FF7FFF0180FFFF0080FFFFC4
:10CBB00010B5044686B0006800238DF80F30037965
:10CBC000012B31D0022B02D0002006B010BD8368AB
:10CBD000D9070DF10F024CBF2721A721FEF7B4FDA5
:10CBE0000028F1D09DF80F301B07EDD520680623F3
:10CBF00004AA2821FDF7A8FE28B3BDF91030BDF91D
:10CC00001220002BB8BF03339B10E386BDF914300C
:10CC1000002AB8BF0332002BB8BF033392109B1019
:10CC20002287638706B010BD826890F910C0417CEE
:10CC300002F0010201920DF10F02009260462722DC
:10CC4000F7F73CFCCCE7C4F8360060870020BCE76F
:10CC500030B504464FF0000C0068C4F836C0A4F8A4
:10CC60003AC00379012B87B02AD0022B02D00020D2
:10CC700007B030BD8368D9070DF10F024CBF614684
:10CC80008021FEF761FD0028F1D09DF80F301B07D1
:10CC9000EDD52068062304AA0121FDF755FE0028E2
:10CCA000E5D0BDF81430BDF81010BDF812205BBA05
:10CCB00049BA52BA5B42E1862287638707B030BD2A
:10CCC0008568417C90F9100005F0010501950DF192
:10CCD0000F0562460095F7F7F1FBD4E710B504465F
:10CCE00000230068C4F8363063870379012B86B0CF
:10CCF00023D0022B02D0002006B010BD8368D907D4
:10CD00000DF10F024CBF06218621FEF71DFD002804
:10CD1000F1D09DF80F30DB07EDD52068062304AA7B
:10CD20000021FDF711FE0028E5D0049ABDF814306B
:10CD3000C4F83620638706B010BD826890F910C031
:10CD4000417C02F0010201920DF10F020092604657
:10CD50000622F7F7B3FBDAE710B5044600230068B4
:10CD6000C4F8363063870379012B86B029D0022BB3
:10CD700002D0002006B010BD8368D9070DF10F0264
:10CD80004CBF09218921FEF7DFFC0028F1D09DF876
:10CD90000F30DB07EDD52068062304AA0121FDF73B
:10CDA000D3FD0028E5D0BDF81210BDF81020BDF865
:10CDB0001430494252425B42E1862287638706B0C3
:10CDC00010BD826890F910C0417C02F0010201920E
:10CDD0000DF10F02009260460922F7F76FFBD4E7CE
:10CDE00010B5044600230068C4F836306387037921
:10CDF000012B86B012D0022B0DD18368DB070DF119
:10CE00000B024CBF3421B421FEF79EFC18B19DF9F2
:10CE10000B30002B11DB002006B010BD826890F9AA
:10CE200010C0417C02F0010201920DF10B02009250
:10CE300060463422F7F742FBE8E72068092303AA9B
:10CE40002421FDF781FD0028E5D09DF810209DF8F4
:10CE50000F109DF81330120442EA0162C2F30F4230
:10CE60009DF8121022871B049DF80D2043EA0163F0
:10CE70009DF80C10120442EA0162C2F30F42C3F3A0
:10CE80000F43E286638706B010BD00BF10B503688C
:10CE9000DA6B82B0044612B1904740B123685B6BF5
:10CEA0001BB1214601A8984718B9FF23E38202B0BD
:10CEB00010BDBDF80630013B9BB2F7E7F0B5044664
:10CEC00083B018460D4616461F4674F003FA2844F0
:10CED000D4F800C0A073E673204600240094DCF868
:10CEE00014403B4632462946A04703B0F0BD00BF80
:10CEF00038B58B68016004460D46984700230B4AFD
:10CF0000226123752B6B13B1204698472075084B7F
:10CF100013F8F03C1BB1237D23F00103237500239C
:10CF2000E3822046BDE83840B0E700BF0001FF00C3
:10CF3000B86E002010B5154B53F8EC4C84B084B19A
:10CF40002379012B10D0022B0BD1A16811F0010124
:10CF5000024618BF8021204604B0BDE81040FCF70F
:10CF6000A7BB002004B010BDA268617C8DF80F0043
:10CF700002F0010294F910000DF10F04CDE9004216
:10CF80008022F7F767FA04B010BD00BFB86E00202A
:10CF9000F0B5294B53F8EC5C85B09DB1B0228021EF
:10CFA0002846FCF7DBFB402280212846FCF7D6FB15
:10CFB000002280212846FCF7D1FB10228021284640
:10CFC000FCF7CCFB4FF480642DB9013CA4B2002CDB
:10CFD000FBD105B0F0BD00270DF10F062B79012B19
:10CFE00008D0022B04F1FF3217D094B2002CF0D0FD
:10CFF000012BF6D1AA6895F91000697C8DF80F70A5
:10D0000002F00102013CCDE90062A4B24022F7F730
:10D0100021FA002CE2D105B0F0BDAA68013C12F063
:10D02000010218BF002240212846A4B2FCF740FBB1
:10D03000002CD3D105B0F0BDB86E00200B4B10B55D
:10D0400053F8EC4C8CB15038C2B280212046FCF72A
:10D0500085FB002280212046FCF780FB2046102221
:10D06000BDE810408021FCF779BB10BDB86E0020F0
:10D07000F0B5264B264C53F8EC5C203800EB8000D2
:10D08000661D85B00444064425B90134A642FCD18E
:10D0900005B0F0BD0DF10F072B792278012B1BD0C5
:10D0A000022B0AD00134A642F7D1002240212846A3
:10D0B00005B0BDE8F040FCF751BBAB68DB074FF0B3
:10D0C0004001284619D50134FCF7F2FAA642E3D113
:10D0D000002DEAD105B0F0BD8DF80F20AA6895F9B2
:10D0E0001000697C02F00102CDE900720134402297
:10D0F000F7F7B0F9B442CFD1D7E70134FCF7D8FA4B
:10D10000B442C9D1002DE5D0CFE700BFB86E0020F2
:10D1100090550808F0B5754B53F8EC5C85B0002DC0
:10D1200000F09680D42280212846FCF717FB80224D
:10D1300011462846FCF712FBA82280212846FCF75E
:10D140000DFB3F2280212846FCF708FBD3228021DB
:10D150002846FCF703FB002280212846FCF7FEFA54
:10D16000402280212846FCF7F9FA8D2280212846AA
:10D17000FCF7F4FA142280212846FCF7EFFAA122EA
:10D1800080212846FCF7EAFAC82280212846FCF7CD
:10D19000E5FADA2280212846FCF7E0FA1222802103
:10D1A0002846FCF7DBFA812280212846FCF7D6FAD4
:10D1B000CF2280212846FCF7D1FAD92280212846A7
:10D1C000FCF7CCFAF12280212846FCF7C7FADB22D3
:10D1D00080212846FCF7C2FA402280212846FCF72D
:10D1E000BDFAA42280212846FCF7B8FAA6228021A5
:10D1F0002846FCF7B3FAAF2280212846FCF7AEFAA6
:10D20000A62280212846FCF7A9FAAE2280212846D2
:10D21000FCF7A4FA202280212846FCF79FFA00227E
:10D2200080212846FCF79AFAB02280212846FCF794
:10D2300095FA402280212846FCF790FA00228021AE
:10D240002846FCF78BFA102280212846FCF786FA44
:10D250004FF4806435B9013CA4B2002CFBD101200D
:10D2600005B0F0BD00270DF10F062B79012B2AD058
:10D27000022B04F1FF3214D094B2002CF6D181229B
:10D2800080212846FCF76AFAC82280212846FCF74C
:10D2900065FAAF2280212846FCF760FA012005B02C
:10D2A000F0BDAA68013C12F0010218BF0022402123
:10D2B0002846A4B2FCF7FCF9002CD6D1002DDED113
:10D2C000012005B0F0BDAA6895F91000697C8DF8C1
:10D2D0000F7002F00102013CCDE90062A4B24022CD
:10D2E000F7F7B8F8002CC0D1C9E700BFB86E00202E
:10D2F000FAF73ABBFAF738BBFAF736BBFAF734BBA2
:10D30000FAF732BBFAF730BB01207047034620B171
:10D31000026812B1D26902B1104793ED017A084B4D
:10D32000B8EEC77A53ED396AF6EE007AE7EE267A60
:10D33000FDEEE77A17EE900A00F30B00704700BF8E
:10D34000B86E0020034620B1026812B1126A02B121
:10D35000104793ED027A084BB8EEC77A53ED386A5E
:10D36000F6EE007AE7EE267AFDEEE77A17EE900AFF
:10D3700000F30B00704700BFB86E0020034628B1D1
:10D3800002681AB1516A09B19369184793ED037A9B
:10D39000074BB8EEC77A53ED376AF6EE007AE7EE40
:10D3A000267AFDEEE77A17EE900A00F30B0070473D
:10D3B000B86E002010B5044630B1036823B1DB68B5
:10D3C00013B1BDE81040184704F026F9D4E904234E
:10D3D0009042994134BF0120002010BDF8B170B5D2
:10D3E00006680F4B06F13F4202F57E0203EB9223E3
:10D3F0000C4682B0054693F82C056CF061FEC4F330
:10D400004112C4F30013A9883046CDE90032C4F3B9
:10D41000810304F0030273F0B1FD02B070BD7047E8
:10D4200008530808B0B3F0B507681B4B144607F162
:10D430003F4202F57E0203EB9223054683B093F848
:10D440002C050E466CF03CFEA988B1FA81F3C3F1BD
:10D450001F03C3F3CC0207EB820203F00703156A34
:10D460004FF00F0C9B009C400CFA03F325EA0303DA
:10D470001362136A1C431462C6F300137209CDE9E8
:10D4800000323846C6F3810306F0030273F076FDDE
:10D4900003B0F0BD704700BF0853080810B5040979
:10D4A000013C032C19D80F4A00F00F0332F8140086
:10D4B00040FA03F212F0010211D0012202FA03F342
:10D4C000013B184077F032FD074B084A1B5D1844BA
:10D4D00000EB400002EB800010BD002010BD1046A4
:10D4E00010BD00BF00530808FC520808A4380020F3
:10D4F0002DE9F04F542204460021C34891B077F043
:10D500007DFCC24A611EE01C144611F8013F5D1EFD
:10D51000052D88BF0023814244F8043BF5D102F178
:10D520001003114651F8040B012800F0588199426C
:10D53000F8D1114651F8040B022800F046819942B7
:10D54000F8D1114651F8040B032800F0528199429A
:10D55000F8D152F8041B042900F02D819A42F8D129
:10D560000520F9F7C5FB0620DFF89C92DFF8BC82A6
:10D57000F9F7BEFB4C464FF01A0A002608F2345B5E
:10D58000277B57B3384694F90D50FFF787FF28B132
:10D5900005238371002380F807A003721321FFF78E
:10D5A0001DFF00231BF83310B9422FD00133102B7D
:10D5B000F8D10021964B216105EB450503EBC5052C
:10D5C0000122D5F8F43923751344C5F8F43907233B
:10D5D000A375627585F8F02916440AF1010A5FFA0D
:10D5E0008AFABAF1200F04F10C04C9D15EB1894D59
:10D5F000894F00262B7C73B90136032E05F11805DF
:10D6000007F58C77F6D111B0BDE8F08F08EBC303B6
:10D61000D3F83815CEE768796CF052FD28796CF0B4
:10D620004FFDD5F808A05046F6F7A6F8D5F81480B7
:10D630002C680397142303FB08F305930023CDE91B
:10D640000C33CDE90E3304930693EB68019304F198
:10D650004C034FF4806202934FF40063CDE907233B
:10D660004FF400514FF48073CDE9091350464FF445
:10D67000003301A90B936CF0F7FCDAF8002067493E
:10D68000674B42F00102CAF800204A68134043F495
:10D6900040334B606368B8F1010F23F04073D4BF8F
:10D6A0000022012223F4807343EA02236360A2680C
:10D6B0005C4B134043F00203A360E36A08F1FF38B8
:10D6C0005FFA88F823F4700343EA0853E36209F130
:10D6D00048014B4601204FFA86FC02E00C338B4296
:10D6E00031D05A7D002AF9D093F90D206245F5D149
:10D6F0001A7C93F816A0092A36D802EB420BD4F80C
:10D7000010800AFA0BFE4FF0070A0AFA0BFA28EA11
:10D710000A084EEA080EC4F810E0062837D800F1CF
:10D72000FF3ED4F834800EEB8E0E4FF01F0A02FA43
:10D730000EF20AFA0EFE28EA0E0E42EA0E026263AA
:10D740000130C0B2CAE7A36843F40073A360A368C2
:10D7500043F48073A360A36843F00103A360A3684C
:10D7600043F08043A36047E7A2F10A0ED4F80C808F
:10D770000EEB4E0E4FF0070B0AFA0EFA0BFA0EFEE6
:10D7800028EA0E0E4AEA0E0EC4F80CE0C5E70C2893
:10D790004ED8A0F1070ED4F830800EEB8E0E4FF06D
:10D7A0001F0A02FA0EF20AFA0EFE28EA0E0E42EAEA
:10D7B0000E022263C4E71C4B93F87C2C302101320B
:10D7C00083F8581C83F87C2CCAE6174991F87C0C26
:10D7D0003524013081F8404C81F87C0CB1E61249C7
:10D7E00091F87C0C3424013081F8344C81F87C0CA5
:10D7F0009FE60D4991F87C0C2024013081F84C4CB7
:10D8000081F87C0CA5E600BFE8690020C45D00201B
:10D81000300C002010160020406A00200023014038
:10D82000E030FCFFFDF7FFC0C05D00200853080892
:10D83000A0F10D0ED4F82C800EEB8E0E4FF01F0AC7
:10D8400002FA0EF20AFA0EFE28EA0E0E42EA0E0262
:10D85000E26275E710B503681A79022A044603D01C
:10D8600000232371236010BD987AFFF717FE00286C
:10D87000F6D040F61A610022C18002722021FFF723
:10D88000ADFD00232371236010BD00BF2DE9F04FD3
:10D89000B24EB34CA64285B057D21D4602E00C36BC
:10D8A000A64252D273798B42F9D13379834201D0A7
:10D8B0000028F4D1F3799342F1D13468002C44D09C
:10D8C00000236360A360E36023616361A361E3619C
:10D8D00026603379237196F806B0C4F808B0317A1F
:10D8E000E160012B33D0022B2FD1F07AFFF7D6FD68
:10D8F00096F90970A061B07A2774FFF7CFFD06464C
:10D900006061F8B1DFF8788207EB870108EB8101ED
:10D91000BB00D1F890990193B9F1000F12D091F8A2
:10D92000A209E8B10E220023F2713372B571092108
:10D930003046FFF753FD3368B2881A83204605B09E
:10D94000BDE8F08F2046FFF785FF0024F6E7F07A68
:10D95000FFF7A4FD727AB37A6374A0612274EDE7D5
:10D9600091F898A950466CF0ABFB4FEA5A10012190
:10D970000AF01F0A023801FA0AF1032808D8DFE882
:10D9800000F0ADA1A702774B586920EA0101596167
:10D99000BB00D91908EB810107F1010A91F895093B
:10D9A000FFF77CFD5FFA8AFA014620B180F808A0F3
:10D9B00040F60A30C880BB00D81908EB80000291FD
:10D9C00090F89709FFF76AFD02990190034620B18C
:10D9D00080F808A040F60A50D880BB00D81908EBA0
:10D9E0008000029190F89609FFF758FD02990346CE
:10D9F00020B180F808A040F60A40D880BA00D019BB
:10DA000008EB80001BF0040290F899A9CDE90223ED
:10DA10000846524668D04A21FFF704FD0198524655
:10DA20002A21FFF7FFFC039B524618460A21FFF705
:10DA3000F9FCBB00DA1908EB820292F894B9BBF149
:10DA4000000F61D1484A914571D0484A914563D051
:10DA5000474A914500F0A180464A914500F09280E6
:10DA6000454A91456ED0454A914500F0A180029B00
:10DA7000B9F80010002B01F441510CBF0322002221
:10DA80000A4342F44572A9F80020B9F81C2022F498
:10DA900000621204120CA9F81C200722A9F8102019
:10DAA000B9F8002092B242F04002A9F80020BBF180
:10DAB000000F20D1BB003B4408EB8308012388F80A
:10DAC000A2392FE7274B186A20EA010119625FE7A4
:10DAD000244B186920EA0101196159E7214B586A62
:10DAE00020EA0101596253E70A21FFF79BFC0198E4
:10DAF00052460A2195E75846FFF7D0FC0028D9D0B6
:10DB0000026883881383D5E75846FFF7C7FC52465F
:10DB10000921FFF787FC95E702F50032116A41F40D
:10DB200080411162116A21F4804111629FE702F580
:10DB30008432516A41F480515162516A21F480511A
:10DB4000516294E702F56842516A41F480115162D2
:10DB5000516A21F48011516289E700BF7885090874
:10DB60009487090800380240003001400038004026
:10DB7000003C00400034014000500140005401408E
:10DB8000300C002002F58232516A41F4005151629A
:10DB9000516A21F40051516269E702F5FE32116ABF
:10DBA00041F400411162116A21F4004111625EE703
:10DBB00002F56442516A41F400115162516A21F444
:10DBC0000011516253E700BF014B1B685B681847A7
:10DBD000106E0020024B1B6808309B68184700BF7E
:10DBE000106E00200120704701207047012070470F
:10DBF000012070470120704731B10C4BD3ED017A01
:10DC0000F8EEE77AC1ED007A72B1084BDFED086AF1
:10DC10009B68A3F5D543333B07EE903AF8EEE77ADD
:10DC200087EEA67A82ED007A704700BF106E002062
:10DC30000000C842012070470120704710B4414CD9
:10DC40000023224692F90410012902F10C022DD082
:10DC50000133052BF6D12246002392F90410032943
:10DC600002F10C0234D00133052BF6D1002394F9D4
:10DC70000420052A04F10C043FD00133052BF6D112
:10DC8000314B1B68D9034ED5304B016803F1F004CA
:10DC900002E01433A34246D01A689142F9D1DA68FF
:10DCA000D201F6D501205DF8044B7047284A03EBFA
:10DCB000430302EB8303DB68EBB1264A037992F856
:10DCC0003DC09C45EED092F83C209A42C3D1E9E792
:10DCD0001F4A03EB430302EB8303DB68002BC6D030
:10DCE0001D4A037992F83D109942DBD092F83C200E
:10DCF0009A42BBD1D6E72246AFE7154A03EB43036E
:10DD000002EB8303DB68002BBAD0144A037992F844
:10DD10003D109942C6D092F83C209A42C2D00A4B9C
:10DD20001B68D903B0D40379203BDBB2152B06D88E
:10DD30000B495DF8044BD94001F001007047002009
:10DD4000B1E700BF1C6E0020B40000105816002080
:10DD5000106E002004030020500500209C070020C6
:10DD6000010031000C4B10B5844603F1F00E002089
:10DD700002E014339E450ED01A686245F9D1DA6884
:10DD80008A4218BFD96000F1010403F1140318BFDF
:10DD9000E0B29E45F0D110BD58160020704700BF7C
:10DDA000044B40F2FF7203EBC0039142A8BF11463F
:10DDB00099807047645F0020112806D8044B03EB5C
:10DDC00080039B6C0BB19B68196028F01BBD00BFE2
:10DDD000106E0020112806D8034B03EB80039B6CC8
:10DDE0000BB19B6819607047106E00200D4A92F8C5
:10DDF000F03083B10C4B93F8901061B193F891100F
:10DE000061B1D2F8F4000022FA2883F89120A8BF6B
:10DE10004FF0FF3070476FF0010070476FF0020065
:10DE2000704700BF58160020106E00202DE9F04109
:10DE3000104C04F1940884F895101746002502232D
:10DE40004246FF21064684F89450FCF703FD68B172
:10DE5000424630460223FF21FCF776FD30B1B4F88C
:10DE600094305BBA28463B80BDE8F0816FF00C002F
:10DE7000FAE700BF106E00200C4B93F894218AB192
:10DE800093F895215AB10A49D1F8F8000022B0F56B
:10DE9000967F83F89521A8BF4FF0FF3070476FF051
:10DEA000020070476FF00100704700BF106E002045
:10DEB00058160020024BD3F898315B68184700BF12
:10DEC000106E0020024BD3F898319B68184700BFB2
:10DED000106E0020024BD3F89831DB68184700BF62
:10DEE000106E0020014BD3F8FC007047581600203C
:10DEF000054B93F89C311BB1044BD3F800017047DC
:10DF00006FF00100704700BF106E0020581600200F
:10DF1000F0B54B4D95F8903083B03BB195F89D61CD
:10DF2000012E044639D0022E57D00EB103B0F0BDF9
:10DF3000012280210068FBF711FC20680122FF21EB
:10DF4000FBF70CFC324631462068FBF707FC95F8DE
:10DF50009E2120689121FBF701FC314620680122B7
:10DF6000FBF7FCFB32462068FF21FBF7F7FB32464C
:10DF700020688021FBF7F2FB314620680122FBF785
:10DF8000EDFB304B30491A6881F8F0000123C5F8E9
:10DF9000A02185F89D3103B0F0BD01AA00682A4F89
:10DFA0000021FDF723FC9DF8043087F8F000DA0724
:10DFB0003DD5D5F8A431002BB8D0224AD5F8A01110
:10DFC000126892B2521A9342B0D24FF0FF3200233D
:10DFD000C7F8F42085F89D31A8E700681A4F01AA18
:10DFE0001321FDF703FC9DF8043087F8F0005B0770
:10DFF000DFD02068334601AA1E21FCF7A5FCBDF83E
:10E000000430206801220B215CBAFBF7A7FB0F4B01
:10E0100087F8F000A4B2A3FB0434E4080122002333
:10E02000C7F8F44085F8912085F89D317EE7054AD0
:10E0300002231268C5F8A02185F89D3176E700BF5C
:10E04000106E0020EC28002058160020CDCCCCCC3F
:10E0500038B5324D04460323006805F5847200216B
:10E06000FCF772FC50B96FF0010300222068C5F87C
:10E0700004311146BDE83840FBF770BB95F80AC182
:10E0800095F80831082158B200284FEA4002A8BF8D
:10E090005B0082F00702B4BFD3B2DBB20139F2D128
:10E0A00095F809215340082259B20029B8BF490008
:10E0B0004FEA4303B6BF81F00701DBB2CBB2013AAE
:10E0C000F2D19C4520681FD1B5F808315BBA9BB2EC
:10E0D000591E89B24FF6FD7C61450CD807EE903A87
:10E0E000F8EEE77AF2EE046A87EEA67AFDEEC77ADA
:10E0F00017EE903AB9E74FF0FF33C5F804311146F7
:10E10000BDE83840FBF72ABB6FF00203C5F80431C5
:10E110001146BDE83840FBF721BB00BF5816002070
:10E12000014BD3F80401704758160020437A5A1C5B
:10E130000344D2B242729972037A934200D9704773
:10E14000002AFCD010B5044604F10A01D0E90030E1
:10E1500098470023637210BD30B5032083B00D468D
:10E160001446FBF7CBF901909DB107EE900A9FEDA5
:10E170000B7AF8EE677AF0EE006A67EE877AB8EE0F
:10E18000047AA7EEA67ADFED067A67EE277AC5ED68
:10E19000007A0CB1034B236003B030BD6740533AA3
:10E1A00000007A443313904300B500680379012BD3
:10E1B00085B00DD0022B07D1012303AAFF21FCF764
:10E1C0006BFB05B05DF804FB002005B05DF804FBB7
:10E1D0008268417C90F9100002F00102019203AACA
:10E1E0000092FF22F6F76AF905B05DF804FB00BF64
:10E1F00030B5044600680379012B85B02DD0022B81
:10E200000ED0224B6FF00102C3F8FC202049214AB6
:10E21000D1F8A83115683233AB422CD305B030BDEC
:10E22000826812F0010F18BF512103AA08BFD12143
:10E23000FCF732FB0028E4D0BDF80C30134A5BBA7F
:10E240009BB2C2F8FC30D2F8FC30B3F5C87FDDDDFC
:10E250004FF0FF33C2F8FC30D8E78368417C90F977
:10E26000100003F00103019303AB0093512202233A
:10E27000F6F724F9DEE701F5D672C1F8A851206857
:10E2800000235121FCF7E6FA05B030BD58160020F6
:10E29000106E0020EC28002000B500680379012BE7
:10E2A00085B02DD0022B24D1826812F0010F18BF47
:10E2B000002103AA08BF8021FCF7EEFA1B4B83F86C
:10E2C0009C0198B1BDF80C305BBA9BB2B3F5FA6F04
:10E2D00024D2174A1749A2FB0323DB0807EE903A22
:10E2E000F8EEE77AFDEEE77AC1ED407A05B05DF829
:10E2F00004FB0E4B002283F89C2105B05DF804FB63
:10E300008368417C90F9100003AA03F00103CDE972
:10E31000002302230022F6F7D1F8CFE7054B4FF098
:10E32000FF32C3F8002105B05DF804FB106E002039
:10E33000CDCCCCCC5816002010B500680379012B49
:10E3400084B00C461FD0022B02D0002004B010BDB8
:10E35000826812F0010F18BF002103AA08BF8021B4
:10E36000FCF79AFA0028F0D05CB19DF80D309DF9C9
:10E370000C20DB0903EB830302EB820203EB420375
:10E38000238004B010BD8368417C90F9100003F035
:10E390000103019303AB009300220223F6F78EF8EA
:10E3A000E0E700BF70B50668F56982B00446002D4D
:10E3B00059D000232B7004230DEB03023046FF21BC
:10E3C000FCF7C2FA10B9002002B070BD2068042327
:10E3D0006A46FF21FCF7B8FA0028F4D09DF8043013
:10E3E0009B09023B012BEED9BDF80430BDF8062095
:10E3F000BDF80010BDF802605BBA43F6FF74C3F3CA
:10E400000D03A342DFD0002BDDD052BAC2F34A1273
:10E4100040F2FF7C6245D6D0002AD4D049BAC1F37D
:10E420000D01A142CFD00029CDD076BAC6F34A164D
:10E430006645C8D0002EC6D05C1A002CB8BF644216
:10E44000FF2CC0DC941B002CB8BF6442FF2CBADC4C
:10E450000B445B1032445210C5F805300123C5F857
:10E4600001202B70B0E709211420FAF747F8F0617A
:10E47000054626689DE700BF70B50668F0690D4641
:10E480001446A0B3D0F80130CDB1D0F805209FEDEF
:10E490001B7ADFED1B5ADFED1B6A07EE902AF8EEC0
:10E4A000677AB7EE006A77EEC77A77EEA77A87EEDB
:10E4B000A57A77EE467A67EEE67AC5ED007AACB1DA
:10E4C00007EE903A9FED107ADFED106A9FED106A2B
:10E4D000F8EEE77A67EE877A87EEA67ADFED0D6AC7
:10E4E00077EE467A77EEA67AC4ED007A70BD092100
:10E4F0001420FAF703F8F061C4E700BF9AC9CC44CE
:10E500009AC94C460E76D7450000484300E0FF44C8
:10E51000000048423393884338B505680446E869EB
:10E5200080B1C3681B0E4FF0010205D12846482177
:10E53000BDE83840FBF712B928465821BDE83840FD
:10E54000FBF70CB909211420F9F7D8FFE861256819
:10E55000E7E700BF70B50668F46982B0ECB1032349
:10E5600001AA00213046E568FCF7EEF998B19DF864
:10E5700005309DF804201B0243EA02439DF8062063
:10E580002D0E43EA02031BBFE268236143F0807350
:10E5900022F07F43E36002B070BD054609211420DC
:10E5A000F9F7ACFFF06104462E68D8E72DE9F04793
:10E5B0000668F0690D461446002867D0C2680369F2
:10E5C00032F07F4C60D0002B5ED002894189D201AD
:10E5D0009B1A62EB0202FDB3B0F804A0C688B0F843
:10E5E00002E0B0F800909FED2C7AAAFB03080AFB2A
:10E5F0000288C0094FEAC93940EA486010EB0900B7
:10E600004FEAE818A0FB0C0948F100080CFB089839
:10E61000A6FB03C906FB02964FEA5C1C4FEA4E4775
:10E62000400D4CEAC66C40EAC8201CEB070C4FEAD0
:10E63000DE3E4EEB661E4FEA6858B0EB0C0068EB0E
:10E640000E08C00B40EA484007EE900AF8EEE77A61
:10E6500067EE877AC5ED007AB4B1A1FB033001FB08
:10E6600002025B0D43EAC22313F5FA6307EE903A08
:10E670009FED0A6ADFED0A6AF8EEE77A87EE867A9E
:10E6800077EE267AC4ED007ABDE8F08709211420E0
:10E69000F9F734FFF06191E77B81303F0000C84219
:10E6A0003393884370B50668F46982B0F4B10023EF
:10E6B000237004230DEB0302FF213046FCF744F9DD
:10E6C00010B39DF804309B0919D1BDF80420BDF8A2
:10E6D000063052BA5BBA92B2C3F34A1301212170D9
:10E6E000C4F80520C4F8013002B070BD0546092108
:10E6F0001420F9F703FFF06104462E68D7E7044AB7
:10E7000004210320F9F772FE002002B070BD00BFA3
:10E71000F8FE080870B50668F06982B00D46144628
:10E72000002848D0D0F80530DFED266A9FED267A24
:10E7300007EE903AF8EE677AD0F8013077EEE67A95
:10E74000F3EE096A67EE877AB2EE047A67EEA67A8C
:10E75000F4EEC77AF1EE10FA20DCBAEE047AF4EEA9
:10E76000C77AF1EE10FA19D42DB19FED187A67EE41
:10E77000877AC5ED007A7CB107EE903A9FED146A76
:10E78000DFED146AB8EE677ADFED137AE7EE067A0A
:10E7900077EEA67AC4ED007A02B070BD17EE900A4B
:10E7A00072F004FF0D4ACDE9000104210320F9F7BE
:10E7B0001DFE02B070BD09211420F9F79FFEF06123
:10E7C000B0E700BF00000046000080380AD7784359
:10E7D0000319C83D33938843000048C21CFF080852
:10E7E000F0B52DED028B4D4E16F84C3C022B83B04C
:10E7F0000D46144619D0DFED4A7A7DB19FED497A76
:10E800009FED496ADFED496A67EEA77A67EE877A7E
:10E8100087EE867A77EE267AC5ED007A0CB1444B06
:10E82000236003B0BDEC028BF0BD424B317C5B68D2
:10E8300003F0020239BB5B0525D42AB3B6F93630A2
:10E8400007EE903AB6F93430F8EEE77A06EE903AF1
:10E8500027EEA77AF8EEE66AB6F93830A6EEA67A81
:10E8600007EE903AF8EEE77AA7EEA77AB5EEC07A0F
:10E87000F1EE10FABFDBF1EEC77AF4EE677AF1EE53
:10E8800010FABAD7B7E71AB9336DD3ED337AB4E7D4
:10E89000294F0DF106002CF0E7FCBDF80630D7F843
:10E8A0009C259FED266ADFED266A9FED267A9B1A4E
:10E8B00007EE903AF8EEE77AB0EE408A67EE867A95
:10E8C000A7EEA67AFDEEC77AB0EE470A17EE903AA9
:10E8D0002033402B1FD8F9F7D1FB1B4B97F8C211FF
:10E8E000D6ED077AA3F12C021846443B002918BF45
:10E8F000134693ED057AD0ED006A77EE877AE8EE5D
:10E90000406A27EEA77AA6EEA67AB5EEC07AF1EEB7
:10E9100010FAB0DA6FE79FED020ADEE7087F002009
:10E9200000000000CDCC9C3F00409C4682E6C547DD
:10E9300033139043B4000010106E00200AD7233C1C
:10E9400035FA8E3CDB0FC93FC073002010B50B4B6E
:10E9500082B053F8304001916CB107EE901A94EDFB
:10E96000047A94ED030AF8EEE77AA7EE870A74F0CA
:10E9700055F9A368186002B010BD00BF645F0020A5
:10E980002DE9F041DFF8BC802C4E2D4D41F0010205
:10E9900084B000210446FAF7E1FED8F80070C6F80A
:10E9A000A07119E0022B3FD1A368DB070DF10F0224
:10E9B0004FF0130120465EBF0DF10F029321204658
:10E9C000FCF7C2FE9DF80F3085F8F00013F0070346
:10E9D00019D1D6F8A4214ABB2379012BE2D1A26830
:10E9E000617C94F9100002F0010201920DF10F0216
:10E9F00000921322F5F762FD9DF80F3085F8F000C4
:10EA000013F00703E5D001220B212046FAF7A6FEFA
:10EA1000002211462046FAF7A1FE012385F8F000F6
:10EA2000184604B0BDE8F0810020CBE7D8F800100C
:10EA300089B2C91B8A42CFD2F2E700BF106E002014
:10EA400058160020EC28002010B5194C84F89510B9
:10EA5000017984F8962001294FF0000282B084F8F1
:10EA6000942016D0022903D06FF00C0002B010BD24
:10EA7000836813F0010F04F194024FF0030314BFF5
:10EA8000FF217F21FBF78EFE0028EDD0002002B091
:10EA900010BD8268417C90F91000943402F00102AC
:10EAA000CDE900420323FF22F5F7D4FCECE700BFD9
:10EAB000106E002000680379012B0BD0022B00D0D0
:10EAC000704783680E4A13F0010315D000235121CB
:10EAD000FBF768BE00B58368094A417C90F91000D5
:10EAE00083B003F00103CDE9002300235122F5F7A1
:10EAF000B1FC03B05DF804FB5121FBF753BE00BF2E
:10EB0000BC6F002030B5194D95F8943183B00BB926
:10EB100003B030BD04460DF10501006871F074FAD0
:10EB20009DF805307BB92068114A01214FF4064455
:10EB300085F896100323FF21A5F8944003B0BDE8A3
:10EB40003040FBF787BE0DF1060296212068FFF7E3
:10EB50006DF9084ABDF806300749A2FB0323DB081C
:10EB60000122C1F8F83085F89521DCE7106E00200D
:10EB7000A46E0020CDCCCCCC5816002000680379C0
:10EB8000012B0AD0022B00D07047826812F00102DC
:10EB900018D000221146FAF78BBD00B5826890F9B3
:10EBA00010C0417C85B002F0010201920DF10F020C
:10EBB0000092604600228DF80F20F5F74BFC05B05F
:10EBC0005DF804FB1146FAF773BD00BFF8B50446C3
:10EBD0000F46164600252046202176F026F90446E9
:10EBE000C8B10378202B03D114F8013F202BFBD0B0
:10EBF0002046FAF789F9B0F5617F10DB40F634035F
:10EC0000984211DD30231A46C5B17B703378013349
:10EC100033702046F8BD002DFBD10125DBE7002332
:10EC20001A46002DF1D109E0074AA0F56173A2FB55
:10EC30000323DA08C3F3C703002DE6D13A70337813
:10EC400001333370E9E700BF1F85EB51074B53F8E1
:10EC5000203021B14BB11A689B8853837047002B39
:10EC6000FCD01A689B88138370477047D4580808F3
:10EC70002DE9F04F604BD3F8549091B0B9F1000FEB
:10EC800004D05E4A03214846F4F78EF80021484636
:10EC9000F4F702F9D9F80430594DD3F800801F6910
:10ECA0000022560105EB4210A959794011F47C5419
:10ECB00002F1010208D0102AF3D10023C9F80C3068
:10ECC000002011B0BDE8F08F027FC9F80C00002AC7
:10ECD000F6D1B8F84420DFF840A16FEA42426FEA6B
:10ECE000524292B2A8F84420B8F8002092B242F002
:10ECF0008002A8F8002093F805B09B791AF80B1051
:10ED0000B8F820205B074CBF042301238B409BB243
:10ED100092B222EA0302A8F82020B8F8202039494C
:10ED200092B21343A8F82030B8F8003042689BB282
:10ED300043F00103A8F80030334B9A42334A136B77
:10ED40000CBF43F4001343F48003136306F118026D
:10ED50004FF0070C354421F802C04B462C490322E2
:10ED6000F4F7FEFAAD682846F4F706FD2B6823F0A9
:10ED700001032B602846F4F7FFFC0023CDE90C3398
:10ED8000CDE90E3306930A93BBF1030F05D8DFE8F4
:10ED90000BF0302D022A08F13C04FFB20AEB870A7F
:10EDA00040F62B4205921B48DAF8043001934FF4E9
:10EDB00080614FF48042079109924FF480514022C4
:10EDC000CDE9030208914FF40033284601A90B93C3
:10EDD00002946BF049F92B68012043F010032B607B
:10EDE00011B0BDE8F08F08F14004D6E708F138040F
:10EDF000D3E708F13404D0E7087F0020009F240007
:10EE0000EC090020F00900200060024000380240B8
:10EE1000A102000848DC0020E058080838B5104D71
:10EE20006C6D24B10F4A64212046F3F7BDFF002129
:10EE30002046F4F731F86368012285F858201A68F3
:10EE4000B2F844306FEA43436FEA53439BB2A2F8EF
:10EE5000443013889BB243F00103138038BD00BFD8
:10EE6000087F0020009F24001D4AF8B5536D73B140
:10EE70005D6892F858206C7906464AB1032C2CD86C
:10EE8000DFE804F0222528022B6840331E60F8BD1D
:10EE90002868144931F81470818989B221EA070180
:10EEA000DF688181D7F808C0DCF8001021F001018B
:10EEB000CCF800101A7403889BB243F0010303805E
:10EEC0003A77FFF7ABFFD9E72B683433DEE72B68DF
:10EED0003833DBE72B683C33D8E700231B60FFDEC9
:10EEE000087F00201052080810B5224C636D83B1D2
:10EEF00094F858206AB194F85C20032A0AD0022AB8
:10EF000010D0002384F85830FFF7B2FE08B984F817
:10EF10005D0010BD5A685379032B27D8DFE803F052
:10EF200023201D185A685379032B1FD8DFE803F0FC
:10EF30000D0A07021368403300221A6010BD1368DF
:10EF40003C33F9E713683833F6E713683433F3E7F3
:10EF50001368403364221A6010BD13683C33F9E72C
:10EF600013683833F6E713683433F3E700231B6084
:10EF7000FFDE00BF087F00202DE9F04FDFF810A36F
:10EF8000C0499AF861809AF860709AF862E083B09C
:10EF90004FF0000C0AF164000AF5197BCDF804C0AB
:10EFA0000122CDF800808378C578C3F1FF039BB2BE
:10EFB0002C46002B00F03281B0F80080B24EC3F135
:10EFC000FF03A6FB089605FB03F376091B12052E2B
:10EFD00000F26381DFE816F01001F400DC00C200EB
:10EFE000A8000600A84EA6FB08E46409C4EB0414BC
:10EFF000A8EB8404A4B2EF1AC4F13C0407FB04F4A8
:10F00000A6FB0464DEB206EB54145FFA84FE2F46BE
:10F010001C462B4601250096F14601951E0246EA44
:10F020000446172446EA09060CEB0408A8EB04037F
:10F0300002FA04F59BB2354203F12A030CBF012505
:10F040000225013C41F82350631CEFD104300CF140
:10F05000180C58451FFA8CFCA5D14FF44063AAF850
:10F0600064328023AAF86632019BDDF800802BB160
:10F070008AF862E08AF861808AF860709AF85D30F8
:10F08000002B4ED0DAF85430002B4AD0EFF3118128
:10F09000102282F312885A68106854797B4A32F839
:10F0A0001440828992B222EA04028281D86885687B
:10F0B00002692C681F2A24F001042C60446840F285
:10F0C000B580203A202000FA02F2E260CAB282F350
:10F0D0001188DA68DAF85400926840F62B415160E2
:10F0E00011680124214311601C7403681A7DA24237
:10F0F00004BF02221A7593F82C100CBF4FF4007253
:10F100000022012900F0AB8093F84410012900F09F
:10F11000928093F85C10012900F0AE80002A40F044
:10F12000B98003B0BDE8F08F574FEE1AA946A7FB90
:10F1300008546409C4EB0414A8EB8404A4B204FBCF
:10F1400006F6A7FB0647DCB204EB5717FFB2012512
:10F150000094CE461C4601953B465FE74A4EEF1AA7
:10F16000A946A6FB08546409C4EB0414A8EB840464
:10F17000A4B2C4F13C0407FB04F4A6FB0464DFB2B0
:10F1800007EB5414E4B201250094CE46019545E7FF
:10F190003D4F0095EE1AA7FB08E56D09C5EB051577
:10F1A000A8EB8505ADB205FB06FEA7FB0E7EDFB220
:10F1B00007EB5E1E5FFA8EFE0125F14601952DE7F5
:10F1C000314E0095A5EB030EA6FB08756D09C5EB46
:10F1D0000515A8EB8507BFB2C7F13C070EFB07F783
:10F1E000A6FB07675FFA83FE0EEB5717FFB299463F
:10F1F000012301933B4611E7EC1A234E08FB04F46C
:10F200005FFA83FEA6FB04640EEB5414E4B2994645
:10F210002F462B46012500940195FFE6AE46A946F0
:10F220002B4600952F4601250195F7E6202000FA90
:10F2300002F2A2604AE7022183F8441093F85C10BE
:10F24000012942F4006217D043681B68002159620B
:10F25000998989B20A439A8103B0BDE8F08F0221EF
:10F2600083F82C1093F84410012942F48062E2D014
:10F2700093F85C100129E7D1022183F85C1042F475
:10F280008052E1E748DC002089888888105208080D
:10F29000087F00204FF40072D6E7009C3B46F14601
:10F2A000BCE600BF2DE9F04FA04FA7B000210A2611
:10F2B0000C4607F51A754FF0050B01968BE0BAF175
:10F2C000000F19D143F04003BEF18C0F87F86C3664
:10F2D00000F2E48004F1010C98340DEB040A0CF107
:10F2E00098040DEB040C74464FF0040E0AF88CECF5
:10F2F0000CF88C3C04F1020EBEF18C0F42F0020CB3
:10F3000000F2CC8004F198036B4403F88BCC04F139
:10F31000040CBCF18C0F03F88CBC00F2BF800EF122
:10F3200098060DEB060E4FF0060A0EF88CAC04EBB7
:10F330000A0E4FEA8909BEF18C0F5FFA89F603F8CD
:10F34000890C00F2AB8004F19C0CEC444FF00709EF
:10F350000CF88C9C04F1080CBCF18C0F03F8876C42
:10F3600000F29C800EF198060DEB060E0EF88CBC98
:10F3700003F8852C04F10A028C2A00F28F8004F134
:10F38000A0060DEB060C0CF88CAC03F8830C04F112
:10F390000C008C2800F2828004F1A20204F1A30385
:10F3A0006A446B4402F88C9C044603F88C8C480930
:10F3B00001F01F0C55F82030012202FA0CF223EA6A
:10F3C000020345F82030019B013B01936ED00131CF
:10F3D000B1F5F07F6AD23C222846F8F7E5FA011E23
:10F3E0005FDB07EB410297F86C36B2F8A4C21CF061
:10F3F000040FC1F30722C8B25FFA8CF94FEA1C2848
:10F4000003F0400A04F1020E7FF459AFBAF1000F85
:10F4100003D103F0380CCC4519D003F0870343EA3D
:10F420000903BEF18C0F87F86C3637D804F1010C54
:10F430000CF1980698346C440DEB060C4FF004095F
:10F4400004F88C9C74460CF88C3C0EF1020EBEF154
:10F450008C0F23D804F198030DEB030C231D8C2B88
:10F460000CF88B2C0CF88CBC18D80EF198020DEB14
:10F47000020E06220EF88C2C0CF8890CA0188C2891
:10F480000CD804F19C0304F19D026B446A440724E8
:10F4900003F88C4C044602F88C8C88E76FF000442B
:10F4A00085E7204614B927B0BDE8F08FD7F8645639
:10F4B0001F4995F91030AA6803EB8303920751F8AE
:10F4C000230020D5234603AA002171F0B1FDAB68CB
:10F4D0009B0701D50120E6E7164B17491A68174B21
:10F4E0004FF4FA7000FB02F2A3FB02324868920963
:10F4F0004B681B1A9A42FBD26B69002BEAD01A6840
:10F500009B881383E6E76B6913B11A689B88538362
:10F51000084B09491A68094B4E68D200A3FB023216
:10F5200092094B689B1B9A42FBD2CBE7087F0020D5
:10F53000C01500205C3B0020001000E0D34D62109D
:10F54000F0B5284CD4F8640683B010B194F86A364C
:10F550000BB103B0F0BD01230DF10702842184F843
:10F560006A36FCF743F994F86C26D4F86406042153
:10F570000A43FAF7F3F8D4F864060DF10702842180
:10F58000FCF734F99DF8073013F00406F3D1164D5B
:10F5900084F86C363C223146284675F02FFC324602
:10F5A000124E05F13A0005F2FA374FF0010E30F82D
:10F5B000023F334002F01F019BB24FEA521C0EFA89
:10F5C00001F1013223B155F82C300B4345F82C30B2
:10F5D000B842ECD1FFF766FE0028FBD184F86A063A
:10F5E00003B0F0BD087F00207081002004DFFFFF22
:10F5F00070B5404DD5F8644682B08CB395F8683646
:10F60000012B41D0022B2DD1082294F910303A4918
:10F6100085F86B2603EB830300208DF8040051F876
:10F620002300A3688DF8052040F20442ADF80620BF
:10F630009A0742D504230DEB0302002171F0F8FC78
:10F64000A3689B0722D52D483C22FF2175F0D6FBED
:10F6500095F8693623B9FFF773FF012385F86936FA
:10F6600002B070BD0DF10302A0212046FCF7BEF8E8
:10F670009DF8033003F00503012B37D0002B2FD169
:10F68000D5F864460822C0E74822BEE71C4B1D4956
:10F690001A681D4B48684FF4FA7606FB02F2A3FB8A
:10F6A000023292094B681B1A9A42FBD26369002B03
:10F6B000C9D01A689B881383C5E7636913B11A68B8
:10F6C0009B8853830E4B0F491A680F4B4E68D2002C
:10F6D000A3FB023292094B689B1B9A42FBD2A9E71B
:10F6E0000A4A126840F2DC539A42B9D9D5F8644606
:10F6F00048228AE7087F0020C01500207081002082
:10F700005C3B0020001000E0D34D6210EC2800208C
:10F710002DE9F041334D95F86A3682B003B1FEE72A
:10F72000012285F86A2695F86B26044602F0F70256
:10F73000D5F8640685F86B260E461946FAF70EF8DA
:10F74000E2B207460921D5F86406FAF707F8B4F5DE
:10F75000807F3FD0D5F86406DFF88C8050220821E6
:10F76000F9F7FCFFD5F864060DF10702A021FCF7BC
:10F770003DF848B9D8F8D830B8F8DC2059690A42C1
:10F7800014BF5A831A83EDE79DF8074014F0200454
:10F79000F0D1E2B20A21D5F86406F9F7DFFF321999
:10F7A000D5F86406C0210134FCF720F8362CF0D1DE
:10F7B00057B995F86B26D5F8640602F0F70239467A
:10F7C00085F86B26F9F7CAFF002385F86A3602B080
:10F7D000BDE8F081D5F8640640220A21F9F7BEFFA2
:10F7E000B8E700BF087F0020A43800202DE9F04FC3
:10F7F0005F4D95F86A76C3B007B1FEE795F86B26C2
:10F80000044602F0F7020123D5F8640685F86B265A
:10F810000E46394685F86A36F9F7A0FFFF2C4FF0FF
:10F8200009038DF8054088BFA40801AA8CBF04F025
:10F83000C008B84602204FF0000C4FF00A0B0DF143
:10F84000050A4FF00B09137014E0B1F5827F02F83E
:10F8500000B00AF8003016F80C3017D80CF1010C83
:10F86000BCF1360F02F8079004F1060402F80E30DE
:10F87000084614D0871C48EA0C03B7F5827F00F1D4
:10F8800004010446DBB200F1030EDED90CF1010CD9
:10F890006FF00041BCF1360F364C0846EAD1B4F5A2
:10F8A000827F61D8082353540DF10503A021195418
:10F8B000831CD5F86446304894F9101001EB81019F
:10F8C00050F82100A168890722D5002171F0B0FB12
:10F8D000A3689B0731D5294CD5F864060DF10302C6
:10F8E000A021FBF783FF48B9D4F8D830B4F8DC2066
:10F8F00059690A4214BF5A831A83EDE79DF8033011
:10F9000013F02003F0D185F86A3643B0BDE8F08FDC
:10F91000616911B10E68898871831949194F0E68A0
:10F920001949D7F804C0F600A1FB0616B609796894
:10F93000A1EB0C018E42FAD2C7E7114B11491A68AC
:10F94000114B48684FF4FA7606FB02F2A3FB023231
:10F9500092094B681B1A9A42FBD26369002BBAD0FA
:10F960001A689B881383B6E76FF00043A1E700BFD6
:10F97000087F002001000080C0150020A43800206E
:10F980005C3B0020001000E0D34D6210002ABCBF99
:10F9900080185242002B30B503EB010503DA0C4608
:10F9A0005B42294625460028B7BF121A8418144620
:10F9B0000020A4F11D0C0029BCBF2B460021BCF186
:10F9C000000FC4BFA2EB0C021418A5F10F02002A0D
:10F9D000C4BF9B1A5D1884421EDBC1F1010C0F4AA3
:10F9E000AC44C1EB0113CCEB0C1C00EB4303013422
:10F9F0004FEA4C0C02EB43024FF0200E8D42A8BFA1
:10FA0000002304DB22F813E01E339C45FAD10130B9
:10FA1000A04202F10202F1D130BD00BFAC81002052
:10FA20001B4B1C48196C1C4A10B441F08051012436
:10FA3000196404625321FF24CA2054625062516247
:10FA40005B6FDB0085B013D400231449029302914D
:10FA5000029A134804320292029A136003930391AC
:10FA6000039B0393039B186005B05DF8044B70473C
:10FA70000A4B002201920193019B0193019A084BCA
:10FA800012689A42E0D105B05DF8044B704700BFA0
:10FA90000038024000000E4200280040502800407C
:10FAA00076614E6970B50546BDF8106001600C4680
:10FAB00019B119462046F3F777F931462046F3F796
:10FAC000EBF961680B68B3F844206FEA42426FEAD1
:10FAD000524292B2A3F844201A8892B242F0010234
:10FAE0001A804A79032A17D8DFE802F0110C0702BE
:10FAF00040330022AB601A6070BD3C330022AB6023
:10FB00001A6070BD38330022AB601A6070BD3433A8
:10FB10000022AB601A6070BD0023AB601B60FFDE8B
:10FB20002DE9F04F85B00646BDF838B09DF83CA0F1
:10FB3000894617469846F3F7E7F8002857D02D4C2A
:10FB400094F870360A2B4DD803EB430204EB4212B3
:10FB500002900020C2F8740682F878065A1CD2B2CD
:10FB600084F8702603EB43033079039204F2746443
:10FB700004EB4314FDF792FC0299054618B3039A6F
:10FB8000027280F806900220E87143463A46CDF8AA
:10FB900000B02046FFF786FFBAF1000F0AD111210D
:10FBA0002846FDF71BFC2B68AA885A83204605B01F
:10FBB000BDE8F08F2846327A0221FDF733FC20465B
:10FBC00005B0BDE8F08FCDF800B043463A46204678
:10FBD000FFF768FFBAF1000FECD111215046FDF795
:10FBE000FDFBE3E7044A00210420F8F7FFFB0024B3
:10FBF000DCE700BF087F002040FF080830B503683D
:10FC0000284D294C2DED028BAB42246883B0F0EED9
:10FC1000408AB0EE608A10D005F58065AB420CD00A
:10FC200005F57055AB4208D005F58065AB4204D0B0
:10FC300005F58065AB4218BF6408B4FBF1F303F52A
:10FC40007F43FF331B0CB4FBF3F40023B4FBF1F54B
:10FC5000019200932246ABB20221FFF761FFE0B1AF
:10FC6000B5EE408A07EE904AF1EE10FAF8EE677AA8
:10FC70000ABF07EE105A28EE278AB8EE478A9FED92
:10FC80000B7AC8EE076A0123037127EE667AC0ED8E
:10FC9000046AA8EEA77A80ED037A03B0BDEC028B6C
:10FCA00030BD00BF00000140E809002000007A4498
:10FCB0002DE9F04F2DED028BAA4BAB4E1B78AB4DCF
:10FCC000DFF8CCA2B5B000270293B046B146BB46E0
:10FCD000D9F80040002355F83320944203D0013373
:10FCE0000E2BF8D1FF23534493F8943A022B00F0E3
:10FCF000BB80032B00F0AF80012B09D1D9F80C3069
:10FD000023F0807323F0080343F00403C9F80C3098
:10FD10004846FDF793FF48B90BEB8B0308EB8303D1
:10FD2000D96801F00C03042B00F0A9800BF1010B42
:10FD3000BBF10C0F09F11409CAD18D4DDDF8088013
:10FD4000A5F1F00408E02068E260FEF70BF84844F3
:10FD5000C7B21434A5421FD02046FDF76FFF00281C
:10FD6000F7D1E368590703F00C02F2D5042AF0D06A
:10FD700023F0080242F00402781C474511465FFA5E
:10FD800080F923F00403DED32068E36019461434BD
:10FD9000FDF7E8FFA542DFD10025764FDFF8F491AB
:10FDA0002C46A846AB463046FDF748FF002840F0F9
:10FDB000A880F06842076AD5029B57F80C2C43458F
:10FDC00000F2A680030764D4002D57F80C3C40F3E2
:10FDD000BD8028A900229C4602E0AA4200F0B5801E
:10FDE00051F8043F1B689C4502F10102F5D1C201A4
:10FDF00064D40BF1010BBBF10C0F06F1140607F1F3
:10FE00001407D0D1574B93F800E0BEF10C0F00F36C
:10FE10001082594B594A1B791370032B40F2BC8056
:10FE20001A1F022A00F27982052B00F06782062B46
:10FE30000CBF4FF47A564FF47A665149514800226C
:10FE40004A600027504AB2FBF6F200260A60C0E979
:10FE500000674E4AA1E0D9F80C3023F00C0343F0C0
:10FE60008073C9F80C3053E7D9F80C3023F0807355
:10FE700023F0040343F00803C9F80C3048E7204698
:10FE8000FDF770FF0137FFB20744FFB24EE70207EC
:10FE9000ADD5002C57F80C3C4BDD1DA900229C462B
:10FEA00001E0A24244D051F8043F1B689C4502F196
:10FEB0000102F6D1410787D4C2019AD5002C57F828
:10FEC0000C3C0ADD1DA9002251F8040F0068834292
:10FED00002F101028DD0A242F6D1002D0ADD28A93F
:10FEE000002251F8040F0068834202F1010280D021
:10FEF000AA42F6D14FF080711846F160FDF732FF4B
:10FF000077E75B464A4601210420F8F76FFA70E76D
:10FF100020F00801F1601046FDF724FFF06808F1B9
:10FF2000010803075FFA88F8B3D44107C4D54BE74B
:10FF30006346184634AB03EB85020821F16042F8B2
:10FF40002C6C0135FDF70EFF53E76346184634ABC2
:10FF500003EB84020421F16042F8586C0134FDF790
:10FF600001FF46E7AC000010581600206C5208084C
:10FF7000481700206416002028610020145F00202C
:10FF8000205F0020285F002040420F00A1DD000814
:10FF9000087F00207CFF0808B84ACAF8A42AB84A9B
:10FFA00012F81330002B00F0B281A64500F3B781A0
:10FFB000BEF1000F00F0A6809FEDB28ADFF820B3FB
:10FFC000DFF8148304951DAC4FF000097746AE4B63
:10FFD000DBF800201B7854F8046FC2F30072062B84
:10FFE00000F23C81DFE803F0B5ABA1790404040022
:10FFF000052B00F07781A549A548062B18BF0146BF
:020000040801F1
:100000000025019200950A46142302213046FFF78D
:1000100087FD0290002800F021819E4B31681A78FC
:10002000002A00F01281CDF80C8003E001359542E2
:1000300000F00D812B0158F803309942F6D1EAB255
:10004000082A00F00B810298934B016805910D6816
:100050004E6807954FF4907101FB0231039BC16517
:1000600003EB02130691996013016A6E08933568D9
:10007000002A00F05881B5F8443088486FEA4343BD
:100080006FEA53439BB2A5F844302B889BB243F0F0
:1000900080032B80737909931946B379405C298CCE
:1000A0005B074CBF0423012383409BB289B221EA42
:1000B00003012984298C89B20B432B842B889BB2A2
:1000C00043F001032B80002A00F05B81029A012398
:1000D0001371734B43F839200EE0DFED720A724B57
:1000E000B0EE600A59883046FFF788FD6C4B43F844
:1000F0003900002800F0A28109F101094F457FF481
:1001000066AF049D694C94F8B03263BB684A022123
:100110000420F8F76BF99AF8A20AB0FA80F04009C7
:1001200035B0BDEC028BBDE8F08FDFED620A9FEDCC
:10013000620A30464FF4FA61FFF760FDD6E7DFED63
:100140005F0A3046B0EE600A4FF47A71FFF756FD51
:10015000CCE79FED4C0AF0EE480A30464FF4C871E8
:10016000FFF74CFDC2E794F8B19294F8B23209F16E
:100170000109A9EB0309B9F1120F0BDD12230221CA
:1001800000934F4A8AF8A21A4B4600210420F8F740
:100190002DF9C0E794F8BC32012B00F0B480022B9B
:1001A00040F0A2806BF094FA464BC4F8C03294F849
:1001B000BC32002B00F0A580022B40F09980122D5C
:1001C0002B46B8BF12239BB24B45C0F2D080A94545
:1001D000A8BFA946B9F1000F9DDD3B4FDFF800B184
:1001E000DFF8E88028AE002504E001354D4547F8EA
:1001F000040B90D0DBF80030B4F8B412C3F30072F3
:10020000B4F8B63201920091B8FBF3F32F4A56F8D6
:10021000040F9BB20321FFF783FC0028E5D10524DE
:1002200001462B4A8AF8A24A2B460420F8F7DEF84A
:1002300071E7284ACDF800B001218AF8A21A734666
:1002400000210420F8F7D2F85CE7234B0393130155
:100250000398C1500F49531C0B70F1E6104A049DDE
:10026000002342F8393005218AF8A21A1B4A4B466E
:1002700000210420F8F7BAF844E700BF4DE9000870
:10028000085308086F12833A145F0020001BB70060
:10029000C0C62D00605F0020B0890020E05808082B
:1002A000645F002000000000286100200090002012
:1002B00044000908ACC5A737ACC5A7366F1203398F
:1002C00060000908B9DD0008586E002040420F00A8
:1002D0000001090894FF0808C45F00201C000908F9
:1002E000B400001056498BE6564AC4F8C02243B108
:1002F000554A02210420F8F779F80CE74FF4FA5632
:100300009BE52B465FE76BF0E3F9504B4DE7504A16
:1003100002210420F8F76AF8F4E64E4A3DE64E4A18
:100320000094032189E7D6F810C04C49099213467E
:100330004FEA431E01EB431051F80E208CEA020EE7
:100340001EF47C5F03F1010309D0102BF0D1059A54
:100350000023D360424B029A43F83920CCE6059B38
:10036000099AD860037F002B3FF485AEF2E70420A2
:1003700000953C4A8AF8A20A4B460021F8F736F865
:10038000C9E6059B3849DB680A931A46374B526821
:100390000A989A42364A136B0CBF43F4001343F495
:1003A00080031363072383830322059BF2F7D8FF9F
:1003B0000A9880680B90F3F7DFF9069A337C0F9266
:1003C0002C4A0B98069002EB83034FF480465B683F
:1003D0000D93036823F0010303600023CDE9183374
:1003E000CDE91A3312931693122311934FF48063BD
:1003F00013934FF48053CDE9143640234C351093BA
:100400000DA94FF400330E95179369F02DFE069851
:10041000089D039A03680A992A44079D43F0100334
:1004200003606966144B099933F81130A5F86830F8
:1004300093815060059A0123137447E6049D12E7E7
:10044000808D5B00D5DD00088C0009080568030875
:10045000C0FF08089DDD0008E0FF0808EC09002047
:10046000645F0020C8000908A10200080060024083
:1004700000380240E05808081052080810B5104C27
:10048000D4E90423A16882B002FB03F38B428DF808
:10049000070012D06368E0680DF10701184474F09A
:1004A00069FC63682269A16813446269B3FBF1F0D7
:1004B000013201FB10336360626102B010BD00BF06
:1004C000385F00202DE9F043674B06461C7820B3C7
:1004D0001CB30021654D07200F4602E001318C421C
:1004E0001BD055F83130002BF8D01A79002AF5D0FE
:1004F000D3F800C0DA6DDCF804305B7902EB8302DC
:10050000002342F823000433402BFAD101318C42FE
:10051000C2F80071C2F81071E3D1554F3B78F3B1C6
:10052000DFF850C151484FF0000E002C6ED0002370
:1005300050F8332001334AB1117939B112682AB128
:100540005568DCF800102D688D420AD09C42EFD12E
:100550003B780EF1010E73450CF1100CE7DCBDE8A1
:10056000F083D368002B51D09B68002B4ED0EFF363
:100570001188102383F31288DCF80010BCF80C50AB
:100580008B899BB223EA05038B81DCF804100B688E
:1005900023F001030B600B68DB070AD542F21073EE
:1005A00001E0013B05D000BFDCF804100D68ED0749
:1005B000F7D40B68DB075FFA88F841D4D5682B695C
:1005C0006D681F2B2BD9203B4FF0200909FA03F34C
:1005D000EB600B685EB343F480730B6048234B60A1
:1005E0000B6823F010030B6003231374BFF34F8FCA
:1005F000DCE900210B6843F001030B609189BCF832
:100600000C300B439BB2938188F311883B780EF139
:10061000010E9E450CF1100C87DBBDE8F0834FF016
:10062000200909FA03F3AB600B68002ED3D123F441
:1006300080730B600B6843F010030B601674D5E7F2
:10064000DCF80020BCF80C3091890B439BB29381FD
:1006500088F311883B780EF1010E9E450CF1100CC9
:10066000FFF663AFD9E700BFAC000010645F002065
:10067000605F0020C45F002010B50379012B84B0B7
:100680000C4627D0022B23D18368DB070DF10F0224
:100690004CBF01218121FBF757F89DF80F30002254
:1006A000C3F3001161F30702C3F3800161F30F226A
:1006B0000F49C3F3C00C6CF3174281F8F000C3F389
:1006C000801161F31F62DB092260237104B010BD49
:1006D0000020E2E782680DF10F0102F00102CDE98E
:1006E00000121A46417C90F91000F3F7E7FED4E7B8
:1006F000581600202DE9F04182B014460E4601AA9A
:1007000050210546FBF772F89DF80430DFF8F080C1
:10071000394F01335B00DBB24621238001AA284612
:10072000FBF764F823789DF8042008FB03F303F536
:10073000FA73A7FB031301329909DB0902FB0133AA
:10074000A280A7FB03239B0901AAE3605121022396
:100750002846FAF7F9F82378BDF8040008FB03F3FC
:1007600040BA03F5FA73A7FB0323C2B2C0F3072014
:100770008240013292B29809DB0902FB0033A7FBE9
:1007800003739B097021E280238201AA2846FBF7AC
:100790002DF89DF8043001335B00DBB201AA6380C1
:1007A000712102232846FAF7CFF8BDF80430134A26
:1007B000F17882F8F0005BBADAB2C3F307239A400B
:1007C000013292B2228119B1E388D21A92B2228107
:1007D0000B48A378084900FB03F303F5FA73A1FB68
:1007E00003039809DB0902FB0033A1FB03139B09F8
:1007F000638202B0BDE8F081D34D6210581600202C
:10080000002F3A002DE9F047DFF89882DFF8989240
:10081000A34F8CB0054600264FF4FA7307AA89212E
:100820000068C8F8A43188F89060FAF7DFFF9DF8F7
:100830001C20286842F001028921F8F78FFF324618
:1008400088212868F8F78AFF012280212868F8F7B4
:1008500085FF0122FF212868F8F780FF32463146E4
:100860002868F8F77BFF07AA91212868FAF7BEFFEE
:100870009DF81C30286888F89E3131460122F8F72F
:100880006DFF3246FF212868F8F768FF3246802165
:100890002868F8F763FF07AA60212868FAF7A6FF1F
:1008A0009DF81C20286842F012026021F8F756FFDC
:1008B0004FF40053ADF81C3007AA022344212868E6
:1008C000F9F7C8FFFF2201212868F8F747FF2C68D5
:1008D000012280212046F8F741FF0122FF21204616
:1008E000F8F73CFF324631462046F8F737FF06223C
:1008F000FF212046F8F732FF07AA83212046FAF7A6
:1009000075FF9DF81C20832142F004022046F8F771
:1009100025FF0722FF212046F8F720FF0122812131
:100920002046F8F71BFF012280212046F8F716FF2A
:100930006B2294212046F8F711FF3246832120468E
:10094000F8F70CFFD9F80060C8F8A0612379012BF3
:1009500000F09880022B0FD000209DF81C3087F803
:10096000F000DBB9D9F800309BB29B1BB3F5FA7FDE
:10097000ECD90CB0BDE8F087A368DB0707AA4FF0FD
:10098000830120465EBF07AA83212046FAF7DCFEDA
:100990009DF81C3087F8F000002BE3D00122832162
:1009A0002046F8F7DBFE07AA92212046FAF71EFF41
:1009B0000022812120469DF81CA0F8F7CFFE0622D8
:1009C000FF212046F8F7CAFE07AA83212046FAF73E
:1009D0000DFF9DF81C20832102F0FB022046F8F752
:1009E000BDFE0122FF212046F8F7B8FE01220021BA
:1009F0002046F8F7B3FE0022FF212046F8F7AEFEAE
:100A0000204600228021F8F7A9FE0623B02105AA7E
:100A10002868F9F799FF0122FF212868F8F79EFE60
:100A200000224F212868F8F799FE2C224E212868D1
:100A3000F8F794FE0022FF212868F8F78FFE4FEAAE
:100A4000DA162868B422B621F8F788FE0024002EB2
:100A500018BF0C260AF07F0AA1464FF0010EC4F31E
:100A6000C40330336B44E2B213F81C0C04F0070CDF
:100A70000EFA0CF1964220EA010117D903F81C1C6A
:100A80000134ECE7A268617C94F9100002F00102E5
:100A9000019207AA00928322F3F710FD5DE700BFE1
:100AA00058160020106E0020EC280020D14540FA96
:100AB0000CF200F01283D30744BF09F101095FFA79
:100AC00089F90134302CCAD1062305AAB02128683F
:100AD000F9F7C0FE0122FF212868F8F73FFE002247
:100AE00011462868F8F73AFE0022FF212868F8F737
:100AF00035FE002209212868F8F730FE0022102177
:100B00002868F8F72BFE002211212868F8F726FE46
:100B1000012224212868F8F721FEFF2225212868D8
:100B2000F8F71CFE002275212868F8F717FE01224D
:100B3000FF212868F8F712FE2C224E212868F8F7CA
:100B40000DFE002248212868F8F708FE21462022E1
:100B50002868F8F703FE0022FF212868F8F7FEFD59
:100B6000214609222868F8F7F9FD00225421286857
:100B7000F8F7F4FD042231212868F8F7EFFD03228D
:100B800032212868F8F7EAFD832240212868F8F727
:100B9000E5FD252246212868F8F7E0FD00226021C6
:100BA0002868F8F7DBFD002227212868F8F7D6FD32
:100BB000062250212868F8F7D1FD0022512128682B
:100BC000F8F7CCFD962252212868F8F7C7FD0822D5
:100BD00056212868F8F7C2FD224657212868F8F701
:100BE000BDFD002261212868F8F7B8FD00226221CE
:100BF0002868F8F7B3FD002264212868F8F7AEFDF5
:100C0000002265212868F8F7A9FDA022662128683E
:100C1000F8F7A4FD0122FF212868F8F79FFD322292
:100C200022212868F8F79AFD142247212868F8F74E
:100C300095FDFF2249212868F8F790FD00224A21FE
:100C40002868F8F78BFD0022FF212868F8F786FD59
:100C50000A227A212868F8F781FD00227B21286882
:100C6000F8F77CFD212278212868F8F777FD01222A
:100C7000FF212868F8F772FD342223212868F8F74D
:100C80006DFD002242212868F8F768FDFF2244210B
:100C90002868F8F763FD262245212868F8F75EFDED
:100CA000052246212868F8F759FD40221146286898
:100CB000F8F754FD06220E212868F8F74FFD1A2296
:100CC00020212868F8F74AFD402243212868F8F7D8
:100CD00045FD0022FF212868F8F740FD032234215A
:100CE0002868F8F73BFD442235212868F8F736FDDF
:100CF0000122FF212868F8F731FD042231212868FC
:100D0000F8F72CFD09224B212868F8F727FD05226A
:100D10004C212868F8F722FD04224D212868F8F7B5
:100D20001DFD0022FF212868F8F718FD002244214C
:100D30002868F8F713FD202245212868F8F70EFDF2
:100D4000082247212868F8F709FD28224821286849
:100D5000F8F704FD002267212868F8F7FFFC042259
:100D600070212868F8F7FAFC012271212868F8F749
:100D7000F5FCFE2272212868F8F7F0FC00227621AB
:100D80002868F8F7EBFC002277212868F8F7E6FCE2
:100D90000122FF212868F8F7E1FC01220D212868D3
:100DA000F8F7DCFC0022FF212868F8F7D7FC0122C5
:100DB00080212868F8F7D2FCF82201212868F8F78A
:100DC000CDFC0122FF212868F8F7C8FC01228E2102
:100DD0002868F8F7C3FC012200212868F8F7BEFC58
:100DE0000022FF212868F8F7B9FC0022802128683A
:100DF000F8F7B4FC04220A212868F8F7AFFC2C6845
:100E000007AA84212046FAF7F1FC9DF81C20204611
:100E100002F0EF028421F8F7A1FC01220B212868DF
:100E2000F8F79CFC2C6803A92046FFF725FC07AACD
:100E300003A92046FFF75EFC9DF80C30002B00F064
:100E40005D810A9C04F684549DF80E30002B00F05E
:100E50004B810A9B03F2B22304EB43049DF80F304D
:100E600023B1BDF82C3003F525731C449DF81030D8
:100E700023B1BDF82E3003F226231C44A44E28686B
:100E8000C6F8C442E8220121F8F768FC2868214628
:100E90006FF0F0F8012211462868F8F75FFC402156
:100EA00087F8F0002868FDF76BFD00283FF461AD7E
:100EB000012128680222F8F751FC002187F8F00090
:100EC0002868FDF75DFD00283FF453ADE8220121BD
:100ED0002868F8F743FC4FF4005307AAADF81C301C
:100EE000442102232868F9F7B5FC2C6803A92046A1
:100EF000FFF7C2FB07AA03A92046FFF7FBFB50221E
:100F000057212046F8F72AFC082256212046F8F7F8
:100F100025FC082250212046F8F720FCBDF82C20A3
:100F20004FF47A7148F20E6301FB0233794A93421F
:100F300040F2EB80784AA2FB0332120C013AFF2AFE
:100F40004FF0000306DD52080133FF2A9BB2FAD8A6
:100F50001B029BB21343C3F30722DBB28DF80820B8
:100F60008DF8093002AA022351212046F9F772FCBC
:100F70000A9A4FF47A7148F20E6301FB0233674A12
:100F8000934200F2C080644AA2FB0332120C013A81
:100F9000D2B246212046F8F7E1FB2046D6F8C4122B
:100FA0006FF068F802AA01212046FAF71FFC02221E
:100FB0009DF8089001212046F8F7D0FB002120463B
:100FC000FDF7DEFC4A4620460121F8F7C7FB2C68F6
:100FD00003A92046FFF750FB07AA03A92046FFF705
:100FE00089FB482211462046F8F7B8FB0822472122
:100FF0002046F8F7B3FB032232212046F8F7AEFB78
:10100000072230212046F8F7A9FB0122FF212046C4
:10101000F8F7A4FB202230212046F8F79FFB00229E
:10102000FF212046F8F79AFB062270212046F8F7A8
:1010300095FBBDF82E103A4A4FF47A7046F64403F9
:1010400000FB0133A2FB03239DF80F201B0B1AB1F9
:10105000BDF8222013449BB2002B52D05A1EFF2A07
:101060004FF0000306DD52080133FF2A9BB2FAD885
:101070001B029BB21343C3F30722DBB28DF8082097
:101080008DF8093002AA022371212046F9F7E2FB0C
:10109000D6F8C41220466EF0EDFF02AA01212046C8
:1010A000FAF7A4FB9DF80850022201212046F8F728
:1010B00055FB00212046FDF763FC2A46012120460E
:1010C000F8F74CFB6422012387F8F000C8F8A4214C
:1010D00088F890300CB0BDE8F0870EFA0CFC20EADE
:1010E0000C0003F81C0CECE49DF80D30002B3FF4D1
:1010F000B5AE0A9B03F525731C44AFE640F63634C3
:10110000A2E61A46BAE7FF2243E700231A4625E77C
:10111000009000201B0C0100950370F41B280D01AA
:101120004963A41310B5194C84F89510017952BA8B
:10113000A4F8962001294FF0000282B084F8942090
:1011400016D0022903D06FF00C0002B010BD8368E6
:1011500013F0010F04F194024FF0040314BFFF21B8
:101160007F21F9F71FFB0028EDD0002002B010BD51
:101170008268417C90F91000943402F00102CDE9BC
:1011800000420423FF22F3F765F9ECE7106E00201C
:101190002DE9F04F9D4F9E4D06683C464FF00008EC
:1011A00085B0834685F894815B37C4F12D0905F13C
:1011B000940A13E0022B0FD1B26812F0010F4FF026
:1011C000030352464FF0FF01304601BF032352464E
:1011D0007F213046F9F7E6FAA7421AD0337985F82D
:1011E000948009EB0401012B14F8012F85F8951068
:1011F00085F89620DED1B368717C96F9100003F073
:101200000103CDE900A3FF220323F3F723F9A7424B
:10121000E4D14FF40743A5F89430402385F8963085
:1012200052460323FF213046F9F714FB00238DF8C3
:101230000E300DF10E0130466EF0E6FE9DF80E30D8
:10124000002BF6D04FF40643A5F894300123714AE1
:1012500085F89630FF2103233046F9F7FBFA4FF467
:1012600007436C4AA5F8943000240323FF2130463D
:1012700085F89640F9F7EEFA4FF40063A5F894303C
:101280000923644A85F89630FF2103233046F9F795
:10129000E1FA4FF43063A5F894305E4A85F8964041
:1012A00030460323FF21F9F7D5FA002800F0AC807F
:1012B000DBF800400DF10E025E212046FCF7B6FD82
:1012C000BDF80E30B3F5D77F00F08C806AD8512B73
:1012D00000F0848078D81D2B7ED10F2608BB0A220F
:1012E0004B212046FDF7B0FB0F2260212046FDF781
:1012F000ABFB0D2263212046FDF7A6FBB822692136
:101300002046FDF7A1FB40F60D7278212046FFF73D
:1013100009FF40F60E627A212046FFF703FF0028FE
:101320006DD0DBF8000021216EF0C4FDDBF8004039
:101330000DF10E02DE212046FCF778FDBDF80E30DF
:101340009FED357AC3F3090303EB8303DB0007EE5C
:10135000903AF8EEE77A4FF4D84267EE877AA5F82C
:101360009420FCEEE77A524617EE903A1BBAC5F885
:101370009630FF2106232046F9F76CFA4FF4074117
:101380004023DBF80000A5F8941085F8963052460B
:101390000323FF21F9F75EFAB0B385F8940105B095
:1013A000BDE8F08F40F2E132934219D01CD840F2F0
:1013B000D922934214D040F2E122934202D0B3F5F5
:1013C000E67FAED1642689E7AD2B0BD0D62B01D0BA
:1013D000602BA6D1212681E71E2BA2D114267DE702
:1013E000C8267BE7322679E740F28F42934203D04A
:1013F00040F29152934294D14FF4FA766EE731461F
:1014000020466EF057FD8CE70020C6E70359080818
:10141000106E0020A46E00209A99893F03682DE980
:10142000F0411F6A1FB13B46BDE8F0411847002A52
:10143000164611DD04460D460E4400E023689B6805
:10144000204698470028F9D0236815F8011B1B682F
:1014500020469847B542F1D1BDE8F081DEE700BFF4
:10146000204A214B116893F8D222C90603D5B3F85C
:10147000D412490715D4F2B993F80423D3F80033F2
:1014800052B143B120B11A689B88138370473BB3B4
:101490001A689B885383704780F00100002BF1D1BC
:1014A000F9E7B2B993F80423D3F80033002AEED158
:1014B000002BE8D17047D3F8F822002AEBD058B1BE
:1014C0009268B3F8FC12094BB3FBF1F35B101360A5
:1014D0007047D3F8F82222B1936800221A6070474F
:1014E00070477047B00000100090002040420F008D
:1014F000BFF34F8F0549064BCA6802F4E0621343FD
:10150000CB60BFF34F8F00BFFDE700BF00ED00E0F1
:101510000400FA0508B572B600224FF0FF319300BF
:1015200003F1604303F561430132082AC3F88010D8
:10153000C3F88011F3D1FFF7DBFF00BF00B583B024
:101540000D49002200920091009B04330093009B00
:101550001B68012B02D003B05DF804FB01920191DE
:10156000019B064904330193019B1A600B6883F3C6
:1015700008884B689847FEE7502800400000FF1F8E
:1015800010B4EFF31183102282F31288094C0A4839
:1015900022684FF0E021013222608A69C0F80823F6
:1015A0000022C0F80C230A69DBB283F311885DF8CE
:1015B000044B7047EC2800200090002030B4EFF37B
:1015C0001182102383F312884FF0E023D2B299697D
:1015D000186910F4803F0D481EBF0121C0F80C139C
:1015E00099690B4B1D68D0F80C3382F311880948B8
:1015F00004684FF47A7202FB04F02B44401A002175
:10160000B0FBF4F030BCE3FB020170470090002017
:10161000EC2800205C3B0020124B5B68C3F30803FE
:10162000FBB9EFF31183E3B930B40F4A0F4C4FF01D
:10163000E02C1368DCF8180011688B42F9D1D4F85B
:1016400008138842F5D80A4A15684FF47A7404FBE7
:1016500005F20021101AB0FBF5F0E3FB040130BCE9
:101660007047ABE700ED00E0EC2800200090002080
:101670005C3B002090B170B5461EFFF7CDFF0446DD
:101680000D46FFF7C9FF001B61EB0501B0F57A7F3E
:1016900071F10001F5D3013EEFD270BD704700BF7C
:1016A00070B5006801220921F8F758F86426FFF7A1
:1016B000B3FF04460D46FFF7AFFF001B61EB0501CA
:1016C000B0F57A7F71F10001F5D3013EEFD170BD25
:1016D0002DE9804883B0431C0193DFF844810A233D
:1016E0000093D8F89C10D8F8D830B8F8A000B8F813
:1016F000DC20DDF804B048834FF0320A1A834FF043
:101700000509D8F89C30B8F8A02059690A4214BFDE
:101710005A831A83D8F8D830B8F8DC2059690A42BD
:1017200014BF5A831A830120FFF79AFE5646574684
:10173000FFF772FF04460D46FFF76EFF001B61EBDB
:101740000501B0F57A7F71F10001F5D3013FEFD1CA
:10175000D8F89C30B8F8A02059690A4214BF5A83BF
:101760001A83D8F8D830B8F8DC2059690A4214BF77
:101770005A831A830020FFF773FEFFF74DFF0446DC
:101780000D46FFF749FF001B61EB0501B0F57A7FBD
:1017900071F10001F5D3013EEFD1B9F1000F1CD07A
:1017A000B9F10109ADD14FF4FA76FFF735FF0446E0
:1017B0000D46FFF731FF001B61EB0501B0F57A7FA5
:1017C00071F10001F5D3013EEFD14FF0FA0ABBF100
:1017D000000F07D04FF0000993E70BF1FF3BBBF17F
:1017E000000FF7D14FF47A76FFF716FF04460D4647
:1017F000FFF712FF001B61EB0501B0F57A7F71F175
:101800000001F5D3013EEFD1009B013B00937FF433
:1018100068AF01210846F2F7DFFFFFF77BFE00BF4C
:10182000A438002018B103685B6903B118477047FA
:1018300018B103681B6A03B118470020704700BF46
:1018400038B50B4D0C4620B10368DB6A0BB19847E5
:1018500060B90020C4E90000C4E90200C4E90655EB
:101860002D2230232061227584F8203038BD00BF3E
:10187000C46109080178F9B1F8B5104F0546002692
:1018800002E015F8011FB1B1D7F81043637A5A1C72
:101890002344D2B262729972237A9342F1D804F14E
:1018A0000A01002AEDD0D4E900309847667215F895
:1018B000011F0029E8D1F8BD704700BF009000204B
:1018C00070B5124C05460E461148FFF7D3FF2A4665
:1018D0001049D4F81003334668F0FAFCD4F81053DA
:1018E0006A7A32B12B68686805F10A0198470023CB
:1018F0006B7294F814333BB194F8163301221344FD
:1019000084F8152384F8163370BD00BF00900020C2
:10191000280109082DE1000870B50C48FFF7AAFF5F
:101920000B4BB3F8186316B970BD013EFCD0FFF73E
:1019300073FE04460D46FFF76FFE001B61EB0501C9
:10194000B0F57A7F71F10001F5D3EEE7780309086D
:101950000090002070B504460F48FFF78BFF20462B
:10196000FFF788FF0D48FFF785FF0D4BB3F81863AD
:1019700016B970BD013EFCD0FFF74EFE04460D4681
:10198000FFF74AFE001B61EB0501B0F57A7F71F1AC
:101990000001F5D3EEE700BF340109087803090818
:1019A00000900020800601D5002933D10CB470B519
:1019B000194C1A49D4F8100382B007AB069A019368
:1019C00068F086FCD4F810536A7A32B12B686868E4
:1019D00005F10A01984700236B721148FFF74AFF8F
:1019E000B4F818633EB9012002B0BDE8704002B0FF
:1019F0007047013EF7D0FFF70FFE04460D46FFF794
:101A00000BFE001B61EB0501B0F57A7F71F100015F
:101A1000F5D3EEE700207047009000202DE100088C
:101A20007803090810F0400031D00CB470B50C46B2
:101A300082B029B1002002B0BDE8704002B070470A
:101A4000194ED6F810536B7A5A1C2B44D2B223216C
:101A50006A7299722B7A93421AD9069A134907AB84
:101A60002846019368F034FCD6F81043627A32B10C
:101A7000D4E9003004F10A01984700236372FFF7AC
:101A80004BFF012002B0BDE8704002B070477047C4
:101A9000002AE2D0D5E9003005F10A0198476C72BE
:101AA000D6F81053D9E700BF009000202DE10008C0
:101AB0000FB410B582B004AB0C4C53F8042BD4F81F
:101AC00010030B49019368F003FCD4F81043627AC9
:101AD00032B1D4E9003004F10A019847002363725F
:101AE00002B0BDE8104004B0704700BF0090002075
:101AF0002DE100082DE9F0413C4884B0FFF7BAFE23
:101B00003B4B1B6D5BB119689A880B691A4206D171
:101B10003848FFF7AFFE04B0BDE8F041FCE6364CB4
:101B20002368002B4AD09B699847002846D0236839
:101B3000002B59D0DB69DFF8E88098470646407CE7
:101B40003268337DB1790290307C0190708A0090C8
:101B500052082A48B51DFFF7ABFF00270B3601E0FE
:101B6000B54216D0D8F8104315F8011F637A5A1CF5
:101B70002344D2B262729972237A9342F0D8002A37
:101B8000EED0D4E9003004F10A019847B5426772FB
:101B9000E8D11B4C1B48FFF76DFE6378022B18D071
:101BA0000ED804F580541848FFF764FE94F8B43159
:101BB000022B15D0032BAED11448AAE71448A8E78E
:101BC000032BA8D11348FFF755FE04B0BDE8F04140
:101BD000A2E61148FFF74EFE04B0BDE8F0419BE6D7
:101BE0000E48FFF747FE96E79B79FFDE3C010908A8
:101BF0009428002048010908603B0020680109087A
:101C00009C4B002098010908C0010908E40109085B
